:020000040000FA
:040000006FD00400B9
:101000006F00104800000000000000009020002049
:10101000AA220020A9BDF9F56C23002000000000E1
:10102000000000006C230020902000200000000041
:101030000000000090200020000000009020002010
:101040000000000090200020902000209020002030
:101050009020002090200020F02B002094240020DD
:101060000000000090200020902000201E2400207E
:1010700090200020D22300209020002090200020EB
:101080009020002090200020902000209020002020
:101090009020002001A04111B7170040985F3AC688
:1010A000945F3247E39CE6FE3245410182800111A4
:1010B00013078008F337078093F787083EC20100C3
:1010C0000100B7170040930570052380B70413068D
:1010D00080FA2380C7040100010083C6B70493F699
:1010E000F60DA385D704238007049246F3A6068055
:1010F0000100010093760502D5CEF336078093F602
:10110000860836C4010001002380B7042380C70489
:1011100001000100B70614007D89558D88C70100C4
:1011200001000100010023800704A246F3A6068007
:101130000100010073370780137787083AC6010062
:1011400001002380B7042380C704010001000100CF
:1011500001003727004093061005A303D7802380A2
:101160000704B247F3A70780010001009307800836
:10117000F3B7078093F787083ECE01000100B71749
:101180000040130770052380E704130780FA2380CB
:10119000E7040100010003C7B70413670708A3852C
:1011A000E70423800704F247F3A70780010001004A
:1011B0000561828093760504BDC6F336078093F6F9
:1011C000860836C8010001002380B7042380C704C5
:1011D00001000100B7061400938606047D89558D31
:1011E00088C7010001000100010023800704C246F6
:1011F000F3A6068001000100733707801377870884
:101200003ACA010001002380B7042380C70401000B
:1012100001003727004093062005A303D7802380D1
:101220000704D24781B773370780137787083ACC12
:10123000010001002380B7042380C70401000100DE
:1012400098471367070C98C723800704E24719BF24
:101250000111814601468145114506CE97000000E7
:10126000E780605893078008F3B7078093F78708F3
:101270003EC601000100B717004013077005238028
:10128000E704130780FA2380E7040100010003C785
:101290006704136717002383E70423800704B2471A
:1012A000F3A7078001000100F2400561828041112F
:1012B000814601468145114597000000E780A05214
:1012C00013078008F337078093F787083EC40100AF
:1012D0000100B7170040130670052380C70493066A
:1012E00080FA2380D70401000100FD552396B70240
:1012F00023800704A245F3A5058001000100733790
:101300000780137787083AC6010001002380C704CD
:101310002380D7040100010003C767041367170087
:101320002383E70423800704B247F3A70780010063
:10133000010001A0BD473305F50201007D1575FDD3
:101340008280411122C426C206C6AA8401446317C2
:101350009400B24022449244410182800504130566
:10136000803E420497000000E78000FD4180C5B741
:101370009305000273A04580824573901534924016
:101380002242B2424243D2436244F2440255925551
:101390002256B2564257D2576258F25806499649D9
:1013A000264AB64A464BD64B664CF64C065D965DD1
:1013B000265EB65E465FD65F09617300203041113C
:1013C000B7170040985F3AC6945F3247E39CE6FE49
:1013D000324541018280B71700401307000323887C
:1013E000E7028547171700002326F7D47300203043
:1013F000411122C42D6426C24AC006C637190040D6
:101400001304A4AAB704002023208900974000E019
:10141000E78020299C408297974000E0E780602881
:10142000E5B737370040834747009146BD8B639E41
:10143000D702B73600401306F00F972500009385BA
:1014400065229727000083D7E73103C7A6001377EB
:10145000F70F1DE3B7E70400BC4F09468945171590
:101460000000034525A5829731A099466394D700D3
:10147000834757007300203003C786001377F70FA8
:10148000E365F6FC13851700AE9717280000231BB1
:10149000A82C2380E70075B7B787004003C7670013
:1014A000098B6309071003C77700930600031377BE
:1014B0000703630DD7081738000003483881172643
:1014C00000001306A67D0547B30606012380E6004B
:1014D00083C57700172700001307477E429793F5CF
:1014E000F50F2300B70003C58700972500009385FB
:1014F000E57BC2951375F50F2380A5000347070010
:1015000089451377F703630CB70C63E7E50A6306B5
:10151000071A8545630CB7129727000083C7177B0E
:101520003307F600034707001377F70F19CB85073A
:1015300093F7F70F3D476363F71A17270000A307D8
:10154000F778B787004009472383E700B787004053
:1015500083C77700E207E18763DE0704972700006F
:1015600083C7D77617270000130747733E97854632
:101570002300D70017270000130747743E979306F0
:1015800000032300D70017270000130727723E9798
:10159000A14685072300D70093F7F70F3D47636403
:1015A000F71417270000A303F772B7870040094715
:1015B0002383E70073002030930610026300D70EE8
:1015C000930620026305D70693060002E316D7F4BC
:1015D00003C727021377C70F13672700D5A803C7D0
:1015E00067001377070465CB03C7A702172800001D
:1015F0001308484C172500001305854313470708B7
:101600002385E70203C7A7021377370F1367870005
:101610002385E702814713070004B305F5008C41D9
:10162000B306F80091078CC2E399E7FEF5B503C74E
:10163000A702134707042385E70203C7A70213770E
:10164000C70F136727002385E702F9B503C76700B3
:101650001377070449C303C767021728000013085C
:101660002839172500001305653013470708238321
:10167000E70203C767021377370F136787002383D7
:10168000E702814713070004B305F5008C41B30658
:10169000F80091078CC2E399E7FEBDBD03C767025E
:1016A000134707042383E70203C767021377C70FB3
:1016B000136727002383E70285B503C76700137705
:1016C000070411CB03C727021377370F136787006F
:1016D0002381E70291B5238006003DBD97270000D6
:1016E000A386075EB9BD97270000A381075E75BD7D
:1016F0002303048015472303E48001002302A48010
:10170000828083076480E3CE07FE23030480828007
:1017100083076480E3CE07FE03454480828083070D
:101720006480E3CE07FE2302A4808280411126C498
:101730004AC24EC006C61377F50BAD47AA892E895B
:101740009544630CF700194597000000E78080FA84
:1017500097000000E78020FB8D444E859700000035
:10176000E78040F9FD59FD1463983401B240A2446A
:101770001249824941018280135509011375F50F01
:1017800097000000E780E0F92209F1BF011126CCA3
:1017900006CEB704080097000000E780C0F61545A4
:1017A00097000000E78000F597000000E78080F6D2
:1017B00097000000E78000F62AC697000000E78047
:1017C00080F432459377150089EB13651500137586
:1017D000F50FF240E24405618280FD14E9F0014515
:1017E000CDBF397126DC4ADA4ED852D656D45AD2F9
:1017F0005ED006DE62CE66CCB7E700E07D5783AAF6
:10180000070022C603AA470023A0E71823A2E7186F
:10181000B7170040130770052380E704130780FA09
:101820002380E70483C74704930B75FFB684E20760
:1018300093FBFB0F8546AA892E8B32893724004003
:10184000E187015763FA76016308D50089461307DB
:1018500000026313D5000157D98F93F7F70FB71C18
:1018600000402382FC0411472303E4801305F00F9A
:1018700097000000E78000E8094C97000000E7802F
:1018800080E863657C15B7050700DA9537870700A0
:10189000795563FEE504B3879500636AF704370B57
:1018A0000800A94733EB65016395F90881E8814495
:1018B00097000000E78020E5268515A8DA85094510
:1018C00097000000E780C0E605090345F9FFFD1415
:1018D000050B97000000E780C0E481C49377FB0FFD
:1018E000E5F797000000E780A0EA69F17D55B7179A
:1018F0000040130770052380E704130780FA238054
:10190000E70403C74704418B2382E704F250B7E79B
:1019100000E023A0571123A24711E2543244525948
:10192000C259325AA25A125B825B724CE24C21615C
:101930008280A547639BF90685691309F00FB306FA
:101940009900B3742B01B6941349F9FFB37499004D
:10195000856B33796901416B9387F9FFB3F72701F1
:1019600099E363FC340193D94900C147E3E637FFAB
:101970003DBF0569C1697D19D9B71305800D63881D
:101980006901130500026384790113051008CA85F3
:1019900097000000E780C0D997000000E78040DF93
:1019A00031D54E99B38434416DBFDA852D4597000A
:1019B0000000E780E0D7CA94E30B99EE0509970091
:1019C0000000E78020D5A30FA9FEFDB79387F9FF9C
:1019D00093F7F70F636DFC0C83C71C0413073008E3
:1019E0006315F706370708006361EB06B3079B0032
:1019F000B706100063FBD704334BEB0089476399AC
:101A0000F9068980D549E38404EADA850945970017
:101A10000000E780E0D111090327C9FF9147232087
:101A2000E48003076480E34E07FE23033481FD173F
:101A3000EDFBFD14110B81C49377FB0FE9FF9700B9
:101A40000000E780E0D461F155B5B717004003C747
:101A50005704B70708001377070219E3B787070091
:101A60007955E376FBE833079B00E3F9E7F841B5E6
:101A70008547E380F9F0DA852D4597000000E7807F
:101A800020CB9389F4FFE38404E297000000E78011
:101A900060C893F7390091EB83260480032709007F
:101AA00093074900E396E6E03E89CE84D9BFB54767
:101AB0006399F9001305900B97000000E78080C33D
:101AC000FDB3B1471305B00AE388F9FE9947639760
:101AD000F904B7050800B365BB002D459700000069
:101AE000E78000C581448D4BA14997000000E78045
:101AF00060C263967401832704802320F900850463
:101B0000E39534FF8327048013172B0163550700E7
:101B10002312F90069BB2322F90051BB9D47639F43
:101B2000F90281451305B00497000000E78040C02A
:101B3000BD442320090023220900FD59970000001D
:101B4000E78040BD93F77400CA9703C70700FD14F0
:101B5000398D2380A700E39334FF91BBA14763979E
:101B6000F90697000000E780A0C28144630D0B00D6
:101B70008D479304C0036308FB00930400056304CE
:101B80008B01930440041375C507E30295D21945F0
:101B900097000000E78000B697000000E780A0B63D
:101BA000054597000000E780E0B426859700000017
:101BB000E78020B7094597000000E78080B69700CE
:101BC0000000E780E0BCE31405CE0DB39147639FAE
:101BD000F9001305600697000000E780A0B19700A8
:101BE0000000E78040B213059009F9B5E38109CC04
:101BF000F1547DB9197106C212C416C61AC81ECA9C
:101C000022CC26CE2AD02ED232D436D63AD83EDABC
:101C100042DC46DECAC0CEC2D2C4D6C6DAC8DECAEC
:101C2000E2CCE6CEEAD0EED2F2D4F6D6FAD8FEDA9C
:101C3000970500009385854F8841E7000500924095
:101C40002242B2424243D2436244F2440255925588
:101C50002256B2564257D2576258F2580649964910
:101C6000264AB64A464BD64B664CF64C065D965D08
:101C7000265EB65E465FD65F0961730020300000C5
:101C8000972100209381013817510020130181B75B
:101C900017F5FFFF13054537970500209385853617
:101CA000171600201306C6FD63FAC500832205003F
:101CB00023A0550011059105E3EAC5FE1785000034
:101CC0001305058F97150020938585FB17160020B7
:101CD0001306462963FAC5008322050023A0550098
:101CE00011059105E3EAC5FE1715002013058527A8
:101CF00097350020938505006377B5002320050004
:101D00001105E36DB5FEFD42739002BC8D427390E8
:101D10004280B7220000938282887390023097023B
:101D200000209382222E93E2320073905230973239
:101D3000000093824280739012346FC0642C730051
:101D400020303D432A876373C3029377F700BDEFCA
:101D5000ADE5937606FF3D8ABA960CC34CC30CC71B
:101D60004CC74107E36BD7FE11E28280B306C34044
:101D70008A069702000096966780A6002307B700A0
:101D8000A306B7002306B700A305B7002305B700D5
:101D9000A304B7002304B700A303B7002303B700CD
:101DA000A302B7002302B700A301B7002301B700C5
:101DB000A300B7002300B700828093F5F50F939638
:101DC0008500D58D93960501D58D61B79396270033
:101DD0009702000096968682E78086FA9680C11761
:101DE0001D8F3E96E374C3F8A5B7B717004003C72D
:101DF00077051377E70FA38BE704130700F8A38D8C
:101E0000E7043D47238CE70413075003A38CE70442
:101E100003C7A7051377D70F238DE7048280B71771
:101E2000004003C7E7020D8941111377C70F498F9F
:101E300093068008F3B6068093F6860836C601003E
:101E40000100930670052380D704930680FA23804F
:101E5000D704010001002387E70223800704B2476B
:101E6000F3A70780010001004101828041112A830C
:101E7000014E930E407E130F0019930F400663E549
:101E80006E129308001913034006B3781503854EAC
:101E90000D4FA14F337365020D891335150063EFA4
:101EA000BE121308F6FF79467298420813580801CB
:101EB0003307C70213D61700BE0732976146B3F641
:101EC000C60213068070B386C6023697A166F58FE8
:101ED00042075D8FB716004083C7F60293F70708E5
:101EE000A303F1000346710083C7F60293F70708C6
:101EF000E394C7FE83477100B716004093F7F70FCE
:101F00006388071293078008F3B7078093F7870861
:101F10003EC401000100B7170040930670052380FE
:101F2000D704930680FA2380D7040100010023AA76
:101F3000070383C6170393E60608A388D702238006
:101F40000704A247F3A70780010001001166B71735
:101F500000407D16D45BC85F93854703A98EF18E40
:101F6000F5FA93068008F3B6068093F6860836C61F
:101F700001000100930670052380D704930680FAC0
:101F80002380D7040100010098C103C7170313671A
:101F90000704A388E70223800704B247F3A707805A
:101FA00001000100410182807D133368E30393083F
:101FB000E016630E08003368F3039308D016630835
:101FC00008009378330093B818009388D816330824
:101FD0001E01131E0801135E0E0155B56393E50340
:101FE0000548638608000148630303002A887108D6
:101FF0007298FD15131E0801C205135E0E01C18102
:1020000079BD13F8150063F4BF007908D5B713380C
:102010001800E5BF83C7F60293F70708A303F10092
:102020000346710083C7F60293F70708E394C7FEDF
:102030008347710093F7F70FF1DFE9B531714AD9A2
:1020400066CB06DF22DD26DB4ED752D556D35AD1DA
:102050005ECF62CD6AC96EC7AA8C02D89710000005
:10206000E78020B12A8993078008F3B7078093F7A8
:1020700087083EDA01000100B7170040130770051A
:102080002380E704130780FA2380E704010001009E
:1020900003C7F7021377770FA387E70203C7F70297
:1020A00013678700A387E70223800704D257F3A7AB
:1020B000078001000100054597000000E78060D619
:1020C000130780C13347E902116A93070AE89306B0
:1020D0005002BD69930BA004814A014B1304800890
:1020E000930470057D1AB347F9023307D7023EC047
:1020F000FD873ECC938709A69309803E3347F702BC
:102100003AC27D873AC4334739038549B399990167
:1021100093D93940B306D702B30B7703B3C6F6029F
:10212000B3CBFB0236C6FD8636C893D6FB4136CE0E
:10213000B7460F00938606243349D90285669386F5
:1021400006FAB3969601B389E9021307605533097D
:10215000D90293060010B389E9023349D902B3C901
:10216000F9029316390036CA37190040FD8636D079
:10217000930D090493D7F9413ED2F336048093F6C8
:10218000860836DC01000100930770052380FD00FE
:10219000930680FA2380DD000100010083463905A3
:1021A00093F6860FA309D9048346390593E61600F2
:1021B000A309D90423800D00E256F3A6068001008E
:1021C0000100130C80FA116DF336048093F6860833
:1021D00036DE01000100930770052380FD00238097
:1021E0008D010100010083463905216693E6060250
:1021F000A309D90483560905B3E6A6012318D90417
:1022000083560905D18E2318D90423800D00F25678
:10221000F3A60680010001008346390593F6060205
:102220006381061A03463905218A6DDE0818971066
:102230000000E78000987336048013768608B2C2E7
:102240000100010023809D0023808D010100010019
:10225000B717004003C637051376F60DA389C704E8
:1022600003C6370513660602A389C704835609050A
:102270002166B3E6A6012318D90483560905D18E39
:102280002318D90423800D009646F3A6068001008A
:1022900001008346390593F60602638B06148346D4
:1022A0003905A18AEDFE97000020E780C0DEAA86EE
:1022B00036D497000020E78000DEA256E30AD5FE60
:1022C000835609054255B3E6A6012318D904971091
:1022D0000000E780C08F83463905A18AEDDE0356F2
:1022E00009058346290582473376CA00B306DA0218
:1022F00093D5F641B296B388F640E24733B8C600AC
:102300002E983308F840A247B3B616013308D840D8
:1023100063C70701631DF800924763FA1701C247BC
:10232000634FF80E63950701B24763EAF80E8946DA
:1023300063E9660FF2469315180013D3F8015E8621
:1023400013951800B365B30042D646D497500000E9
:10235000E780E0D43258050B137BFB0F6347000185
:10236000631A0838A2586387083813081500B33673
:10237000A800B69513D6F5013298B336C800AE96CC
:1023800013581800FE06B3E6060173360480137670
:102390008608B2C60100010023809D0023808D01C4
:1023A000010001000356C902B296C206C18223167B
:1023B000D90223800D00B646F3A606800100010075
:1023C00021B5F336048093F68608B6C001000100FB
:1023D00023809D0023808D01010001008346390583
:1023E00093E60602A309D90423800D0086460DB5A5
:1023F000F336048093F68608B6C4010001002380FA
:102400009D0023808D01010001008346390593E67C
:102410000602A309D90423800D00A646BDB5E30B2F
:102420000BF0F336048093F68608B6C8010001006D
:10243000930680FA23809D002380DD0001000100C7
:102440008346390593F5FC0F93F6860FA309D9044B
:1024500083463905CD8EA309D90423800D00C646D5
:10246000F3A6068001000100130580FA0346390532
:10247000930639051D8A631C9629733604801376EA
:102480008608B2CC01000100130680FA23809D006B
:102490002380CD000100010003C606001376F60D6F
:1024A0002380C60003C60600136606022380C6000A
:1024B000835609051166D18E2318D9048356090560
:1024C0002166D18E2318D90423800D00E646F3A699
:1024D000068001000100130680FA8346390593F651
:1024E00006026380062683463905130C3905A18A46
:1024F000FDDA081897000000E780A06BF33604802F
:1025000093F68608B6D001000100930680FA238076
:102510009D002380DD000100010083460C00116650
:1025200093F6F60D2300DC0083460C0093E60602CA
:102530002300DC0083560905D18E2318D904835665
:1025400009052166D18E2318D90423800D008656F3
:10255000F3A6068001000100130680FA83463905C0
:1025600093F60602638A062083463905A18AEDFEAA
:1025700097000020E78020B22A8C97000020E78097
:1025800080B1E30C85FF8356090511664255D18E53
:102590002318D90497000000E7806063834639055B
:1025A00013063905A18AFDDAF336048093F686080E
:1025B000B6D401000100930680FA23809D00238099
:1025C000DD00010001008346060093F6F60D2300AE
:1025D000D60023800D00A656F3A606800100010058
:1025E0008356090503462905D247B376DA00330638
:1025F000CA021305800C9355F6413696330DF6400A
:102600008257333CD6002E9C3336A601330CFC4057
:10261000330CCC403308850392564E86B335A50360
:102620003305A503C29597500000E78040A7634695
:102630008001631E0C16630C0D161306150033354E
:10264000A6002E959356F5013696B335D600AA9579
:102650009396F50105828585D18E6346B000639D12
:10266000051A638B061A0356C90215823305D60074
:102670003336C500B2956348B00063910524130654
:10268000F00F637DA622894663F3561593078008F1
:10269000F3B7078093F78708BED60100010037170C
:1026A0000040930770052300F704930780FA230086
:1026B000F704010001008356C70289678117D58F8F
:1026C000C207C1832316F70223000704B657F3A7F6
:1026D000078001000100FA506A54DA544A59BA5985
:1026E0002A5A9A5A0A5BFA4B6A4CDA4C4A4DBA4D4E
:1026F000296182801308F5FF3335A800FD152E955A
:102700001356F5013298B336C800AA9695B9F33638
:10271000048093F68608B6CA0100010023809D005C
:102720002380AD000100010083463905CD8EA30949
:10273000D90423800D00D646F3A6068001000100CF
:1027400035B3F336048093F68608B6CE0100010057
:1027500023809D002380CD000100010083463905C0
:1027600093E60602A309D90423800D00F646F3A6DA
:1027700006800100010095B3F336048093F68608C5
:10278000B6D20100010023809D002380CD0001000E
:1027900001008346390593E60602A309D904238084
:1027A0000D009656F3A606800100010045BB930676
:1027B000F5FF33B5A600FD152E959355F501AE96A0
:1027C000B3B5B600AA951396F501858269B5F336BF
:1027D000048093F68608B6D801000100930680FABB
:1027E00023809D002380DD00010001008356C90283
:1027F0000566011693F6F60FD18EC206C182231626
:10280000D90223800D00C656F3A606800100010000
:10281000850A93FAFA0F95B233E6B60045C203561D
:10282000C9023305D0403338A000B305B040B385AA
:10283000054115826345B000D1E16371A608894660
:1028400063F0560593078008F3B7078093F787086E
:10285000BEDA01000100B71700401307700523809E
:10286000E704130780FA2380E7040100010003D77F
:10287000C7027D8B2396E70223800704D65781BDCC
:10288000F336048093F68608B6DC01000100930657
:1028900080FA23809D002380DD0001000100835623
:1028A000C9020566011693F6F60FD18EC206C182E3
:1028B0002316D90223800D00E656B9B79307800886
:1028C000F3B7078093F78708BEDE010001003717D2
:1028D0000040930770052300F704930780FA230054
:1028E000F704010001000356C70293975600B29700
:1028F000C207C1832316F70223000704F657C1BBA2
:10290000914763EEB70217670000130727138A0584
:10291000BA959C41BA978287B717004003A7470B27
:102920001345F5FF698F23AAE70A03A7070B698FF1
:1029300023A8E70A03A7070A798D23A0A70A8280A4
:10294000B717004083A6470B1347F5FFF98E23AA5C
:10295000D70A83A6070B558D23A8A70A83A6070AC3
:10296000758F23A0E70A8280B717004003A7470BA3
:10297000498F23AAE70A03A7070B1345F5FF45BFB5
:10298000B717004083A6470B1347F5FF758F23AA9F
:10299000E70A03A7070A598D4DB7B717004003A7E9
:1029A000470B498FEDB7914763EEB70217670000F9
:1029B0001307070A8A05BA959C41BA978287B71709
:1029C000004003A7470D1345F5FF698F23AAE70CC5
:1029D00003A7070D698F23A8E70C03A7070C798DC0
:1029E00023A0A70C8280B717004083A6470D13478A
:1029F000F5FFF98E23AAD70C83A6070D558D23A8C2
:102A0000A70C83A6070C758F23A0E70C8280B7174D
:102A1000004003A7470D498F23AAE70C03A7070D22
:102A20001345F5FF45BFB717004083A6470D134771
:102A3000F5FF758F23AAE70C03A7070C598D4DB737
:102A4000B717004003A7470D498FEDB7797122D41E
:102A50003714004026D24AD003592402835404027A
:102A600006D64209C2044ECE52CC56CA13590901A9
:102A7000C1802DE11379F9F793F4F49F4209C20460
:102A800013590901C18093078008F3B7078093F7B2
:102A900087083EC401000100930770052300F40479
:102AA000930780FA2300F40401000100231124039A
:102AB0002310940223000404A247F3A70780010017
:102AC0000100B250225492540259F249624AD24A49
:102AD00045618280B7F5070081463000B105194590
:102AE00097000020E780E0CFA24713972701E34A31
:102AF00007FC1369090893E4044093098008F3B7BD
:102B0000098093F787083EC001000100930A700511
:102B100023005405130A80FA230044050100010034
:102B20002311240323109402230004048247F3A7F3
:102B3000078001000100294597F0FF1FE780807F93
:102B4000F3B9098093F989084EC2010001002300FE
:102B5000540523004405010001008357040293E754
:102B600007202310F402230004049247B9B7B717D3
:102B700000408847420541819377050491EB9377A4
:102B8000F5013755E801130505803345F5028280CC
:102B90009377050C130700046397E7009377F5011B
:102BA00037459C1CCDB72165130505D0828037E7DA
:102BB00000E01C435443A183E206D58F1CC1FD579E
:102BC0002320F7182322F718828013178500B7E710
:102BD00000E023A0E710618123A2A7108280B7F74D
:102BE00000E08847CC478280814737370040A146C4
:102BF00063C4C700328582800345B740E38EA6FEDA
:102C00003385F5000345050085072304A740CDB7AC
:102C1000970700209387C7069C43172700201307B8
:102C2000670D3E95636EE500174700201307878DFB
:102C30006368A700170700202324A7043E8582802D
:102C4000FD57EDBF8280411122C406C62A84970039
:102C50000000E78000F22947B307E502B2408D8308
:102C6000B3D7870222449507B3D7E702373700402E
:102C7000C207C1832316F700410182804111371535
:102C80000E0006C697000000E78020FCB737004022
:102C9000130770F82381E7000D47A381E7001307AE
:102CA0000004A380E70005472387E700B240410105
:102CB000828037370040834727001A0593F7F703D0
:102CC000C98F93F7F70F2301F7008280B7370040D1
:102CD00003C7170019C9D98DA380B70003C7070020
:102CE000136787002380E700828093C5F5FFF98D85
:102CF000A380B7008280AE872A87B736004021467E
:102D00003738004089E7170300006700E3F383C802
:102D1000B600E30916FF05078348F7FFFD17C20752
:102D200023041801C183F9BF411122C406C62A84B5
:102D300097000000E780E0E32947B307E502B240CF
:102D40008D83B3D7870222449507B3D7E70237377D
:102D50000040C207C1832316F7404101828071659C
:102D600041111305052006C697000000E78000FC0E
:102D7000B7370040130770F82381E7400D47A38160
:102D8000E74013070004A380E74005472387E74097
:102D9000B24041018280CC41411106C6328503C652
:102DA000150083C5050022064D8E42068D654186BD
:102DB000138875A2630C0611634BC804138845A2DF
:102DC0006300060D634AC800938535A26301B60807
:102DD0002390060029464DA0138855A26305060DD1
:102DE000938565A2E316B6FE8D451D4663E6E508AC
:102DF0001146198E63F3C7003E86B7E7040023909F
:102E0000C600FC47976500009385C5C69DA0138842
:102E100095A263030611634E060D1388A5A26300F5
:102E20000613938505A5E315B6FA99451D4663E596
:102E3000E504198E63F3C7003E86B7E704002390CC
:102E4000C600FC47970500209385C5ED1DA09D4554
:102E50001D4663E3E5022146198E63F3C7003E86F3
:102E6000B7E70400FC472390C60097050020938530
:102E7000E50FBA9582970146B240328541018280C2
:102E8000AD451D46E3EAE5FE3146198E63F3C70002
:102E90003E86B7E704002390C600FC479765000014
:102EA0009385C5BFF9B7B1451D46E3E7E5FC354657
:102EB000198E63F3C7003E86B7E704002390C6006F
:102EC000FC4797650000938565BE65B78D451D4637
:102ED000E3E4E5FA1146198E63F3C7003E86B7E7CF
:102EE00004002390C600FC4797650000938545B910
:102EF00049B78D451D46E3E1E5F81146198E63F3A8
:102F0000C7003E86B7E704002390C600FC479765DC
:102F10000000938565BBB1BFA5451D46E3EEE5F412
:102F20002946198E63F3C7003E86B7E70400239055
:102F3000C600FC4797650000938545B51DBFB545A4
:102F40001D46E3EBE5F23946198E63F3C7003E8672
:102F5000B7E704002390C600FC47976500009385FF
:102F600065B001BFB7E7040003A30713970600206D
:102F7000938646DA4146A54517050020130585D0FE
:102F800002832D455DE703C505000947631FE5087A
:102F900003A84500411106C60347180032850346C1
:102FA000080022074168518F930828FE6307170520
:102FB00063E9E80005186303070323900600294529
:102FC00091A8130648FE630AC7041518E31707FF04
:102FD00015463E87637BF600154701A813060002DD
:102FE0003E876374F60013070002B7E704002390DE
:102FF000E600FC471316070111A83E8691C305465B
:10300000B7E70400FC472390C6004206CC45418246
:1030100082970145B24041018280130600083E8735
:10302000E375F6FC13070008C9B7239006000545B1
:1030300082808280416779176304E504411122C4CC
:1030400006C685472A84639FF500B7E704002285FA
:103050002244B24003A38713970500209385450BB4
:103060004101028389476399F500B7E7040083A70C
:10307000070B8545829771D9B24022444101828075
:103080008280797126D252CCAE842A8A976500005C
:10309000938585A517650000130585A706D63AC652
:1030A00022D44AD0368432894ECE97400000E78041
:1030B000404AA28517650000130585A697400000C9
:1030C000E7802049294597400000E780604D83C78D
:1030D000840093F70702F9E383C904008947054593
:1030E00032476396F908D44083C7160083C60600AA
:1030F000A207D58FC166138616FE638CC7028D1694
:10310000638FD7068D669386269029456391D706EF
:10311000B7E70400A286225403A34714B250F24931
:103120004A86A685025992545285624A854745616E
:1031300002832D450DEF93070002354563E98702B1
:10314000B7E70400FC47C84413060002CA8582970B
:10315000814997070020938767FC9C43014581CBF9
:103160009C4391C74E852286CA8582970145B250FD
:10317000225492540259F249624A456182802D4597
:103180007DF79307700F3545E3E387FEB7E704004B
:10319000FC47C8442286CA85829765BF2145C1BFC6
:1031A000411122C437E404008327841326C2AA8471
:1031B000416506C697050020938585F57D158297A4
:1031C0008327C40A17050000130505E78588829741
:1031D00095C0032304132244B24092449706002072
:1031E0009386C6C54146C54517050020130505B49D
:1031F00041010283B2402244924401454101828050
:1032000019C59707002023ABA7F0014582804545EB
:1032100082801147636AA70A976600009386868BAF
:103220000A0536951841411106C63697AE87B28514
:103230000287130700026145639DE700B7E70400BA
:10324000FC4713060002170500201305A5D282973C
:103250000145B2404101828005476145E39BE7FE9D
:10326000B7E70400FC47054617050020130585D283
:10327000F9BF1307700F6145E39DE7FCB7E7040052
:10328000FC471306700F170500201305E5D0C1B7E2
:10329000130700086145E39EE7FAB7E70400FC471F
:1032A0001306000817050020130585DE4DB71547E6
:1032B0006145E390E7FAB7E70400FC4715461705B8
:1032C0000020130525E561B709458280411126C21A
:1032D000B7E4040083A7C41322C44AC006C62E84E0
:1032E000970500209385C5E22A898297058905C53F
:1032F00097070020938787A383D7A70BA28503A3F3
:10330000440D2310F4002244B24092444A850249FD
:10331000014641010283B240224492440249494598
:103320004101828097070020238C07DE9707002049
:1033300023AA07DEB717004003A7070CB706C0FF94
:10334000FD16758F23A0E70C03A7070DB7064000F5
:10335000558F23A8E70C03A7070C3D9B23A0E70C80
:1033600003A7070D1367070123A8E70C8280B7178F
:10337000004003A5470C83A7470C5981134515004E
:10338000C18B058999E3136525009707002083C742
:1033900027D96380A702970700202383A7D811C9E4
:1033A00097070020938707D803A307006303030050
:1033B00002838280114517F3FFFF670063C8011184
:1033C00022CC06CE3714004026CA4AC84EC652C484
:1033D00083447405034AB40583498405034994056D
:1033E00097F0FFFFE780A0A08347A40593F4F40FB4
:1033F000137AFA0F93E71700230DF40493F9F90FEA
:103400001379F90FB717004003C7A705058B6DFFA8
:1034100003D5C705A38D4705238C3705A38C270546
:10342000A38B9704F2406244D2444249B249224AF3
:103430000561828041119397050122C406C626C208
:10344000C1872E8463DC0700B7E40400FC54829734
:1034500019C1BC5482972165218D15A893F71500D9
:1034600013C515008DE793F725009DC79700000051
:10347000E78020F0B7E70400BC4F1306000A894537
:1034800017050020034585CA829713452400B240E2
:1034900022449244410182809397250163D8070218
:1034A000B7E4040083A7C41E829797000000E7805A
:1034B000A0F0BC4C37560700130606308965170587
:1034C00000200345A5C68297096579B79397150132
:1034D0000145E3DE07FA175500001305656C9740B8
:1034E0000000E780E01EB7E70400BC4F130600644D
:1034F000916517050020034565C382971165A9BF33
:103500001D71A2CC37E404005C5C485886CE494665
:103510009755000093854564829711E9175500007F
:103520001305C56497400000E780801A01A0B7F634
:1035300000E0795798CAFD57DCCA0567B7E700E095
:1035400023A0E7101306F00290C223A0E7180100A1
:10355000010037070020184713060004814597062D
:10356000002023A3E6BC4157A38AE7403C44080857
:10357000829797070020938767CE3EC88567138799
:103580000740938757D1231AE1002312F102130752
:10359000B00F97F7FFFF9387C7642310E1023ED86F
:1035A0001547970700009387C7E1B7F50700A30FFA
:1035B000E1003EDC0547970700009387E7DF81467F
:1035C0003000E10519452301E1023EDE97F0FF1FBF
:1035D000E780202118088147994630003E9603462F
:1035E000060085070507A30BC700E398D7FEC2476F
:1035F00091C70357410185676373F70001A0B7E7DF
:10360000040083A7470A08088297AA8511C917559D
:1036100000001305E55697400000E78080F301A005
:10362000F640664425618280411126C2B7E4040059
:1036300083A7040806C622C4170500001305C5DFCA
:10364000829717040020130464AE2300A40097009F
:103650000000E780800297000000E780E0CC03458F
:103660000400224403A38405B240924413060032AE
:10367000896541010283797106D622D41307800837
:10368000F337078093F787083EC201000100B717A0
:103690000040930570052380B704130680FA238049
:1036A000C7040100010083C6F70293F6A60FA387A3
:1036B000D702238007049246F3A60680010001008A
:1036C00073370780137787083AC40100010023800D
:1036D000B7042380C7040100010003C7F702136782
:1036E0002700A387E70223800704A247F3A70780E8
:1036F00001000100054597E0FFFFE7808072970019
:103700000000E78060CB014781468147054685453B
:103710001305407E97E0FFFFE780807537E40400E3
:103720003C446800514681458297B707C0A83EC80F
:10373000B787E803938707D03ECA97F7FF1F9387A1
:1037400007C83EC67C5868008297B2502254456133
:10375000828009CDB7E70400BC47411106C6414647
:1037600081458297B24001454101828001458280B6
:10377000B7F5070001118146170600201306869B46
:10378000E105194506CE22CC97F0FF1FE7806005C2
:1037900037E404008327041A829797300000E780FB
:1037A000C03E8547A307F100832744171306F100A5
:1037B0008545130550308297175500001305853E47
:1037C00097400000E780C0F0F240624405618280CB
:1037D0008280411122C491462A84170600201306D4
:1037E00066A69D652D4506C697F0FF1FE78060FF22
:1037F000B7F7070003C70701A5476313F70001A048
:103800009306001001469D65254597F0FF1FE78050
:1038100040FD97070020238787A22244B2409146AB
:1038200017060020130606A29D652945410117F3DE
:10383000FF1F670003FB1171CED7B7E9040083A710
:10384000C904CAD9170900201309C98FA2DD2E8621
:1038500086DFA6DB2E84AA854A85829797070020FB
:1038600083C7478E1307700A6385E710636DF700FF
:103870001307600A6385E704FE506E54DE544E5908
:10388000BE59116182801307800A6385E71613070A
:10389000900AE393E7FE8D476306F41C97550000FA
:1038A0009385053C175500001305852697400000B9
:1038B000E78020CA175500001305C53725A08D479E
:1038C000630CF40297550000938585391755000065
:1038D0001305052497400000E780A0C71755000096
:1038E0001305852E97400000E780A0C62945974024
:1038F0000000E780E0CA49B7854717550000130567
:10390000652E17070020230AF78297400000E78002
:1039100020DCB7750200B76602000146054597F046
:10392000FF1FE78000EC930760F817070020230BC8
:10393000F78097070020A3880780930700261707C2
:1039400000202323F780E5779387072117F7FF1FD0
:10395000231EF77EB14597F7FF1F238A077E97F74F
:10396000FF1FA386A77E4A8597000000E780E01628
:1039700021B7914763E38702975500009385452E51
:10398000175500001305C51897400000E78060BC7C
:103990001755000013050527B1B797F4FF1F83C41F
:1039A000A47A97F7FF1F83C7177AA204DD8C83A739
:1039B000C9046D14228697F5FF1F9385F5782800BA
:1039C00082978E0493160401B7750200C1823000FD
:1039D000A695094597F0FF1FE780A0E0930770F8D0
:1039E00017F7FF1F2300F776994597F7FF1FA38D61
:1039F000A77495BF914763E38702975500009385AD
:103A00002526175500001305A51097400000E780F4
:103A100040B41755000013056520E9B597F4FF1F62
:103A200083C4847297F7FF1F83C7F771A204DD8CEC
:103A300083A7C9046D14228697F5FF1F9385D5705F
:103A4000280082978E0493160401B7750200C18284
:103A50003000A6950D4597F0FF1FE78080D89307AB
:103A600080F8BDBF175500001305051E97400000E4
:103A7000E78000C6930790F82304F10083471900FC
:103A80008D452800A304F100834729002305F10098
:103A900097000000E78060041305C01297F0FF1F35
:103AA000E780208A014597F0FFFFE78080100D45F1
:103AB00097000000E78020D2294597F0FF1FE7809C
:103AC000408897E0FF1FE780A0787DB397F7FF1F3E
:103AD00023A2A778828097F7FF1F9387A77703A376
:103AE0000700630303000283173300006700A3305D
:103AF00041114AC09716002083D6A6C6328917F610
:103B0000FF1F0356063B22C426C206C62A84AE8483
:103B100097000000E780206629C921C8994763F60D
:103B200097048347140003470400A207D98F139713
:103B30008700A183D98FC2073167C1831307C75597
:103B40006395E70297F7FF1F83D7A736A301F40019
:103B5000A1832302F4009717002083D787C091C761
:103B6000A302F400A1832303F400630D0902971755
:103B7000002083C7A7AE9DE797F7FF1F83C7C76DD8
:103B800095C38DC097F7FF1F83C7275B81EF228501
:103B90002244B2400249A6859244410117330000F5
:103BA00067006325B2402244924402494101828069
:103BB0008347550083454500175500001305050D43
:103BC000A207DD8D174300006700A398175500007A
:103BD0001305C50A17430000670083AF8D4763F6DE
:103BE000B708011126CA06CE22CC0344350097F44B
:103BF000FF1F83C47466975500009385650AB33729
:103C0000800017F7FF1FA309F76409C49755000048
:103C10009385C509175500001305C5099740000095
:103C2000E780209397F7FF1F83C71763638697008A
:103C300097000000E780004397300000E780A04530
:103C40009967938757EE2316F100680085479145E1
:103C5000A30781002307F10097000000E780E0E759
:103C6000F2406244D244056182808280894763F7D2
:103C7000B708011122CC06CE26CA83442500854709
:103C80002A84639DF404914763F5B7040345450016
:103C90008347340022055D8D97F7FF1F239BA720E4
:103CA00097000000E78000569967938767EE23141A
:103CB000F1008347340023059100A305F1008347F9
:103CC0004400954528002306F10097000000E78096
:103CD000C0E0F2406244D24405618280FDF89967F9
:103CE000938767EE2314F10097F7FF1F83D7671CB4
:103CF000A305F10023050100A183E1B78280011132
:103D0000996722CCD5171714002013042495231487
:103D1000F1008347040026CA97140020938464A40A
:103D20002305F10083D7040028009545A305F10081
:103D3000A18306CE2306F10097000000E780E0D9BA
:103D400003D604008345040017550000130585F7CA
:103D500097300000E780E07FF2406244D244056182
:103D600082809D677971D9172316F100971700207B
:103D70009387C78E83C707001305F10006D6230774
:103D8000F10097000000E780009D09E9B7E7040013
:103D9000BC47414681451305F10082976800CD4537
:103DA00097000000E78060D39715002083C5058B3E
:103DB00017550000130505F497300000E78060797F
:103DC000B250456182806308051641114AC006C69B
:103DD00022C426C297F7FF1F83C717481719002070
:103DE0000349C98799C3136929002A8497100000E1
:103DF000E78040F79364490119E19364490037E98A
:103E000004008327890422851306200381458297B5
:103E1000930750FA2300F4009307A005A300F400D1
:103E20008D472301F4009147A301F4009307800418
:103E3000A302F4009717002083D7A7922304F4006D
:103E4000A18393E40402A304F40097F7FF1F83D730
:103E50004706230394002305F4009304C400A183C0
:103E600023020400A305F400268597000000E780E4
:103E7000808E19E5832789044146814526858297EE
:103E8000FD57230EF400A30EF40093070002230F46
:103E9000F400930710FAA30FF4009D472300F402E7
:103EA000A3000402B7E70400FC47130524021946E7
:103EB00097F5FF1F93850528829797F7FF1F83D7F4
:103EC00027282304F402A183A304F40297F7FF1F19
:103ED00083D7C7262305F402A183A305F40297F72D
:103EE000FF1F9387C725839707002285930500034B
:103EF0002306F402C207C183A183A306F40297F745
:103F0000FF1F9387C7FA839707002307F402C207AE
:103F1000C183A183A307F40297000000E780A021DA
:103F20002308A4022181A308A402B240224492449F
:103F300002494101828082805D71E17793C777FFFA
:103F40001305E10086C62316F10097000000E78004
:103F5000C0E768009305400397000000E780E0B7E2
:103F6000B640616182805DC9411122C426C206C685
:103F7000930750FA2300F5009307A005A300F5006E
:103F800089472301F5009147A301F50093078004B9
:103F9000A302F500970700209387476C83C70700AB
:103FA0009304C5002A842303F50097F7FF1F938726
:103FB000B72A83C7070023020500A303F50097076C
:103FC000002083D7077A2304F500A183A304F5001A
:103FD00097F7FF1F83D7E7ED2305F500A183A3051E
:103FE000F500268597F0FFFFE780E07601E9B7E767
:103FF0000400BC4741468145268582972285F145CC
:1040000097000000E7802013230EA4002181A30E57
:10401000A400B240224492444101828082805D71BA
:104020000A8586C6A2C497000000E78000F437E442
:1040300004007C448A850810794682973C44130525
:10404000E10309468145829710109305000201455E
:1040500097F0FFFFE780201CB64026446161828014
:104060000111B7C7A55A22CC9387C73317F4FF1F96
:104070001304941E3EC48347040085660146996577
:10408000254506CE3EC697E0FF1FE78080753000CD
:10409000A1469965294597E0FF1FE7808074834515
:1040A000040017550000130565CF97300000E78026
:1040B000404AF2406244056182800111A14630000D
:1040C00099652D4522CC06CE97E0FF1FE7806071F1
:1040D000A24737C4A55A1304C43363958702B24577
:1040E00017550000130545C3B335B00097F7FF1F00
:1040F000A384B71697300000E780A045F2406244E1
:10410000056182809165A1463000938505F02D45BB
:1041100097E0FF1FE780E06CA247E38287FC97F7F8
:10412000FF1FA38B0712814517550000130505C11A
:10413000D1B7C16769768146FD1705061397060159
:1041400041836364B7003E8582803307D50003470F
:104150000700B98F214713F817008583630508000E
:10416000B18FC207C1837D171377F70F6DF78506EF
:10417000F1B741C5A547054763F2B7088347150066
:10418000034705003168A207D98F13978700A183E1
:10419000D98FC207C1831308C85505476390070725
:1041A000411106C622C426C203442500914763F08C
:1041B00087049307540063ECF502A301C500218234
:1041C0002302C5009304340091C6A302D500A18246
:1041D0002303D5002A84A68597000000E780A0F578
:1041E00026942300A4002181A300A4000147B2402B
:1041F000224492443A854101828005473A85828073
:104200000111B7C7A55A22CC9387E7342A842AC65E
:10421000856601469565254506CE3EC497E0FF1F9D
:10422000E780205C3000A1469565294597E0FF1F97
:10423000E780205BA28517550000130525B897304D
:104240000000E780003197000000E78080DDF24049
:104250006244056182800111A146300095652D45BB
:1042600022CC06CE97E0FF1FE780A057A24737C4B5
:10427000A55A1304E43463958702B245175500002C
:104280001305C5AD97F7FF1F2395B7C2C205C181BE
:1042900097300000E780E02BF240624405618280A5
:1042A0009165A1463000938505EE2D4597E0FF1FEF
:1042B000E7802053A247E38287FCD14717F7FF1F0F
:1042C0002319F7BED14517550000130525ABC9B713
:1042D00021C1411126C206C622C4AE848DC52A84DE
:1042E00097100000E780A0A897F7FF1F83C7C7F6C5
:1042F00099CB22852244B240A685924441011733CE
:104300000000670043AFB2402244924441018280E2
:10431000828001114EC606CE22CC26CA4AC893F727
:104320001500AE899DCBAD67371700409387A7AACC
:104330001CC3B7E70400BC4F13060019854517F5E9
:10434000FF1F0345E5B6829713C51900F24062448A
:10435000D2444249B2490561828093F72500014564
:10436000F5D7170700200357A73F954763F9E70CD8
:104370000144170600201306A62E930630051305E8
:104380005004130810049308B00413039005930716
:1043900064006374F7043A847D599704002083C451
:1043A000242C9707002083C7B72BA204DD8CAD67B0
:1043B0009387B755638BF41463E3970AA9679387D0
:1043C000A755638EF414A28517050020130545290F
:1043D00097000000E78000F0E9A0B307860083C5DE
:1043E0000700639AD50483C517006396A50483C5A7
:1043F00027006392050583C53700639ED50283C5F8
:104400004700639A150383C75700639667022289A2
:104410000DE89705002083D5A534B3852541C20555
:10442000170500201305C523C1814A959700000098
:10443000E78040EAE1A005044204418089BF3A8454
:104440007D598547E3EB87F45DC48545170500205A
:104450001305052197000000E780C0E769A8B16750
:104460009387C7556389F404B5679387D755E39C51
:10447000F4F4A285170500201305851E973000006F
:10448000E78060978947630EF4009305E4FFC20557
:10449000C181170500201305C51C97100000E78097
:1044A000008DA68517550000130505939730000071
:1044B000E780200A89A097200000E780401E97101F
:1044C0000000E780208A11C9A28517050020130586
:1044D000251997100000E78080890546A2851705F9
:1044E00000201305E51797F0FFFFE780A0609720F5
:1044F0000000E780C01AFD57E31DF9F09707002080
:104500002390072613C5290091B5A2851705002021
:104510001305051597F0FFFFE780C06959B7A2851D
:10452000170500201305C51397F0FFFFE780406AC9
:104530008DBF4111054506C622C426C297E0FFFF84
:10454000E78000511305A00497E0FF1FE78020B625
:10455000757585457D1597E0FFFFE780A03A7D756D
:1045600085451305F53697E0FFFFE78000443714D3
:1045700000408327840A8D451305002093E7072018
:104580002324F40A97E0FFFFE780C037B7E4040074
:1045900097E0FFFFE780E07CC85897300000E78095
:1045A00020138327840C8545414593E7070823247E
:1045B000F40C97E0FFFFE780403F8D4513050008AE
:1045C00097E0FFFFE780603E97E0FFFFE780406BEA
:1045D00037A507001305051297E0FFFFE780E066A7
:1045E000014597E0FFFFE780006D95450545894748
:1045F000170700202308F71697E0FFFFE780406DBC
:10460000B7E700E013070006238DE74037070004F3
:1046100023A0E71097F0FFFFE780C0EE97F0FFFFC1
:10462000E780C00097000000E78060A997000000C5
:10463000E780A0C297F0FFFFE780C013970000005B
:10464000E780207497000000E780000383A7040838
:1046500017050000130525CC829797F7FF1F2389C4
:10466000A784BC4C130600648545829797E0FF1F22
:10467000E78000D841110D658D4506C697E0FFFF24
:10468000E7804028B71700408D6623A6D70A170594
:1046900000201305650D1387C70A9387870A1CC17D
:1046A0005CC5856689675CC958C114C518C9B7E778
:1046B0000400B24003A3871E410102838145B30772
:1046C000B5008387070089E7172300006700C3034D
:1046D0008505C205C181E5B7011106CE230701009A
:1046E00001ED175500001305258E97000000E780A7
:1046F00020FDF240056182805800A947BA8529460D
:104700002548B376C502FD1793F7F70F9386060386
:10471000A304D700B356C5026375A8007D1736857C
:10472000EDF33385F500D1B7975700009387078ADB
:104730001357C5003E9703470700011106CE230417
:10474000E100135785003D8B3E9703470700230682
:104750000100A304E100135745003D8B3D893E97BE
:10476000AA970347070083C7070028002305E10035
:10477000A305F10097000000E78080F4F240056196
:1047800082807971174500001305057E06D622D474
:1047900026D24AD04ECE97000000E78060F217057F
:1047A0000020035505FC97000000E78020F89707DC
:1047B000002083C7A7EA174500001305657889C75D
:1047C000174500001305457797000000E78040EF8C
:1047D000174500001305857997000000E78040EE3B
:1047E000174500001305057997000000E78040EDAC
:1047F000114597000000E78060EE17550000130593
:10480000E5B697000000E780A0EB014597000000A7
:10481000E780C0EC17550000130545B59700000070
:10482000E78000EA1305800497000000E78000EBB2
:1048300097F7FF1F83C757A2174500001305C570E0
:1048400089E7174500001305A57097000000E78071
:1048500020E7174500001305657297000000E78008
:1048600020E637A507001305051297000000E78032
:10487000E0E6174500001305E57097000000E780AB
:1048800020E49707002083C7A7EF17450000130512
:10489000A56C89E7174500001305856C970000009B
:1048A000E78000E2174500001305856E97000000C1
:1048B000E78000E1174500001305056E9700000032
:1048C000E78000E017E5FF1F0355A55E9700000095
:1048D000E780C0E5174500001305856C97000000D0
:1048E000E78000DE17F5FF1F035585859700000060
:1048F000E780C0E3174500001305056B9700000033
:10490000E78000DC17F5FF1F035545839700000083
:10491000E780C0E117450000130585699700000096
:10492000E78000DA17F5FF1F035565819700000047
:10493000E780C0DF174500001305C567970000003A
:10494000E78000D817E5FF1F035565569700000064
:10495000E780C0DD1745000013054566970000009D
:10496000E78000D6014497E9FF1F9389A97C97440B
:1049700000009384A4651949B307340183C7070075
:104980000A85050413D74700BD8B2697A6970347D2
:10499000070083C70700230101002300E100A300F3
:1049A000F10097000000E780A0D1E31724FD174530
:1049B00000001305256197000000E78060D00A859C
:1049C00097F0FFFFE78020D90A840408834704009A
:1049D000034514000904A2075D8D97000000E780DD
:1049E000E0D4E39584FEB250225492540259F24925
:1049F00045618280411126C2E977970400209384A3
:104A000064EC22C49387A7552E842381B4002E869C
:104A1000AA8517050020130525EB06C62390F40090
:104A2000A381040097300000E78040A7930524008D
:104A3000C205C181170500201305E5E897F0FFFFC7
:104A4000E780606FB38784002382A7002181A3825F
:104A5000A700930564002244B24026859244C20513
:104A6000C181410117230000670003CA09C99307E8
:104A7000000463E6B700170300006700E3F78280D5
:104A80009306F0030307060019E79307F00363F0AA
:104A9000B7022E85828093871500C207C183E3E6A3
:104AA000F6FEAA952380E5000506BE85E1BF2E959A
:104AB00023000500F9BF5971B7064000A2D486D67D
:104AC000A6D2CAD0CECE170700201307A7CB014429
:104AD0005946A5066304A42883470700BA84D9175A
:104AE00093F7F70F6367F600B3D7F600858B0507DA
:104AF00085EF3304854042044180BD4763EA870265
:104B00000147631FF4063D46974500009385C5366F
:104B1000268597300000E7800096014735E117456C
:104B200000001305653625A00504420441805DB7E9
:104B30004146974500009385A531268597300000B2
:104B4000E780609369F1174500001305A5319700D0
:104B50000000E780E0B697000000E780C0C217457C
:104B600000001305E53A97000000E78060B585472F
:104B7000B650265496540659F6493E8565618280A2
:104B8000B70640005946A506B387E40083C707006F
:104B9000131507014181D91793F7F70F636FF600DB
:104BA000B3D7F600858B91CB050705059317070151
:104BB0004205C1834181E3E987FCB309A440C209EE
:104BC00093D90901A14763F937133389A400254616
:104BD000974500009385852C4A8597300000E78033
:104BE0008089631B0510A547638DF90083479900F1
:104BF00035476388E70029476385E70093F7F70D9A
:104C0000E5EF174600001306262A8145080897009D
:104C10000000E78020E7AA85174600001306062A51
:104C2000080897000000E780E0E5AA851746000025
:104C300013068629080897000000E780A0E4930780
:104C40004003AA851306D1000808A306F100230734
:104C5000010097000000E780E0E2AA851746000007
:104C60001306C670080897000000E780A0E1AA8537
:104C70001746000013064635080897000000E78035
:104C800060E0AA85174600001306466E08089700E4
:104C90000000E78020DFAA8523070100580029468D
:104CA0009307800429482545B3F607037D1613763C
:104CB000F60F93860603A304D700B3D607036375E4
:104CC000F5007D17B6876DF25C003E9608089700E8
:104CD0000000E78020DBAA85174600001306462364
:104CE000080897000000E780E0D9AA850808972007
:104CF0000000E78060A1A5BD41478147E37A87E6D0
:104D00004146974500009385A51C26859720000005
:104D1000E78060768147E31D05E483C7040113073C
:104D20001003639CE700854717070020230AF7A4B8
:104D3000174500001305051B3DB513070003174574
:104D400000001305251DE390E7E297070020238963
:104D500007A2174500001305651A31B5814709BD43
:104D6000170500200345C5A182809707002083C74F
:104D700027B589E71723000067000399828097070A
:104D8000002083C787B899EF411106C6972000001D
:104D9000E780608FB2408547170700202307F7B6EA
:104DA00041018280828063070536638505361D7167
:104DB000CAC8CEC686CEA2CCA6CAD2C4D6C2DAC0D3
:104DC0005EDE62DC66DA6AD86ED6B947AA892E89B9
:104DD00063FFB70839469745000093852501972062
:104DE0000000E780406941E583C7E900130710032D
:104DF0006396E7048547170700202303F7AC1745A0
:104E000000001305A5FF97070020239A07AA97071C
:104E100000202391079C97000000E780608AF640FD
:104E20006644D6444649B649264A964A064BF25B42
:104E3000625CD25C425DB25D256182801307000333
:104E400017450000130585FEE397E7FC9707002050
:104E5000238807A697070020239307A6970700201B
:104E6000239A0796174500001305C5FA6DB79707F3
:104E7000002083C7E7A4639207240144B544294A6C
:104E8000930AE004170B0020130BCB8F9317040138
:104E9000C183170500200355E59363EE272341D115
:104EA00097000000E78060C13DD997070020239359
:104EB0000792B5B7B387490183C60700970700205B
:104EC00083D7E79F8DE79307A005639BF60085478F
:104ED000170700202315F79E97070020238ED78EF3
:104EE000050A93170A01C183E3E627FD0DBF854D2F
:104EF000639BB7039307500A639EF6008947170721
:104F00000020231EF79A930750FA17070020A305E5
:104F1000F78CF9B79307A005E384F6FC9707002008
:104F2000239F079875BF138717004207DA974183BD
:104F30002380D700170600202313E6988D47E3F15E
:104F4000E7FA17040020034454899707002083C719
:104F5000C78822045D8C9307F4FFC207C1839306C0
:104F6000F00DE3EDF6FA93076400C207C183E3197D
:104F7000F7F693052400C205C1811705002013052B
:104F8000C58597F0FFFFE780001B33078B00834741
:104F9000570003474700A207D98F170700202310A7
:104FA00007926311F5108144630CB401970400204B
:104FB00083C4C482A2049707002083C73782DD8C94
:104FC000170500001305C5AA97F0FFFFE78040B062
:104FD0006385740963EF9B026388A4059307EC65FE
:104FE0006383F40697F7FF1F83C7477F05476380F6
:104FF000E70881CB1387A7051377F70F8D4663F971
:10500000E6081307F0072300E100A300F10089453B
:1050100095A8638994059387FA77E395F4FC97F054
:10502000FFFFE780A0F111A8A28517F5FF1F130568
:10503000E57A97F0FFFFE780A0BA014597F0FFFF00
:10504000E78000A971BDA28517F5FF1F130505793B
:1050500097F0FFFFE780C0C1CDB797F0FFFFE78073
:1050600040CAE1BF97F0FFFFE780E0CFF9B79307B1
:1050700010F8130511002300F10097F0FFFFE780FF
:10508000C0EEFD450A8597000000E780E09675B701
:10509000A28517F5FF1F1305657497E0FFFFE780F2
:1050A000C07961BF9307F00789450A852310F10095
:1050B00097000000E780409425B5BD6A396C014A2D
:1050C00017FBFF1F130B4B71938BFA55938CFA66EA
:1050D000130DEC5539B5B387890083C70700638486
:1050E0009700639C47010DC597000000E780E09C96
:1050F00097F7FF1F2390076E21A8E3EBAAFE130783
:1051000015005A9597F6FF1F2396E66C2300F500CD
:105110000504ADBB828017F6FF1F1306667F81472B
:10512000B2861303F00FA9483308F60003480800BD
:1051300013F7F70F6307A80C630668008507E3956C
:1051400017FF2947B387E6002380A70097F7FF1FC3
:105150009387C77C5DA8411113D7650013471700DB
:1051600006C693F63500058B954791CA05469947C3
:105170006387C60009469D476383C600A14713F6AF
:1051800045003336C00093F68503050685C2A14568
:10519000638BB604E145638AB60493058002638895
:1051A000B604930580036393B600914697050020EB
:1051B000238BF59C970500202386C59C970500202E
:1051C000A382D59CBE8517450000130525E49720D2
:1051D0000000E7800038B240854717070020A3048D
:1051E000F79A410182808546D1B78946C1B78D467D
:1051F00075BF174500001305E5E31723000067009E
:10520000433517F7FF1F13076771BA972380B7005D
:10521000E147E302F5F493077002E30CF5FC8280AA
:105220002A8723800500814717F5FF1F1305456E68
:105230001308F00F2946B306F50083C606006396EF
:10524000E60297F6FF1F9386666DB69783C7070041
:1052500005452380F5009947636EF7029D4763FD7E
:10526000E700E147630DF70082806385060185074B
:10527000E393C7FC0145C5B7238005008280B7379B
:10528000004003C7370083C7050093F70704D98F91
:105290002380F50082805D7152DC56DA5ED6716A39
:1052A000970B0020938B4B9F8D6AA6C24EDE62D473
:1052B00086C6A2C4CAC05AD866D26AD06ECEC149C8
:1052C0005E8C97F4FF1F93842466130A0A20938A46
:1052D0007ADC170900200349299FB3872B0183C774
:1052E000070093F7F70FC9EFB787004003C76700C0
:1052F000058BE310077C03C76700118BE30D077E66
:1053000083C75700918B99E36F1020031707002084
:105310000347A79B85476304F7006F104001970779
:105320000020A382E78697F7FF1F238F076A97F76E
:10533000FF1F238D077697070020238B078297078F
:1053400000202388078297F7FF1FA38F076897F72E
:10535000FF1FA38D077497070020A38B0780970773
:105360000020A388078097070020A38F0780970756
:105370000020A38C0794B787004011476F00707717
:105380009307190093F7F70F3D476364F706170774
:105390000020230BF792970700209387E791CA9785
:1053A00083C707001307100293F7F703638EE71E06
:1053B0006366F70405446385871CE38C076209472D
:1053C000638EE71013070002E384E74EB7E700E0BF
:1053D0003707400023A0E71801000100629923006D
:1053E0000900FD1923A0E71093F9F90FE39309EEE3
:1053F000E5BD970700202389078C71BF1307300292
:105400006388E70C63E8E71613074002638CE70A3A
:1054100013070003E39CE7FA970700209387C788E8
:10542000CA9703C70700A1471377F70FE31BF714C9
:1054300083C7640097F6FF1F238EF67297F7FF1F4E
:1054400083C7F74E91C7FD5797F6FF1F2384F67267
:1054500097F5FF1F83C5554D97F7FF1FA38CB770B6
:1054600097F7FF1F83C7474C13FB070893060004F9
:1054700093F70706639FD74C9307A009638DF51632
:1054800063EAB7129307F0056386F54A930750095C
:105490006384F52A014497F7FF1F83C7B76D15474B
:1054A000E392E736B7E700E03707400023A0E718AC
:1054B00001000100B786004023808602130680FCAD
:1054C0006F00500EFD5717F7FF1F2304F76AFDBD4D
:1054D000FD5717F7FF1F230DF768CDBD17450000D7
:1054E0001305C5C697200000E780801E97F7FF1FB1
:1054F0009387877BCA9703C40700014B97FCFF1F64
:10550000938C0C5B1374F40F174D0000130D8DC4B6
:1055100063478B04294597200000E7806008854792
:1055200017F7FF1FA304F75817F7FF1F230187582A
:1055300017F7FF1F230AF76437E700E0B7064000BC
:105540002320D71801000100378600408347A602B8
:1055500093F7370F2305F6022320D71085BDB387B5
:105560006C0183C507006A85050B97200000E78062
:1055700040FE79BF854717F7FF1F2309F752B9B5DA
:1055800017F7FF1F130747724A970347070097F65D
:10559000FF1FA38BF64497F6FF1F2388E64417F7F7
:1055A000FF1F2303F75E1DB5854717F7FF1F230D68
:1055B000F74229BD9307400A6389F5349307200B0E
:1055C0006384F5369307100AE396F5EC838724008D
:1055D0000144E3D207EC97F7FF1F83C7173593F613
:1055E0003700638A061A0546638AC6220946639510
:1055F000C61A1D4755A217F5FF1F03450533C947B6
:1056000097FCFF1F83CC7C3297F5FF1F83C50532C3
:1056100017F4FF1F034494316315F510CD476392CF
:10562000FC1093077008639CF5021307300FB7173F
:105630000E006308E4001307900DB7B7040063146D
:10564000E40817F7FF1F232DF752BE85174500000A
:105650001305C5B097200000E780A0EF25BD930794
:105660008008639DF500B307804013F4F70FB77708
:105670004600938787CDB3D78702E1B79307900899
:10568000639AF500B307804013F4F70F916793878F
:10569000C766D5B79307A008639BF500B3078040A2
:1056A00013F4F70FB7173D0093870790E9B79307F7
:1056B000B008639AF500B307804013F4F70F9167C1
:1056C000938797D04DBF93F5F5078D47639BF50002
:1056D000B307804013F4F70FB7975B00938707D8A1
:1056E00059BF8947639BF500B307804013F4F70F58
:1056F000B7770B009387071BBDBF8547639AF500FB
:10570000B307804013F4F70FDD67938767E3A5B70E
:10571000D28785F9B307804093F7F70FB3D7FA0222
:105720000DB797000000E780409FA285668597002F
:105730000000E780809EB9BB9305610017F5FF1F4D
:105740000345A51E17F4FF1F0344341E97000000F5
:10575000E78040AD93057100228597000000E78047
:1057600060AC3C0017F7FF1F2326F7528347610008
:105770002304F10083477100A304F100894717F760
:10578000FF1F2309F73E8357810017F7FF1F231DD3
:10579000F718094409B3154793F64700B336D0000C
:1057A00093F78703850685C32146638BC706614649
:1057B000638AC706130680026388C7061306800340
:1057C0006393C700914717F6FF1F230DD63A97F64C
:1057D000FF1FA389F63A97F7FF1F2386E73A17F7CB
:1057E000FF1F0347A7149376070497F7FF1F83C78C
:1057F000F7138DEE1377770C93067008630CD702BE
:105800001377F7078D466312D70CB307F040B795AF
:105810005B0093F7F70F938505D849A81947ADBFEB
:10582000854755B7894745B78D4771BF93067008BF
:105830006311D7021307300FB7150E006389E70213
:105840001307900DB7B504006383E70213077008D0
:1058500045BF9306800C6311D702B307F040B775BC
:10586000460013F7F70F938785CDB3D5E70297F777
:10587000FF1F23A7B730D9BB9306900C631CD7003A
:10588000B307F04093F5F70F91679387C766B3D5D9
:10589000B702F1BF9306A00C631DD700B307F04019
:1058A000B7153D0093F7F70F93850590B3D5F50233
:1058B0007DBF9306B00CE315D7F4B307F04093F522
:1058C000F70F9167938797D0D9B78946631BD700A5
:1058D000B307F040B7750B0093F7F70F9385051BDF
:1058E000F1B78546631AD700B307F040DD6593F73B
:1058F000F70F938565E35DBFD28535FBB305F040B7
:1059000093F5F50FB3D5BA029DB783C72400C18BB9
:1059100099C7854717F7FF1F2301F726A5BE97F7FD
:10592000FF1F238C0724BDB6854717F7FF1FA30C65
:10593000F7248DB63C0017F7FF1F232DF7340947D6
:10594000930700032314F10097F6FF1F2384E62238
:105950002DBD63940756A94763E5B742173700008A
:10596000130707688A05BA959C41BA97828717F48E
:10597000FF1F034494FB894C6306940D63E68C0679
:1059800085476303F4089307F00F17F7FF1F0347DA
:10599000671E63F6E70017F7FF1F230DF71C97FC40
:1059A000FF1F83CC2C1D9307000413F4FC0F63F43A
:1059B00097011304000497F7FF1F9387A72D03ADEA
:1059C000070022862685EA85B38C8C40229D97208D
:1059D0000000E780A0AC97F7FF1F238D971997F77A
:1059E000FF1F23A9A72B45BC8D47630CF40A9947D9
:1059F000E31BF4F8973700009387076517F7FF1F3D
:105A0000232AF728A94751B717F7FF1F0347E72BAA
:105A100097F7FF1F9387071849469735000093852E
:105A2000A56B63068700973500009385E5663E8584
:105A300097200000E78080A617F7FF1F232CA724DC
:105A4000C947A1B797F6FF1F83C62628054797F7D2
:105A5000FF1F938727146394E6023E8513067002A6
:105A6000973500009385C56497200000E78000A368
:105A700017F7FF1F2320A7229307700239B73E852F
:105A800013063004973500009385C55C972000000D
:105A9000E780C0A017F7FF1F232EA71E930730042F
:105AA000EDB597F5FF1F83C545E8173500001305D1
:105AB000256C97200000E780C0A9054D97FDFF1FCA
:105AC00083CDAD2097F5FF1F83C525E61735000070
:105AD0001305056A6398AD0B97200000E78060A767
:105AE00097F7FF1F83C767E4B5CBE36EF4E817347D
:105AF00000001304A462638CB70117340000130480
:105B000064626386970117340000130424632285BE
:105B100097200000E78000BD1375F50F930715006F
:105B2000860717F7FF1F2307F7068D4717F7FF1F95
:105B3000A302F70697F7FF1F9387C7050147BE86A5
:105B40001376F70F89076365A60297F7FF1F23A354
:105B5000D71497F7FF1F83C7E70305BD97370000EA
:105B60009387C75417F7FF1F2326F712914731BDBC
:105B70003306E40003460600A380070005072380E0
:105B8000C7007DBF97200000E780A09C97F7FF1F0C
:105B900083C7A7D9E1D7E368F4DE17340000130404
:105BA000E454638CA701173400001304A4546386E3
:105BB00097011734000013046455228597200000D4
:105BC000E78040B21375F50F93071500860717F7A6
:105BD000FF1F2301F7FC8D4717F7FF1FA30CF7FAF0
:105BE00097F7FF1F938707FB0147BE861376F70FD2
:105BF0008907E37CA6F43306E40003460600A3808D
:105C0000070005072380C700D5B797F5FF1F83C599
:105C1000C5D1173500001305655697200000E780B1
:105C2000409397F7FF1F83C7B7F693E7470017F72F
:105C3000FF1FA30FF7F483C7240017F7FF1FA30765
:105C4000F7F489B817350000130585549720000034
:105C5000E78000A897F7FF1F938747F383C70700E4
:105C600017F7FF1F2302F7CC17F4FF1F034484F03C
:105C7000333480000DB0173500001305A55297206E
:105C80000000E780E0A497F7FF1F83C777F093E752
:105C9000070117F7FF1FA30DF7EE83C7240017F7BF
:105CA000FF1F2305F7EE6FF0EFFE17350000130519
:105CB000A55097200000E780A0A103C704007D8BBA
:105CC00051EFB787004003C767021377C70B13670D
:105CD00027002383E70203C7A7021377C70B1367C5
:105CE00027002385E70203C7E7021377C70B136773
:105CF00027002387E70203C727031377C70B136720
:105D000027002389E702854717F7FF1F230EF7CCEB
:105D100017F7FF1F230CF7D817F7FF1F230AF7E425
:105D200017F7FF1F2307F7E497F7FF1FA38E07CA94
:105D300097F7FF1FA38C07D697F7FF1FA38A07E2E9
:105D400097F7FF1FA38707E297F7FF1FA38E07E2CE
:105D500097F7FF1FA38B07F66FF0CFF38947631206
:105D6000F70297F7FF1F83C767BC9146638CD7087C
:105D700063E0F604638EE70C6369F70A0547638006
:105D8000E70EFD5717F7FF1FA306F7DE37074000A2
:105D9000B7E700E023A0E71801000100B786004044
:105DA0001306F0FC2381C60223A0E7106FF00FE278
:105DB000130720086382E7086362F70213071008DD
:105DC000E391E7FC378700408347670293F7C70BEF
:105DD00093E727002303F7026FF0CFEB1307300898
:105DE0006389E70213074008E39DE7F8378700401F
:105DF0008347270393F7C70B93E727002309F7028D
:105E00006FF04FE9378700408347270393F7370741
:105E1000F5B7378700408347E70293F7C70B93E74F
:105E200027002307F7026FF0EFE63787004083472C
:105E3000E70293F73707F5B7378700408347A70294
:105E400093F7C70B93E727002305F7026FF08FE462
:105E5000378700408347A70293F73707F5B737879F
:105E600000408347670293F73707ADB71735000047
:105E70001305853597200000E780808597F7FF1F81
:105E8000238407AAD5B3173500001305E5349720FE
:105E90000000E780E08397F7FF1F239707A897F795
:105EA000FF1F938727CD03C40700894763F387004B
:105EB00009441374F40F6FF00FDE13070002E3922E
:105EC000E7EC631B0B0A638FF500930720026383E3
:105ED000F508173500001305A53397100000E7807B
:105EE000406745B5173500001305C52F9710000012
:105EF000E780007E0144173D0000130DED2FA14CFB
:105F0000B387840083C507006A85050497100000E5
:105F1000E7802064E31694FF17350000130545CE93
:105F200097100000E780C07A17F4FF1F034404A015
:105F300001E897F7FF1F238B079C014B6FF0AFD54C
:105F40008947E310F4E4854717F7FF1F2300F79C08
:105F50006FF04FD417F6FF1F0346369D97F5FF1FCE
:105F600083C5A59C173500001305852997100000EF
:105F7000E780205E6FF00FD26380F5069307100272
:105F8000E399F5F497F5FF1F83C5459A173500008F
:105F90001305052997100000E780A05B97F7FF1F06
:105FA00023AA97CE97F7FF1F938787BD944383D784
:105FB000470017F7FF1F034707BD17F6FF1F2325ED
:105FC000D6961D4497F6FF1F2392F69697F7FF1F6C
:105FD000238FE7946FF02FCC97F5FF1F83C50595AE
:105FE000173500001305452597100000E78060561F
:105FF00097F7FF1F238C079097F7FF1F23960792B1
:106000006FF02FF92547638FE7C89946378700401F
:106010006394D70223008702B7E700E0B706400089
:1060200023A0D71801000100130600FC2301C702BA
:1060300023A0D7106FF08FB99306100A639FD70083
:1060400023008702B7E700E0B706400023A0D71877
:1060500001000100130680FCD1BF9306A009E38173
:10606000D7FE9306400AE38DD7FC93062002639D7A
:10607000D700B7E700E0B706400023A0D71801001B
:10608000010023008702F9B78546E384D7FE930712
:106090000008E300FBFEB7E700E0B706400023A0DE
:1060A000D71801000100130620FC23008702BDBFA2
:1060B00017F7FF1F034717AC6302F71E63E7E702FA
:1060C00095476300F7109947630AF704B7860040C5
:1060D00023800602B7E700E03707400023A0E71857
:1060E000010001001306A0FC75B99307F005630ACF
:1060F000F700930750096306F70093071002E317B0
:10610000F7FCB7E700E03707400023A0E7180100DD
:106110000100B7860040130620FC69B117FBFF1F82
:10612000034B4BA5930700045A8D63F46701130DCD
:10613000000497F7FF1F9387E7B583AC070013743C
:10614000FD0F2286E685268597100000E780003542
:10615000B3078B40669417F7FF1F230DF7A097F73F
:10616000FF1F23A987B2B7870040630C0B0223806F
:10617000A703B7E600E03706400023A0C6180100D9
:10618000010003C72702134707042381E70203C75F
:1061900027021377C70F2381E70223A0C6106FF0F1
:1061A000EFA22380070237E700E0B7064000232074
:1061B000D71801000100130620FC2381C7026FF0ED
:1061C000AFB9378700408347370097F6FF1F83C674
:1061D000F69B93F70708D58FA301F700B706400099
:1061E000B7E700E023A0D718010001001306A0FCC8
:1061F00035BD97F7FF1F938727ABCA9783C7070063
:1062000093F7F70FC1CF97F7FF1F83C707ACD9E705
:1062100017F7FF1F03471796930700026310F7084D
:1062200083AD040017EDFF1F034D4D7097ECFF1F6A
:1062300083CCDC6F17EBFF1F034B6B6FE6876A871E
:10624000DA866E8697E5FF1F83C5456C173500001B
:106250001305050097100000E780A02F97F7FF1F98
:1062600023A0B79397F7FF1F238EA79197F7FF1FE0
:10627000A38A979197F7FF1F2387679197E7FF1FDF
:10628000A3858768B7E700E03707400023A0E71839
:1062900001000100B78600406FF04FA2B7E700E0B1
:1062A0003707400023A0E71801000100B78600402F
:1062B00015BD97F6FF1F83C646A10547639CE604FC
:1062C00029472381E70209472383E7022385E70261
:1062D00097F7FF1FA38A078A97F7FF1FA387079ED9
:1062E000B7870040A381070017F7FF1FA300078AA5
:1062F00005472383E700B640264496440649F259F1
:10630000625AD25A425BB25B225C925C025DF24DF1
:106310006161828029472381E70209472383E702DD
:106320002385E7022387E7022389E70255B717E7AA
:10633000FF1FA30CF75C6FE01FFF854717E7FF1FE8
:106340002304F76A17E7FF1F2302F77617F7FF1FEB
:106350002300F78217F7FF1F230DF7806FE0BFFEC2
:10636000854717E7FF1F2301F76817E7FF1F230F74
:10637000F77217E7FF1F230DF77E17E7FF1F230AAA
:10638000F77E17E7FF1FA301076617E7FF1FA30F9D
:10639000077017E7FF1FA30D077C97E7FF1FA38A6E
:1063A000077C8280411106C697000000E78080FBD1
:1063B000B787004023800700130740FC2386E700CF
:1063C0001307C004A386E70017E7FF1F1307C7558D
:1063D0002398E70017E7FF1F13070759239AE700E1
:1063E00017E7FF1F13078764239CE70017E7FF1FCA
:1063F00013070770239EE70029472381E702094717
:106400002383E7022385E7022387E7022389E70244
:10641000A3810700930600F8A380D700930690029B
:106420002380D700FD562383D7002381E7009306FE
:10643000000537E700E0230BD740B70640002320D4
:10644000D71003C7170013671700A380E700B240F7
:1064500097E7FF1F239C077241018280411106C606
:1064600097000000E78000F0B78700402380070016
:10647000130700FC2386E7003147A386E70017E7F0
:10648000FF1F1307674A2398E70017E7FF1F13074B
:10649000A74D239AE70017E7FF1F13072759239CEF
:1064A000E70029472381E70209472383E702238581
:1064B000E702A3810700930600F8A380D7009306A4
:1064C00090022380D700FD562383D7002381E70065
:1064D0009306000537E700E0230BD740B7064000DE
:1064E0002320D71003C7170013671700A380E70006
:1064F000B24097E7FF1F239B076841018280F16745
:106500009387072017E7FF1F232CF766854717E7B8
:10651000FF1F2319F766A14717E7FF1F2305F7663B
:1065200097E7FF1FA381076697E7FF1F238E076486
:1065300097E7FF1F238C073C97E7FF1FA387073CC4
:10654000814717E5FF1F1305A53CFD5517E6FF1F03
:106550001306C63C2947B306F5002380B600B306F0
:10656000F600238006008507E397E7FE97E7FF1F05
:10657000A383076097E7FF1FA381076097E7FF1FCB
:10658000238C075E97E7FF1F2387075E97E7FF1FB0
:106590002386075E97E7FF1FA380075E97E7FF1F2D
:1065A000238D075C814717E6FF1F1306E66E414700
:1065B000B306F600238006008507E39BE7FE828092
:1065C00017E7FF1F0347677085476316F700170338
:1065D00000006700E3E8170300006700E3DC4111F7
:1065E00022C406C617E7FF1F0347276E85472E867E
:1065F00013F4F50FAA856317F70417E5FF1F1305BA
:10660000E54697100000E78060E997E7FF1F238FBA
:106610000748B787004023848702B7E600E03706C3
:10662000400023A0C6180100010003C7A70213778A
:10663000C70F2385E702B240224423A0C6100145BC
:106640004101828017E5FF1F1305053697100000F2
:10665000E780C0E497E7FF1F23880738B78700402B
:1066600023828702B7E600E03706400023A0C61861
:106670000100010003C767021377C70F2383E702F6
:106680005DBF411106C697000000E78080E7B24079
:106690004101170300006700E3F2411106C697F0BD
:1066A000FFFFE78080BF97E7FF1F83C7F733A1CBCA
:1066B00097E5FF1F83C5653389C917E5FF1F1305DC
:1066C000E53297E0FFFFE780406E97E7FF1FA38D5D
:1066D000073097E7FF1F2389074A37E700E0B7062F
:1066E00040002320D718010001003786004083476F
:1066F000660293F7370F2303F6022320D710B24028
:106700004101828041C9D9C597E7FF1F83C7074868
:10671000D1C3011122CC4AC84EC656C25AC006CEB9
:1067200026CA52C42E89AA890144930A0004371B41
:10673000030063772403B3078940C207C183BE8483
:1067400063F4FA0093040004C204C180130A1BD44A
:1067500097E7FF1F83C747299DE37D1A631C0A0043
:10676000F2406244D2444249B249224A924A024B20
:106770000561828097F0FFFFE78020B2D1BF3385AB
:1067800089002694A685420497000000E78060E512
:10679000418045B7828001113335A000A307A100D5
:1067A000B7E7040083A7471706CE1306F100854517
:1067B000130550308297F24005618280828041113A
:1067C00022C406C697D7FF1F83C717A9054489EFC0
:1067D00097E7FF1F83C787E8014499E717D4FF1F96
:1067E000034484A713441400228597000000E78027
:1067F000C0FA17350000130525A909E41735000074
:10680000130585A92244B240410117130000670017
:1068100043D441119397050122C406C626C2C187FD
:106820002E8463D40702B7E40400FC5417C5FF1F8D
:1068300003454569829719C1BC5482972165218D12
:10684000B240224492444101828093F715008DC7E3
:10685000B7E7040083A7471A17C6FF1F130686650C
:1068600097E5FF1F9385054717C5FF1F03458565FE
:10687000829713451400E9B793F725000145E9D342
:1068800097E7FF1F83C7874685E7B7E7040003A89C
:10689000871A1307401F97C7FF1F83C7A762814648
:1068A00013064006994517E5FF1F0355A5430298B7
:1068B0001345240071B797E7FF1F83D7A74263985A
:1068C000A70217E7FF1F2310B74217E7FF1F231D7B
:1068D000C74017E7FF1F231AD7402E861735000041
:1068E000130505A2BE8517130000670083C6173580
:1068F0000000130565A217130000670063DD03574E
:10690000450097E7FF1F83D7E73D6318F702C1678C
:10691000F91717E7FF1F2327F73C97E7FF1F23A56A
:10692000073C97E7FF1F238D073A97E7FF1F238F49
:10693000073A170300006700C3E817350000130586
:10694000A59D171300006700A3D87D15954763E246
:10695000A71C173700001307A7910A053A951C4199
:10696000011122CC06CEBA972E84828717350000FB
:106970001305059B97100000E78080D5A1A203C7EF
:10698000250099476311F7022E8597000000E780E4
:1069900040F783456400173500001305659997108B
:1069A0000000E78000BB97D7FF1F2387078A1735B2
:1069B00000001305A5997DBF03C7250095476319FE
:1069C000F702C16717E7FF1F0357C731F91703D550
:1069D000A5006309F702B7E7040083A7C7178297EA
:1069E000173500001305859797100000E78040CE0B
:1069F000854717D7FF1F2301F786173500001305BA
:106A000065988DBF97E7FF1F239EA72C83D7E500CE
:106A100097E6FF1F2399F62C83D7050197E6FF1F02
:106A20002394F62C83D7250197E6FF1F239FF62A90
:106A300097E7FF1F2386072A631BE502B7E70400D9
:106A4000BC4F096613060690894517C5FF1F03450D
:106A5000654782970356E4008355A400173500006C
:106A60001305059197100000E780A0AE51B793077A
:106A7000700F2316F100B7E7040083A7870D17C630
:106A8000FF1F034626446C0082974DF9854717E7A0
:106A9000FF1F2307F7245DB7173500001305458F47
:106AA000D1BD83C5250091476392F50217350000DB
:106AB0001305858F97100000E78080C197000000C4
:106AC000E78020D0F240624405618280994763925A
:106AD000F502228597000000E780A0E2834564006C
:106AE000173500001305C58497100000E78060A6E5
:106AF000D1BF9547639AF50083471400E1F317353A
:106B000000001305A58CBDB5173500001305858C55
:106B1000E1BF82803757315F97C7FF1F9387C73B1D
:106B2000130777D598C39356C5001727000013079E
:106B3000E779BA9683C5060093568500BD8ABA9652
:106B400003C6060093564500BD8A3D89BA962A972A
:106B500083C6060003470700238407002383D7006A
:106B6000A383E7002382B700A382C70097C7FF1F54
:106B7000938787372383B700A383C7002384D70075
:106B8000A384E700828061712324811A37E4040022
:106B9000832704082326111A2322911A2320211B5C
:106BA000232E3119170500001305E5C6829717C972
:106BB000FF1F13092931994785442300A900231C8D
:106BC000F100972500009385656F93074006172510
:106BD00000001305E5F3231CF1082308910097E951
:106BE000FF1F938909B897100000E780809683D52E
:106BF0000900172500001305656B97100000E7805A
:106C00004095294597100000E780809903D5090039
:106C100097000000E78040F083274417100885455F
:106C20001305503082978327441717C6FF1F13069A
:106C3000A62BCD451305703082978327441717C6BE
:106C4000FF1F13066628B54513056030829783271A
:106C5000441730088945130510318297832744175C
:106C60003009894513052031829783274415930500
:106C7000000A0D458297832744159305000A1145A4
:106C80008297A30591002306910002CD23080100FD
:106C9000230C0100832784163009914513057040A9
:106CA0008297832784161306B1008545130500409B
:106CB00082978327841670008545130510408297BC
:106CC0008327841630088545130520408297832743
:106CD00084161008854513055040829783270415B4
:106CE0007D558297832744137D5582977D5597C0A4
:106CF000FFFFE780204B8327440C829797C0FFFF5C
:106D0000E78080268327841417C6FF1F1306C61C3E
:106D1000D5450145829789471306700F814528099B
:106D20002306F10097B0FFFFE780E0018D471306CF
:106D3000000881452808230CF10897B0FFFFE78081
:106D400080009147230CF10097270000938787CE9E
:106D5000984383C747003AC8230AF10097D0FFFF42
:106D6000E780202C70008545054597C0FFFFE78030
:106D7000804A30099305700F094597C0FFFFE780EF
:106D800080493008930500080D4597C0FFFFE78054
:106D9000804810089545114597C0FFFFE780A04740
:106DA000C16717E7FF1F1307E7F3F9171CC3232277
:106DB000070017C5FF1F1305A51097C0FFFFE78049
:106DC00060448327C41D17E5FF1F130525F0829734
:106DD0003C4803450900854582978320C11A032456
:106DE000811A8324411A0329011A8329C1195D617B
:106DF0008280C16717E8FF1F0358C8EEF9176301C7
:106E0000F8083DCDB5CD011126CAB7E4040083A72B
:106E1000841222CC2E862315B10006CE2A84014787
:106E20008146ED45428582972AC611ED172500005F
:106E30001305054B97100000E7808089F2406244FB
:106E4000D24405618280FC440356A100A28582974A
:106E50002C0017E5FF1F0355E5E897C0FFFFE7800B
:106E6000204769DD172500001305C548971000006D
:106E7000E780008683A7C412ED45280082977DBF76
:106E8000828097E7FF1F83C767E6A9EFC16717E70F
:106E9000FF1F035727E5F9176306F70441118547DC
:106EA00022C417E7FF1F2303F7E437E404007C4CF8
:106EB00006C6894517C5FF1F0345C50082970323F2
:106EC000841A2244B24097C7FF1F83C7A7FF17E564
:106ED000FF1F035525E11307401F814631469945A1
:106EE0004101028382806D712324811023261110B9
:106EF00023229110328401CD8947630AF502832051
:106F0000C110032481108324411051618280172510
:106F100000001305E54CAE8497000000E780407B3D
:106F2000A285268597D0FFFFE780C08AC9BFB7E753
:106F30000400FC4728008297172500001305054B25
:106F400097000000E780C0788347810039C41307A9
:106F5000000B6380E7021387A7051377F70F8D46B1
:106F600063EDE602A285280097D0FFFFE780E08C62
:106F700079B78547E3F587F8834591001725000029
:106F800013058547B335B00097C7FF1F2387B71A8E
:106F900097000000E780E05B9DB703479100A207E0
:106FA000B966D98F1387E6556384E70C636DF704E0
:106FB0002D671307B755638FE708636AF7002967E2
:106FC0001307A755638FE708A2852800A1BF316783
:106FD0001307C7556388E70635671307D755E39549
:106FE000E7FE8947E3FD87F097000000E780A0E90E
:106FF0009305E4FFC205C1811305A10097C0FFFFFF
:10700000E780A0CFEDBD3D671306F7556389C7063E
:10701000636DF6009386E665E398D7FAA2852800AB
:1070200097D0FFFFE780C0C4D9BD9306F766638D94
:10703000D7041307F777E399E7F897D0FFFFE780C6
:10704000E0EF75BD0146A285280097D0FFFFE780DD
:1070500060AA75B5A285280097D0FFFFE78080B5AC
:1070600079BDA285280097D0FFFFE78060B641BDBB
:10707000A285280097D0FFFFE78080B649B597D05A
:10708000FFFFE78000C8A5BD97D0FFFFE780A0CD38
:10709000BDB517F3FFFF6700C372014863C6050E55
:1070A00063DB06003306C040B337C000B306D040F0
:1070B0001348F8FF9D8EB6873283AA8EAE886391FF
:1070C000061863FCC50C41676361E61EB707000143
:1070D0006365F63693568601E147172700001307CC
:1070E0002733369703470700BA97130700021D8F0F
:1070F00019CBB395E500B357F5003313E600B3E8B9
:10710000B700B31EE50013560301B3D7C8029316A8
:107110000301C18213D70E01B3F5C8023385F6020D
:10712000C205B3E8E50063FAA8009A981387F7FF51
:1071300063E4680063E9A832BA87B388A840B3D58E
:10714000C802C20E93DE0E01B3F8C802B386B602BF
:10715000C208B3E8D80163FBD8009A981387F5FFFB
:1071600063E56800F91563E3D800BA851395070154
:107170004D8D8145630908003305A040B337A00059
:10718000B305B0409D8D82803305A040B337A00089
:10719000B305B0409D8D7D5821B701E605433353BB
:1071A000D3024167636AE30EB7070001636BF328FC
:1071B00093568301E1471727000013076725369789
:1071C00003470700BA97130700021D8F65EB93185A
:1071D0000301B3866540135F030193D80801854519
:1071E00013D70E01B3D7E603B3F6E60333861703CE
:1071F000C206558F637AC7001A979386F7FF6364B8
:1072000067006365C726B687118FB356E703C20EC2
:1072100093DE0E013377E703B38816034207336723
:10722000D701637B17011A971386F6FF6365670022
:10723000F91663631701B28613950701558D1DBFBB
:1072400063E1D504C16763E1F604B707000163E2B7
:10725000F61E93D886016147972700009387471B46
:10726000C69703C30700930700023A93B3876740AA
:10727000E9EB63ECB61C3335C500134515008145B9
:10728000D5BD81450145FDB59307F00F63F2D71CCD
:1072900093D886002147C9B71307F00F9A86E37C7D
:1072A00067F093568300A14739B71307F00FB286F2
:1072B000E375C7E293568600A14705B53313E30093
:1072C00033D6F500135F0301335EE603B396E500A2
:1072D000B357F500DD8E9318030193D80801B31E50
:1072E000E50093D50601B377E6033387C803C207E9
:1072F000CD8F63FBE7009A971306FEFF63E36716E3
:1073000063F1E716791E9A97998F33D6E70313979F
:1073100006014183B3F7E7033385C802939607015B
:10732000D98E63FBA6009A969307F6FF63E7661271
:1073300063F5A61279169A9693150E01898ED18D52
:1073400045B533576600B396F600D98EB3D86500BD
:1073500013DF0601B3DEE803139E06013353650015
:10736000135E0E01B395F500B365B30013D70501A5
:107370003316F600B3F8E8033303DE03C20833E73D
:10738000E800637B670036979388FEFF6369D70C3C
:107390006377670CF91E3697330767403353E7036B
:1073A000C205C1813377E703B3086E024207D98D66
:1073B00063FB1501B6951307F3FF63EED50863FC75
:1073C00015097913B695C20E416FB3EE6E0013071F
:1073D000FFFFB3F6EE0013D30E01718F4182338E9F
:1073E000E602B3851541B386C60293580E013307F2
:1073F000E302BA96C6963306C30263F3E6007A96B2
:1074000013D306011A9663E2C5026385C50076852B
:1074100081458DB341677D17F98EC206337EEE003C
:10742000B317F500F296E3F4D7FE1385FEFF81450E
:1074300091B393D80601414705B593560601C1475C
:1074400069B993560301C147BDB3814505451DB3D5
:10745000B688014711B53A83BDB73E86F1BDC68EE9
:1074600025BF328E55B5F9179A98C1B9F9171A97F1
:1074700061BB01476314E60001458280B307E50064
:107480000507B386E50083C7070083C6F6FFE383DD
:10749000D7FE3385D7408280B3C7A5008D8B3307D5
:1074A000C50081E78D4763EEC700AA876370E50AD0
:1074B00083C6050085078505A38FD7FEE3EAE7FEAF
:1074C000828093763500AA8791CA83C60500850716
:1074D0008505A38FD7FE93F63700FDB79376C7FFD8
:1074E000138606FE63F0C70683A3050083A245004A
:1074F00083AF850003AFC50083AE050103AE450130
:1075000003A3850183A8C5019385450223A07700C5
:1075100003A8C5FF23A2570023A4F70123A6E70170
:1075200023A8D70123AAC70123AC670023AE170104
:107530009387470223AE07FF75B7904191079105E6
:1075400023AEC7FEE3EBD7FEE3E4E7F682803971B2
:107550003EDA2ED232D436D63AD842DC46DE97C74F
:10756000FF1F9387A79F22CC804326CA06CEAA84FA
:1075700001C81C4C91E7228597000000E780405F1E
:107580000C4454102686228536C697100000E780EA
:1075900080ACF2406244D24421618280011197C7DD
:1075A000FF1F9387A79B22CC804306CEAA8511C8D4
:1075B0001C4C81EB2AC6228597000000E780405BC7
:1075C000B245104422856244F24005611713000061
:1075D00067006310011126CA4AC806CE22CC4EC6E7
:1075E00052C4AA842E8919C51C4D89E79700000052
:1075F000E78000589C4C804491E726859700000066
:10760000E780005797270000938787F2631FF402F3
:10761000C0408357C400A18BA9CB1C48B9C7FD59F2
:10762000294A1C4483450900FD17A5E11CC463D702
:1076300007082286A945268597000000E780A00B51
:10764000FD57630BF50229450DA897270000938786
:1076500027F06314F40080446DBF972700009387E0
:1076600027EBE318F4FAC0446DB7A285268597008E
:107670000000E780C01545D57D55F2406244D244F4
:107680004249B249224A056182801CC4050963D778
:107690000700184C63CBE700638945011C40138742
:1076A000170018C02380B700ADBF2286268597003B
:1076B0000000E7804004E31635F77DBF1C401387C8
:1076C000170018C029472380E700B5BF97C7FF1FE1
:1076D0009387C788AA858843170300006700C3EF14
:1076E000AA87850703C7F7FF6DFF3385A7407D1580
:1076F0008280011122CC26CA4AC806CE4EC6AA8470
:107700002E89328419C51C4D89E797000000E78057
:107710002046972700009387A7E1631FF406C04027
:107720001C4C1CC48357C400A18BD9C71C48C9C7B3
:107730001C4808409379F90F1379F90F1D8D5C48A7
:107740006349F500A285268597000000E780602E3A
:107750003DE91C440505FD171CC41C401387170098
:1077600018C0238037015C486389A7008357C40091
:10777000858B99CBA9476319F900A28526859700C7
:107780000000E780002B21E1F24062444A85D244A8
:107790004249B2490561828097270000938747DB01
:1077A0006314F4008044ADBF97270000938747D649
:1077B000E318F4F6C044ADB7A28526859700000013
:1077C000E780E00035D57D59C1B7411197B7FF1F5C
:1077D0009387C77826C2844322C44AC006C62A8932
:1077E0002E8481C89C4C91E7268597000000E78095
:1077F0002038972700009387A7D3631CF402C0406A
:107800000317C40093170701C18393F68700C9E2E9
:1078100093F607019DEEA5472320F900136707049F
:107820002316E4007D55B2402244924402494101AE
:107830008280972700009387A7D16314F4008044C7
:10784000C1B7972700009387A7CCE31BF4FAC04485
:1078500045BF918B85CB4C5881CD930744046387FA
:10786000F5004A8597000000E780E05B232A0402C8
:107870008357C4002322040093F7B7FD2316F400B6
:107880001C481CC08357C40093E787002316F400EC
:107890001C4899EF8357C4001307002093F707286B
:1078A0006388E700A2854A8597000000E780C04C06
:1078B0008357C40013F7170005C75C48232404004E
:1078C000B307F0401CCC1C480145B1FF8317C4002E
:1078D00013F7070829DB93E707042316F40099B789
:1078E000898B014791E3584818C4F1BF83D7C5007D
:1078F000011122CC26CA06CE4AC84EC613F787000D
:10790000AA842E846DE3D841634DE000B841634AF8
:10791000E0000145F2406244D2444249B249056167
:10792000828058547DD703A904009396370123A081
:10793000040063D0060870488357C400918B99C730
:107940005C401D8E5C5899C33C401D8E5C540C50AD
:10795000814626858297FD570357C400631DF500B5
:107960009440F54763EBD706B70740208507B3D7A8
:10797000D700858BBDC31C48232204001CC093176D
:10798000370163D80700FD576314F5009C4091E36D
:1079900068C84C5823A02401ADDD930744046387D5
:1079A000F500268597000000E780E047232A0402BF
:1079B0008DB70C500146854626850297FD572A86CD
:1079C000E31CF5F69C40ADDB75476385E70059473E
:1079D0006394E70423A024012DBF13670704231633
:1079E000E4007D5505BF83A90501E38409F203A9DD
:1079F00005008D8B23A0350133093941014791E3FF
:107A0000D84918C4E35720F11C540C50CA864E863E
:107A1000268582976349A0008357C40093E7070433
:107A20002316F4007DBFAA993309A940E1BF9C4900
:107A3000ADC7011122CC06CE2A8409C91C4D99E795
:107A40002EC697000000E780A012B24597270000DD
:107A5000938707AE639EF5004C408397C5008DCB9E
:107A600022856244F240056117030000670043E885
:107A7000972700009387C7AD6394F5000C44F1BFCE
:107A8000972700009387C7A8E399F5FC4C44F1B70A
:107A9000F2406244014505618280014582804111C6
:107AA00022C406C62A842316B5002317C500232046
:107AB0000500232205002324050023220506232890
:107AC0000500232A0500232C0500214681451305C6
:107AD000C50597A0FFFFE780002797170000938751
:107AE000C7CB5CD097170000938787CE1CD497171D
:107AF0000000938787D35CD4971700009387A7D69D
:107B000000D01CD8B2402244410182809705000079
:107B1000938525F21703000067006319411126C2FF
:107B2000130680069384F5FFB384C4024AC02E89ED
:107B300022C406C69385440797000000E780203AD8
:107B40002A8411CD2320050023222501310508C4F4
:107B500013868406814597A0FFFFE780C01E22851B
:107B6000B240224492440249410182801C4DC9E73F
:107B7000411106C622C497070000938767F91CD5F8
:107B800097270000938787A29C432324050423267C
:107B90000504232805046314F50085471CCD2A84B9
:107BA00097000000E780A00548C0228597000000EC
:107BB000E780E00408C4228597000000E7802004E5
:107BC00048C448400146914597000000E78060EDB9
:107BD00008440546A54597000000E78080EC48442E
:107BE0000946C94597000000E780A0EB85471CCCFB
:107BF000B2402244410182808280411197270000D7
:107C00009387C79A26C284434AC006C69C4C22C4A6
:107C10002A8991E7268597000000E78060F5938424
:107C200084048044DC40FD1763D607009C40ADC34C
:107C30008440C5BF0317C40029EBC1778507232201
:107C400004062320040023220400232404005CC42F
:107C500023280400232A0400232C04002146814504
:107C60001305C40597A0FFFFE780E00D232A040257
:107C7000232C040223240404232604042285B24076
:107C8000224492440249410182801304840661BF68
:107C900091454A8597000000E78080E888C049F94F
:107CA000B1472320F9000144D1BF797122D44AD0D1
:107CB00052CC56CA5AC85EC606D626D24ECE2A8A9C
:107CC000AE8A130485040149054BFD5B09ECB250F3
:107CD00022544A8592540259F249624AD24A424B8E
:107CE000B24B45618280044483294400FD1963D46A
:107CF00009000040E1BF83D7C400637BFB0083978A
:107D0000E40063877701A6855285829A3369A900CA
:107D100093848406E1BF1971A6DAAE848395E500E9
:107D2000A2DC86DE328463DC050083D7C40023A096
:107D3000060093F7070895E7930700402DA0300849
:107D400036C697100000E780C0B9B246E34F05FC85
:107D50007247BD67F98F7977BA9793B717009CC2BE
:107D6000E1BF930700041CC0F6506654D654014589
:107D70000961828083D7C500011122CC06CE26CAB4
:107D80004AC8898B2E8489CF930774041CC01CC8F1
:107D900085475CC8F2406244D24442490561828012
:107DA00074003000AA8497000000E78000F7A24525
:107DB0002A89268597000000E780601201ED83176D
:107DC000C40013F7072079F7F19B93E727002316E8
:107DD000F4005DBF97070000938787D39CD4835737
:107DE000C40008C008C893E707082316F400A24798
:107DF0005CC8B24785C38315E40026859710000050
:107E0000E780A0B101C98357C400F19B93E7170035
:107E10002316F4008357C4003369F90023162401A4
:107E200095BFDDC983A7C5FF411122C406C626C27E
:107E30001384C5FF63D307003E94AA849710000003
:107E4000E78040B697B7FF1F9387C7119C4385E330
:107E50002322040097B7FF1F23A687102244B240B5
:107E6000268592444101171300006700C3B3637E67
:107E7000F40014403307D4006396E7009843DC43D2
:107E8000369718C05CC0F9B7BA87D84319C3E37DE9
:107E9000E4FE94433386D700631F86001040B296F9
:107EA00094C33386D700E31BC7FA10435843B296F6
:107EB00094C3D8C365B76375C400B1479CC079BF8C
:107EC0001040B306C4006316D70014435843B2965B
:107ED00014C058C0C0C359B78280011126CA938408
:107EE0003500F19806CE22CC4AC84EC6A104B1474F
:107EF00063F3F406B14463E2B4062A8997100000E4
:107F0000E78040AA97B7FF1F9387C70598433A8435
:107F100039EC97B7FF1F938727059C4399EB814561
:107F20004A8597100000E780E08397B7FF1F23ADD5
:107F3000A702A6854A8597100000E780A082FD5918
:107F4000631F3507B1472320F9004A8597100000C9
:107F5000E78060A529A0E3D004FAB1471CC1014520
:107F6000F2406244D2444249B249056182801C40D9
:107F7000858F63C30704AD4663F6F6001CC03E94CC
:107F800004C001A85C406317870217B7FF1F232BAB
:107F9000F7FC4A8597100000E780E0A01305B400C5
:107FA0009307440061993307F5405DDB3A94898F6C
:107FB0001CC07DB75CC3F1BF2287404091BF130452
:107FC00035007198E30E85FAB305A4404A85970001
:107FD0000000E7802079E31535FBADB71C46FD179F
:107FE0001CC663DC0700184E63C5E700A94763960B
:107FF000F50017F3FFFF670003701C422E851387FF
:10800000170018C22380B7008280011122CC26CA33
:108010004AC84EC652C406CE2A89AE893284B304F9
:10802000D6007D5A63149400014521A883450400BD
:108030004E864A8597000000E78080FA0504E31326
:1080400045FFF2406244D2444249B249224A0561A6
:108050008280357122CD26CB4AC94EC706CF52C584
:1080600056C35AC1DEDEE2DCE6DAAA89AE84328982
:10807000368419C51C4D89E797000000E78040AFA2
:10808000971700009387C74A6391F40E83A44900B1
:1080900083D7C400A18BE5CF9C48F5CB93070002A2
:1080A000A304F1029307000302D22305F10222C6C2
:1080B000930B5002971A0000938A8A4B054C294B68
:1080C0004A848347040099C36398770FB30C244113
:1080D00063800C02E6864A86A6854E8597000000DE
:1080E000E780E0F2FD576301F5209256E69636D21E
:1080F00083470400638A071EFD571309140002C852
:1081000002CE3ECA02CCA309010482D483450900F1
:108110001546568597100000E78020871304190044
:10812000C24749ED13F7070109C713070002A30966
:10813000E10413F7870009C71307B002A309E1049C
:10814000834609001307A0026382E608F2474A84C7
:10815000814625460347040093051400130707FDD5
:10816000637BE60AA5CE3ECE95A8971700009387BD
:10817000273E6395F40083A4890019BF9717000078
:1081800093870739E396F4F083A4C90011B7A68555
:108190004E8597F0FFFFE780806309D17D55FA4057
:1081A0006A44DA444A49BA492A4A9A4A0A4BF65B6F
:1081B000665CD65C0D618280050421B733055541AC
:1081C0003315AC00C98F3EC8228989B73247930660
:1081D0004700184336C6634907023ACE03470400F6
:1081E0009307E002631FF704034714009307A002FC
:1081F000631BF702B2470904138747009C433AC642
:1082000063C107023ECA35A83307E04093E7270061
:108210003ACE3EC8E1B7B387670385462E84BA9746
:1082200015BFFD57C5B7050402CA814681472546DB
:108230000347040093051400130707FD637CE6065B
:10824000F1F2834504000D46171500001305C532F1
:1082500097000000E780607311CD971700009387A7
:10826000A7311D8D93070004B397A700424505046D
:108270005D8D2AC8834504001946171500001305B3
:10828000E52F130914002304B10297000000E780D2
:10829000C06F3DC19787FFFF9387C7D695E74247D9
:1082A000B2471377071009CF91073EC69257D2976E
:1082B0003ED239B5B387670385462E84BA978DBF02
:1082C0009D07E19BA107D5B778009706000093862C
:1082D00006D426860C084E8597000000E7000000B3
:1082E000FD572A8AE314F5FC83D7C40093F70704EB
:1082F000E39607EA125565B5780097060000938665
:1083000006D126860C084E8597000000E780601194
:10831000C1BF797156CA9C49BA8A984522D426D2DF
:108320004ECE52CC06D64AD05AC85EC6AA892E84F2
:10833000B284368A63D3E700BA879CC0034734040B
:1083400019C385079CC01C4093F7070281C79C4056
:1083500089079CC00329040013796900631A090086
:10836000130B9401FD5B5C449840998F634CF904B6
:108370001C408346340493F70702B336D000A5EBC4
:1083800013063404D2854E85829AFD576303F504A3
:108390001C4011469840998B544481446397C70010
:1083A000B384E64063D3040081441C4418486354FA
:1083B000F700998FBE94014969047D5B6398240599
:1083C000014509A885465A86D2854E85829A631E44
:1083D00075017D55B250225492540259F249624AB5
:1083E000D24A424BB24B456182800509ADBF33078B
:1083F000D40013060003A301C70403475404938762
:108400001600A2978906A381E7049DBF85462286B0
:10841000D2854E85829AE30E65FB050945B77971D1
:1084200022D426D24AD04ECE06D652CC56CA5AC8EC
:10843000B68983C68501930790063289AA842E8463
:1084400013863504638DF60263E2D7069307800531
:10845000638DF61863EDD700638606229307300418
:108460006381F60C930A24042301D404E1A093074A
:1084700030066388F60A93074006E395F6FE1C4033
:10848000084393F6070893054500DDC61C410CC35D
:1084900063D807001307D002B307F040A301E40438
:1084A000971600009386060E2947C1A09307000780
:1084B0006389F61663E5D7029307E0066380F61A30
:1084C0009307F006E390F6FA0C401C4313F80508F6
:1084D00013854700630A080608C39C43A5A89307B1
:1084E0005007E383F6FE930780076380F614930733
:1084F0003007E399F6F61C43D04181459386470047
:1085000014C383AA0700568597000000E780E04760
:1085100001C53305554148C05C401CC8A301040493
:1085200071A81C43930A2404938647009C4314C3F8
:108530002301F4048547D5B793F607041C410CC307
:10854000A1DAC207C187A9B793F5050408C3D1D53D
:1085500083D707001307F006638AE60E971600001C
:10856000938646022947A30104044C400CC463C50A
:10857000050008406D9908C099E3B28A91CDB28A8E
:10858000B3F5E702FD1AB69583C505002380BA004E
:10859000B3D5E70263F2E70CA147631EF7001C4066
:1085A000858B91CB58401C4863C7E70093070003B5
:1085B000A38FFAFEFD1A3306564110C84E87CA86AD
:1085C0007000A285268597000000E780C0D47D5A00
:1085D000631E450B7D55B250225492540259F24904
:1085E000624AD24A424B45618280A382D5049716E3
:1085F0000000938626F90C40084313F805081C4137
:108600001105630D080208C313F7150001C793E5B0
:1086100005020CC04147A1FB0C4093F5F5FD0CC0D1
:1086200099B79C4193E707029CC193078007A30277
:10863000F40497160000938626F675BF13F8050418
:1086400008C3E30308FCC207C1837DBF971600007F
:10865000938646F3214701BFAE871DB794411C4363
:10866000CC4913F80608138547006306080008C3C1
:108670009C438CC301A808C393F606049C43F5DA17
:108680002390B70023280400B28A0DBF14485686F1
:10869000CA8526858299E30F45F31C40898B8DE7B7
:1086A000B2474844E359F5F23E8535B785465686CC
:1086B000CA8526858299E30F65F1050A5C44324735
:1086C000998FE345FAFEE9BF014A930A94017D5B65
:1086D000F5B7011122CC06CE2A8419C91C4D89EBAD
:1086E00032C62EC497F0FFFFE78080483246A2458D
:1086F000971700009387C7E36318F60250401C46A3
:10870000FD171CC663D20704184E63C7E70093F732
:10871000F50F2947639AE70222856244F24005611A
:1087200017F3FFFF670023FD97170000938747E2C9
:108730006314F6001044E1B797170000938747DDF4
:10874000E31FF6FA504465BF1C4213F5F50F13877B
:10875000170018C22380B700F2406244056182808E
:10876000411122C42A842E8597C7FF1F23A20758D0
:1087700006C697A0FFFFE780E049FD576319F500A3
:1087800097C7FF1F9387C7569C4391C31CC0B24035
:10879000224441018280411122C42E848395E50048
:1087A00006C697000000E7802020634905007C484A
:1087B000AA977CC8B2402244410182808357C400FA
:1087C0007D777D17F98F2316F400EDB783D7C500A9
:1087D000011122CC26CA4AC84EC606CE93F707100E
:1087E000AA842E843289B68989CB8395E50089468F
:1087F000014697000000E780A0158357C4007D77ED
:108800007D17F98F2316F4008315E4006244F240CB
:10881000CE864A86B24942492685D244056117036D
:10882000000067000305411122C42E848395E500F2
:1088300006C697000000E780A011FD570357C4004B
:10884000631BF500FD77FD17F98F2316F400B24086
:108850002244410182808567D98F2316F40068C8BD
:10886000FDB78395E500170300006700230441115D
:1088700022C42A842E85B285368697C7FF1F23A976
:10888000074606C697A0FFFFE7804036FD576319ED
:10889000F50097C7FF1F9387A7459C4391C31CC052
:1088A000B240224441018280411122C42A842E8593
:1088B00097C7FF1F23AE074206C697000000E78058
:1088C0004012FD576319F50097C7FF1F9387474272
:1088D0009C4391C31CC0B24022444101828041119B
:1088E00022C42A842E85B28597C7FF1F23A2074082
:1088F00006C697000000E780C00FFD576319F5001A
:1089000097C7FF1F9387C73E9C4391C31CC0B240CB
:10891000224441018280411122C42A842E8597C7B6
:10892000FF1F23A7073C06C697000000E780600DE5
:10893000FD576319F50097C7FF1F9387673B9C435B
:1089400091C31CC0B240224441018280411122C423
:108950002A842E85B285368697C7FF1F23AA07383B
:1089600006C697000000E780C00AFD576319F500AE
:1089700097C7FF1F9387C7379C4391C31CC0B24062
:1089800022444101828093F5F50F2A966314C500B5
:108990000145828083470500E38DB7FE0505FDB7DD
:1089A00082808280411122C42A842E85B285368637
:1089B00097C7FF1F23AE073206C697000000E78067
:1089C0004006FD576319F50097C7FF1F938747328D
:1089D0009C4391C31CC0B240224441018280930752
:1089E000800517C7FF1F2325F7307D558280930729
:1089F000800517C7FF1F232DF72E7D558280930713
:108A0000800517C7FF1F2325F72E01458280930796
:108A1000800517C7FF1F232DF72C7D5582809307F4
:108A2000800517C7FF1F2325F72C7D558280000086
:108A30000102030405000000E09EFFFF089FFFFF06
:108A4000309FFFFF489FFFFF629FFFFF729FFFFF66
:108A50009A9FFFFFC29FFFFFDA9FFFFFF49FFFFF78
:108A6000FE006578706572696D656E74616C0000FA
:108A700076312E3000000000262A000076312E309C
:108A800000000000272A0000626C656465732E6395
:108A90006F6D0000292A00004D6F64656C204E75D3
:108AA0006D6265720000000053657269616C204E52
:108AB000756D6265720000000A1800000200000077
:108AC000B88A000076312E3000000000282A00000D
:108AD00062A7FFFF88A7FFFFA2A7FFFFC0A7FFFFB6
:108AE000DEA7FFFF73696D706C6550726F66696C0D
:108AF000655F577269746541747472434200000087
:108B0000E0FF000002000000008B00004150505FB9
:108B10004442472025733E200000000073696D70B9
:108B20006C6550726F66696C655F577269746541F8
:108B30007474724342206C656E3A20256400000014
:108B4000E1FF0000E2FF0000E3FF0000E4FF00009F
:108B5000E5FF000043483539785F424C455F4C499A
:108B6000425F56312E330000686561642066696C8F
:108B700065206572726F722E2E2E00004C494220C5
:108B8000696E6974206572726F7220636F64653AF2
:108B9000202578202E2E2E0A000000002A2000001A
:108BA0004170705F496E69743A20424C452D6F6E7A
:108BB0006C7920286E6F204D657368207374616333
:108BC0006B290D006C6F63616C20696D61676520B6
:108BD000696E666F206C656E206572720000000021
:108BE0004F54413A2073757370656E642043353578
:108BF0004320424C45206E6F746966790D00000079
:108C00006C6F63616C20757064617465206C656E57
:108C100020657272000000006C6F63616C207665E5
:108C200072696679206C656E2065727200000000C2
:108C30006C6F63616C20656E64206C656E2065727C
:108C4000720000004941505F454E442028424C4587
:108C5000206C6F63616C290D000000004170705F33
:108C6000426C655F4C6F63616C5F4F74615F48611C
:108C70006E646C6500000000436F6E666967204794
:108C80006174657761790D007461726765745F6402
:108C9000657620253034580D0A00000044495341C0
:108CA000424C454400000000454E41424C454400C2
:108CB0004465627567206D6F64652025730D0A0039
:108CC0005175657279204D65736820416464722026
:108CD0002D2050726F766973696F6E65643A2564F2
:108CE0002C20416464723A3078253034580D0A00E3
:108CF0005175657279204D657368204B6579202D1B
:108D00002050726F766973696F6E65643A25640DE1
:108D10000A0000004465627567206D6F6465206C11
:108D20006F616465642066726F6D20666C61736844
:108D30003A2025640A0000004465627567206D6F63
:108D40006465207573696E672064656661756C740F
:108D50003A2025640A0000004D65736820475720BB
:108D6000647374206C6F616465643A2030782530D8
:108D700034580D0A000000004D65736820475720E5
:108D80006473742064656661756C743A203078256C
:108D90003034580D0A0000004465627567206D6F1D
:108DA000646520736176656420746F20666C6173FE
:108DB000683A2025640A00004D65736820475720F3
:108DC0006473742073617665643A2030782530349A
:108DD000580D0A00434D445F484541443A307825D8
:108DE0003034580D0A000000534541534B5920437D
:108DF00044432047573D0000534541534B59204FB2
:108E00004B204344432047573D310D0A00000000EA
:108E1000534541534B59204F4B2043444320475720
:108E20003D300D0A00000000534541534B59204589
:108E3000525220434443204757204D53473D6261DF
:108E4000645F76616C75650D0A00000053454153FF
:108E50004B5920434443204D4553483F00000000F8
:108E6000534541534B59204F4B20434443204D45DC
:108E700053480000534541534B592043444320433A
:108E800046473F00534541534B59204F4B204344E5
:108E90004320434647000000534541534B59204966
:108EA00044000000534541534B59204944204D4F45
:108EB00044454C3D22000000574D2D473330302DA6
:108EC00047570000222046573D00000053454153BC
:108ED0004B592043444320574156453D0000000074
:108EE000534541534B59204F4B2043444320574156
:108EF00056453D310D0A0000534541534B59204F13
:108F00004B2043444320574156453D300D0A000055
:108F1000534541534B592045525220434443205717
:108F2000415645204D53473D6261645F76616C75E3
:108F3000650D0A0020503D310000000020503D30FA
:108F400000000000204144563D31000020414456BD
:108F50003D30000020574156453D310020574156D5
:108F6000453D300020413D0020523D4700000000BB
:108F70002046573D0000000020424155443D00007E
:108F80002052454C41593D300000000020424C45E4
:108F90003D310000204453543D0000002054583D12
:108FA00000000000204552523D00000020453D00D9
:108FB0002050453D00000000204D41433D00000091
:108FC000204B3D003000000030313233343536372D
:108FD000383941424344454600000000AACEFFFF15
:108FE000CECCFFFFA6CDFFFFA6CDFFFFA6CDFFFF96
:108FF0002ECCFFFF92C9FFFFA6CDFFFF68CCFFFF7D
:109000009ACCFFFF90CEFFFF434833343120736585
:109010007420706172613A256420256420256420E3
:10902000627265616B3A253032780D0A00000000EB
:109030006D6F64656D207365743A253032780D0A62
:10904000000000000A060002FF00FF4001000000CF
:1090500009024300020100803009040000010202FD
:109060000100052400100104240202052406000169
:10907000052401010007058403080001090401001B
:10908000020A0000000705010240000007058102F6
:10909000400000001201100102000040861A4080CA
:1090A0000030010203010000040309040902270043
:1090B00001010080300904000003FF0102000705E0
:1090C000820220000007050202200000070581033C
:1090D0000800010012011001FF000240861A2375EA
:1090E00000310102030100007763682E636E000007
:1090F000555342322E3020546F2053657269616C93
:1091000020506F72740000005743483132313231C1
:1091100032545331000000007763682E636E000004
:10912000555342322E3020546F2053657269616C62
:1091300020506F7274000000574348343534353482
:1091400035545332000000007573625F726563002E
:1091500025303278202000004348333431207365B5
:1091600074206270733A25640D0A000073747220D3
:1091700025640D0A000000005345545F41444452E9
:109180004553533A25640D0A000000004745545FDB
:10919000434F4E46494755524154494F4E0D0000EA
:1091A0005345545F434F4E46494755524154494FEA
:1091B0004E0D0000434C4541525F464541545552C7
:1091C000450D00004745545F494E544552464143C2
:1091D000450D00004745545F5354415455530D000D
:1091E0005345545F4C494E455F434F44494E470DEC
:1091F00000000000253032782000000063746C20ED
:109200002530327820253032780D0A00434443203F
:10921000526571436F646525780D0A004745545FB8
:109220004C494E455F434F44494E473A25640D0A29
:10923000000000004745545F53455249414C5F537D
:10924000544154453A25640D0A0000004C494E45EE
:109250005F434F44494E4720256420256420256400
:109260002025642025640D0A0000000000D7FFFFC0
:1092700012D7FFFF36D8FFFF4CD7FFFF2CD8FFFFD8
:1092800092D8FFFF41445620706F6C6963793A2091
:109290004F4E0A0041445620706F6C6963793A2042
:1092A0004F46460A000000006D795F6E65745F618D
:1092B0006464723A25640000506572697068657272
:1092C000616C5F496E697400303132333435363742
:1092D0003839414243444546000000004E6F7469EE
:1092E000667920616C6C6F6320455252000000006B
:1092F0004E6F746966792045525220005570646142
:109300007465202578202D20496E74202578200A48
:10931000000000004552522E2E000000496E697474
:1093200069616C697A65642E2E000000446973637C
:109330006F6E6E65637465642E2E20526561736F67
:109340006E3A25780A00000041647665727469738C
:10935000696E672E2E000000436F6E6E6563746940
:109360006F6E206D61782E2E2E000000436F6E6EA2
:10937000202578202D20496E74202578200A0000B1
:10938000436F6E6E65637465642E2E00436F6E6E60
:109390006563746564204164766572746973696E8F
:1093A000672E2E00446973636F76657261626C6527
:1093B00020646F6E652C206170706C79204144567A
:1093C00020706F6C696379004572726F722E2E0087
:1093D0004572726F722E2E25780A00005265762033
:1093E00043484152310000005265762043484152C3
:1093F000332E2E004F54412043353543207375736F
:1094000070656E642025750D0A00000000010202DF
:10941000030303030404040404040404050505050C
:1094200005050505050505050505050506060606E8
:1094300006060606060606060606060606060606CC
:1094400006060606060606060606060607070707B8
:10945000070707070707070707070707070707079C
:10946000070707070707070707070707070707078C
:10947000070707070707070707070707070707077C
:109480000707070707070707070707070808080868
:10949000080808080808080808080808080808084C
:1094A000080808080808080808080808080808083C
:1094B000080808080808080808080808080808082C
:1094C000080808080808080808080808080808081C
:1094D000080808080808080808080808080808080C
:1094E00008080808080808080808080808080808FC
:1094F00008080808080808080808080808080808EC
:1095000008080808080808080808080800000000FB
:10951000000000000000000000000000000000004B
:10952000000000000000000000000000000000003B
:10953000000000000000000000000000000000002B
:10954000000000000000000000000000000000001B
:10955000000000000000000000000000000000000B
:10956000000000000000000000000000232D302B50
:1095700020000000686C4C006566674546470000A7
:109580003031323334353637383941424344454639
:1095900000000000303132333435363738396162FB
:1095A0006364656600000000F82E0020F04C002087
:1095B000020000000CE0040001000000BC8A000072
:1095C0000200000012E00400010000001E2D002037
:1095D00002000000948A000001000000888A000058
:1095E0000200000012E00400010000001C2D002019
:1095F00002000000788A000001000000708A00006C
:109600000200000012E00400010000001D2D0020F7
:1096100002000000848A0000010000007C8A000033
:109620000200000012E0040001000000272D0020CD
:1096300002000000CC8A000001000000C48A000083
:10964000962D000000000000000000000202020051
:1096500001D7070000100102020000000CE0040026
:1096600001000000048B00000200000012E0040072
:1096700001000000442E002002000000408B00008A
:1096800003000000702F00200200000016E004001C
:1096900001000000482E00200200000012E004003B
:1096A000010000005A2E002002000000448B000040
:1096B00001000000902F00200200000016E00400CE
:1096C000010000005C2E00200200000012E00400F7
:1096D000010000006E2E002002000000488B0000F8
:1096E00002000000942F00200200000016E0040099
:1096F00001000000702E00200200000012E00400B3
:1097000001000000822E0020020000004C8B0000AF
:10971000000000008C3000200200000018E004006F
:10972000030000000C3100200200000016E00400DD
:1097300001000000842E00200200000012E004005E
:1097400001000000962E002002000000508B000057
:1097500004000000103100200200000016E00400A8
:1097600001000000982E0020822F000082300000AF
:10977000000000000A0000004368617261637465C4
:10978000726973746963203100000200436861727A
:1097900061637465726973746963203200000C0040
:1097A00043686172616374657269737469632033BD
:1097B00000001000436861726163746572697374BC
:1097C000696320340000020043686172616374655C
:1097D00072697374696320350000FF7FFF00140015
:1097E0004A690000BC670000B6680000E66E000031
:1097F000FF0000000201060302E0FF05FFD707009B
:1098000000000000574D315F303030300000000064
:10981000000000000909574D315F3030303005122B
:1098200006006400020A0000000000002C95000001
:109830004C9500000C9500000000000000000000A6
:109840000000000000000000000000000000000018
:109850000000000000000000000000000000000008
:1098600000000000000000000000000000000000F8
:1098700000000000000000000000000000000000E8
:109880000000000000000000F82E00200000000092
:020000040004F6
:10D000006F00C076000000000000000090000020CB
:10D010008C020020A9BDF9F590000020000000005E
:10D0200000000000900000209000002000000000A0
:10D030000000000090000020000000009000002090
:10D0400000000000900000209000002090000020D0
:10D050009000002090000020900000209000002010
:10D0600000000000900000209000002090000020B0
:10D0700090000020900000209000002090000020F0
:10D0800090000020900000209000002090000020E0
:10D090009000002001A0011113078008F3370780DA
:10D0A00093F787083EC201000100B71700409305BF
:10D0B00070052380B704130680FA2380C70401009B
:10D0C000010083C6B70493F6F60DA385D704238029
:10D0D00007049246F3A6068001000100937605023C
:10D0E000D5CEF336078093F6860836C401000100DA
:10D0F0002380B7042380C70401000100B706140091
:10D100007D89558D88C70100010001000100238041
:10D110000704A246F3A606800100010073370780CA
:10D12000137787083AC6010001002380B7042380E3
:10D13000C7040100010001000100372700409306E9
:10D140001005A303D78023800704B247F3A7078005
:10D150000100010093078008F3B7078093F7870861
:10D160003ECE01000100B717004013077005238071
:10D17000E704130780FA2380E7040100010003C7D6
:10D18000B70413670708A385E70423800704F24761
:10D19000F3A70780010001000561828093760504F2
:10D1A000BDC6F336078093F6860836C80100010035
:10D1B0002380B7042380C70401000100B7061400D0
:10D1C000938606047D89558D88C701000100010002
:10D1D000010023800704C246F3A606800100010077
:10D1E00073370780137787083ACA0100010023804C
:10D1F000B7042380C70401000100372700409306CD
:10D200002005A303D78023800704D24781B7733753
:10D210000780137787083ACC010001002380B70408
:10D220002380C7040100010098471367070C98C7C3
:10D2300023800704E24719BF011181460146814559
:10D24000114506CE7D2A93078008F3B7078093F730
:10D2500087083EC601000100B7170040130770059C
:10D260002380E704130780FA2380E704010001000C
:10D2700003C76704136717002383E70423800704A9
:10D28000B247F3A7078001000100F24005618280E8
:10D2900041118146014681451145A52213078008A9
:10D2A000F337078093F787083EC401000100B717E2
:10D2B0000040130670052380C704930680FA23807C
:10D2C000D70401000100FD552396B702238007040F
:10D2D000A245F3A50580010001007337078013778D
:10D2E00087083AC6010001002380C7042380D704C1
:10D2F0000100010003C76704136717002383E704D5
:10D3000023800704B247F3A707800100010001A0B2
:10D31000BD473305F50201007D1575FD8280411181
:10D3200022C426C206C6AA84014463179400B240F0
:10D33000224492444101828005041305803E420448
:10D34000C13F4180DDB72303048015472303E480F8
:10D3500001002302A480828083076480E3CE07FE5D
:10D3600023030480828083076480E3CE07FE0345A5
:10D370004480828083076480E3CE07FE2302A4807A
:10D380008280411126C44AC24EC006C61377F50BEF
:10D39000AD47AA892E8995446306F700194565377C
:10D3A000653F8D444E854537FD59FD146398340122
:10D3B000B240A244124982494101828013550901B9
:10D3C0001375F50F453F2209CDB7011126CC06CEC6
:10D3D000B704080051371545BD37713769372AC67C
:10D3E000A53F32459377150089EB1365150013753A
:10D3F000F50FF240E24405618280FD14E9FC01452D
:10D40000CDBF397126DC4ADA4ED852D656D45AD21C
:10D410005ED006DE62CE66CCB7E700E07D5783AA19
:10D42000070022C603AA470023A0E71823A2E71893
:10D43000B7170040130770052380E704130780FA2D
:10D440002380E70483C74704930B75FFB684E20784
:10D4500093FBFB0F8546AA892E8B32893724004027
:10D46000E187015763FA76016308D50089461307FF
:10D4700000026313D5000157D98F93F7F70FB71C3C
:10D4800000402382FC0411472303E4801305F00FBE
:10D490005D3D094CD135636D7C11B7050700DA9508
:10D4A00037870700795563F2E504B3879500636E0B
:10D4B000F702370B0800A94733EB65016399F906BA
:10D4C00089E48144513D26850DA0DA850945553D05
:10D4D00005090345F9FFFD14050B693D81C49377E8
:10D4E000FB0FFDF7DD3569FD7D55B71700401307CC
:10D4F00070052380E704130780FA2380E70403C73D
:10D500004704418B2382E704F250B7E700E023A0F1
:10D51000571123A24711E25432445259C259325A88
:10D52000A25A125B825B724CE24C21618280A54759
:10D530006395F90685691309F00FB3069900B37472
:10D540002B01B6941349F9FFB3749900856B3379B5
:10D550006901416B9387F9FFB3F7270199E363FCF6
:10D56000340193D94900C147E3E637FF99BF056904
:10D57000C1697D19D9B71305800D63886901130549
:10D5800000026384790113051008CA85DD3B353D2F
:10D5900021DD4E99B3843441D9B7DA852D45D53391
:10D5A000CA94E30099F205097D3BA30FA9FED5BFFC
:10D5B0009387F9FF93F7F70F6361FC0C83C71C0493
:10D5C00013073008631FF70437070800636BEB0489
:10D5D000B3079B00B706100063F5D704334BEB008D
:10D5E00089476393F9068980D549E38C04ECDA8591
:10D5F0000945413B11090327C9FF91472320E480D6
:10D6000003076480E34E07FE23033481FD17EDFB1F
:10D61000FD14110B81C49377FB0FE9FF7D3371F586
:10D62000E1B5B717004003C75704B70708001377E1
:10D63000070219E3B78707007955E378FBEA330758
:10D640009B00E3FFE7F855B58547E382F9F2DA85F9
:10D650002D45053B9389F4FFE38504E6293393F7D1
:10D66000390091EB832604800327090093074900C2
:10D67000E39AE6E43E89CE84F1BFB5476396F900AC
:10D680001305900BC93135BDB1471305B00AE38BC3
:10D69000F9FE99476391F904B7050800B365BB002B
:10D6A0002D45C53181448D4BA1497539639674016F
:10D6B000832704802320F9008504E39834FF83271F
:10D6C000048013172B01635507002312F900D5BB03
:10D6D0002322F900FDB39D476399F90281451305A3
:10D6E000B0044531BD442320090023220900FD591F
:10D6F0009D3993F77400CA9703C70700FD14398D4D
:10D700002380A700E39634FF6DBBA1476392F90421
:10D710006D398144630D0B008D479304C00363088A
:10D72000FB009304000563048B019304400413750C
:10D73000C507E30895D819453931393905452131EF
:10D7400026850D3909453D314931E31C05D669BBB4
:10D7500091476399F90013056006F536F53E130508
:10D7600090090DB7E38F09D4F154A9BB9731FB1F82
:10D770009381C17F1791FB1F1301C188170500001A
:10D78000130585889735FB1F9385C5871736FB1FC3
:10D790001306C6FD63FAC5008322050023A05500C9
:10D7A00011059105E3EAC5FE170500001305857311
:10D7B0009735FB1F938585FB1386818063FAC5002F
:10D7C0008322050023A0550011059105E3EAC5FE5B
:10D7D00013858180938581816377B50023200500BF
:10D7E0001105E36DB5FEFD42739002BC8D4273904E
:10D7F0004280B72200009382828873900230973271
:10D80000FB1F9382228093E2320073905230970282
:10D8100000009382622B73901234730020300D0647
:10D82000719A81473307F5006393C70082801443E0
:10D830003387F500910714C3F5B7914763EEB7023C
:10D8400017070000130787628A05BA959C41BA97AB
:10D850008287B717004003A7470B1345F5FF698F71
:10D8600023AAE70A03A7070B698F23A8E70A03A7E0
:10D87000070A798D23A0A70A8280B717004083A6E4
:10D88000470B1347F5FFF98E23AAD70A83A6070B88
:10D89000558D23A8A70A83A6070A758F23A0E70A38
:10D8A0008280B717004003A7470B498F23AAE70AD6
:10D8B00003A7070B1345F5FF45BFB717004083A625
:10D8C000470B1347F5FF758F23AAE70A03A7070A3B
:10D8D000598D4DB7B717004003A7470B498FEDB7D8
:10D8E000B71700408847420541819377050491EBC3
:10D8F0009377F5013755E801130505803345F502A7
:10D9000082809377050C130700046397E7009377F1
:10D91000F50137459C1CCDB72165130505D08280E4
:10D92000411122C406C62A84653F2947B307E50290
:10D93000B2408D83B3D7870222449507B3D7E7025D
:10D9400037370040C207C1832316F7404101828068
:10D95000716541111305052006C6D937B737004058
:10D96000130770F82381E7400D47A381E7401307B1
:10D970000004A380E74005472387E740B240410108
:10D980008280411122C491462A84138681809D653C
:10D990002D4506C69730FB1FE780A0A6B7F7070006
:10D9A00003C70701A5476313F70001A09306001002
:10D9B00001469D6525459730FB1FE78080A42384A1
:10D9C00081802244B2409146138681809D6529451D
:10D9D00041011733FB1F6700C3A2130101BF2326B8
:10D9E00011402324814023229140232021411737D5
:10D9F000FB1F0347A7D78D476310F706B7660200E2
:10DA00000146856505459730FB1FE780809F377489
:10DA1000020037A9FDFFB7D4040022851306004099
:10DA20008A85F53BB3052401930600400A86094523
:10DA3000130404409730FB1FE780A09CE31F94FC75
:10DA400005458137B76602000146B77502000545F6
:10DA50009730FB1FE780E09A856782978320C1405B
:10DA600003248140832441400329014013010141E3
:10DA700082800111914670009D652D4506CE97303C
:10DA8000FB1FE78000980347C10089469307F7FF13
:10DA900093F7F70F63E2F6029737FB1F2388E7CC73
:10DAA0009735FB1F83C585CC170500001305453D41
:10DAB0008528F2400561828085471737FB1F2307C1
:10DAC000F7CAF9BF41111305800406C69720FB1F52
:10DAD000E780605C371700408327870A1305002022
:10DAE0008D4593E707202324F70A813B953551376D
:10DAF000ED35B24001454101828081473737004012
:10DB0000A14663C3B70082800346B740E38EC6FEDA
:10DB10003306F5000346060085072304C740D5B742
:10DB20003571CAD813094108A6DAD2D4DAD02EC387
:10DB300086DEA2DCCED6D6D2DECEE2CCE6CAEAC8FB
:10DB4000AA8432C536C73AC93ECB42CD46CF4AC475
:10DB50008145014A170B0000130B4B3683870400E5
:10DB600085E789C5C205C1815285413FF65066549B
:10DB7000D6544659B659265A965A065BF64B664C09
:10DB8000D64C464D0D618280130750026389E70031
:10DB900063140A00268A814585058504C1B791C5AD
:10DBA000C2055285C181913F014A81471307B002E6
:10DBB0009305D002130500031308000293083002F6
:10DBC0008386140013861400638EE6026341D70235
:10DBD000638D0603638E1603138706FD1377F70F15
:10DBE000A54563EDE5060147254529481DA863873E
:10DBF000B600E393A6FE93E7170019A093E7070189
:10DC0000B2847DBF93E74700E5BF93E78700CDBFB0
:10DC100093E70702F5B73307070305062E971307A7
:10DC200007FD83050600938605FD93F6F60FE37462
:10DC3000D5FE830506009306E002639AD50C8305A2
:10DC40001600254593041600938605FD93F6F60FFE
:10DC5000636FD50881462545294805A89305A0028C
:10DC60007D57E398B6FC03270900138624001109A9
:10DC7000E35107FC3307E04093E707015DBFB3863C
:10DC800006038504AE96938606FD838504001386FD
:10DC900005FD1376F60FE374C5FE038604009305B5
:10DCA00080066308B6001376F6FD9305C00463137F
:10DCB000B60085040386040093058005630CB60452
:10DCC00093058007630AB604930750026307F600C2
:10DCD000854548002302F1000D3583870400A9CF54
:10DCE000854548002302F100093D81457DB51305B6
:10DCF000A0028146E393A5FA832609009304260037
:10DD00001306490063D306008146328979B7B2848D
:10DD1000FD5661B793E7070413F607045A8809E62E
:10DD2000170800001308081793FA070163880A0010
:10DD3000F99B9305000201A8FD1445BF13F61700D7
:10DD4000930500037DD6A302B1002303010093FBDA
:10DD500007020326090063830B00791741E61306C7
:10DD600000032306C1008549368C63D336014E8CEF
:10DD7000C58B330487418DE7A28C130D00026341EC
:10DD800090099307F4FF228763530400014733840B
:10DD9000E7408307610089C7854513056100B13BF2
:10DDA00063820B0293070003854513057100A303EB
:10DDB000F100A13393078007854513057100A30384
:10DDC000F100253B639D0A00A28A63435005930737
:10DDD000F4FF22876353040001473384E740930A2A
:10DDE0000003A1A06C0081491375F600429503451C
:10DDF0000500118285092380A500850575F6ADB75C
:10DE0000854513057100A303A101FD1CFD3185BFEC
:10DE1000854513055100D531FD1A45BF85451305CC
:10DE20007100A30351017D1CC939E3C989FFFD5A63
:10DE3000FD196398590193090002634F800011098D
:10DE40006DB57C00CE9783C707008545130571002B
:10DE5000A303F1005D31E9BF854513057100A303FC
:10DE600031017D145939D1BFEAF9FFFF12FAFFFFE2
:10DE70003AFAFFFF52FAFFFF6CFAFFFF496D616744
:10DE80006520466C616720253032780A000000006A
:10DE90003031323334353637383961626364656620
:10DEA0006768696A6B6C6D6E6F707172737475768A
:10DEB0007778797A000000003031323334353637E4
:10DEC00038394142434445464748494A4B4C4D4EF8
:10DED0004F505152535455565758595A000000004C
:08DEE000FF000000000000003B
:10E000006F00E2110000000000180118002801282C
:10E0100002280328002901290229032904290529A6
:10E02000062907290829002A012A022A032A042A84
:10E03000052AA62A78E8060056FD0400F002002012
:10E0400076030020C00200208E0200201C02002067
:10E050005EFF0400A6FF04004C010500D803050084
:10E06000C6040500B4FB040072FA040034FB04008B
:10E07000C4FA0400B60A05000C05002034FF0400B1
:10E0800082070500CC9F0600C4A106003CA2060042
:10E09000F66106002A62060056180600960D060074
:10E0A000A6990600B80705004669060004AA0500FF
:10E0B00092AA0500EAAA050046130500921305007E
:10E0C000FC1105002C660500E6600500C26F050026
:10E0D000927305003E7705001A530500B8520500FB
:10E0E000A0560500665305008E5205001253050028
:10E0F00040520500EA53050042540500F253050062
:10E10000F6530500905405004A5405007C54050060
:10E110009459050098590500E6530500EE53050093
:10E120008E540500965905003E550500065B050016
:10E130008685050004860500428605009068050076
:10E14000A8680500E4680500F24C0500104E0500C3
:10E15000864E05001C320500C22C05000843050050
:10E16000402D05006C3E0500C0C9060040C20600F7
:10E170001CC7060022DD060008DC060094DF06004E
:10E1800084DF06008CDF0600CCDF06005AB40600F0
:10E19000000000000000000000000000000000007F
:10E1A0003CE0060004DA06009AD9060000000000F0
:10E1B000000000000000000000000000000000005F
:10E1C00092830600B0710600367506000E730600D5
:10E1D000647D06004E9A0600000000008EB4060022
:10E1E000440C050066630600266906001E6A0600E8
:10E1F0000000000000000000000000008C6C050022
:10E20000C4820600000000000000000000000000C2
:10E21000607106001C0700203E640600B8DF06009F
:10E22000000000000000000088DF06006403050015
:10E23000E2690500C0DF0600688406003685060036
:10E24000B085060062C70600BCDF0600C4DF06001A
:10E25000220D0600C8DF060026110020EC10002069
:10E2600000000000000000000000000000000000AE
:10E27000000000000000000000000000000000009E
:10E280006373B60082801C419105110523AEF5FE33
:10E29000C5BFB72700203727002093878780130743
:10E2A00047D86373F700828023A007009107D5BF8A
:10E2B0004111B7E700E022C480433707200006C6BB
:10E2C000798C23A0E7180F10000011C199E5B7E77A
:10E2D00000E023A08710014545A893073500C20739
:10E2E000C183F19BC207C183130740036366F70232
:10E2F000372700200325079337270020832687929E
:10E300006391A602372700200327079C69D3C20721
:10E31000DD8D0545029765BF372700200325C7928D
:10E32000E1BF035765002DE7035745006362F70619
:10E33000B72600203306F7402148938686936378FA
:10E34000C8028328050003D86600138687001D8F46
:10E350002A9661172312E6002320160123130600D4
:10E3600010C12312F500130788FF2393E60023133F
:10E37000B50083D566002105B387F5402393F600E9
:10E38000B7E700E023A08710B24022444101828019
:10E390000841BDB7B7E700E003A807003707200032
:10E3A00023A0E7183378E8000F10000001E523A050
:10E3B00007118280B727002003AE0793B7270020FC
:10E3C00003A387928146F28763FC670A83A807004C
:10E3D000636BF50A63E9A80A138787006362E50A9D
:10E3E00003D66700216705076319E600372600207A
:10E3F0000347068905072308E6883726002013050A
:10E40000869383D5470003576500239307001306BF
:10E4100086932E97420741832313E5006387C70342
:10E42000372500200325C5926301F50203D5660058
:10E4300009ED83D7460023A016012107BE95A1054B
:10E440002392B6002313E600B6879843630A670257
:10E45000B726002083A6C6926304D70283566700BE
:10E4600085E283D64700835547001843A106AE9640
:10E470002392D70098C383576600A1072313F600A1
:10E48000B7E700E02DB7BE86C6873DBFB7E700E01F
:10E490009843B706200023A0D718758F0F100000EF
:10E4A00001C599C1814711E6B7E700E023A0E71055
:10E4B0008280B386F50003C80600B306F500850721
:10E4C00023800601E317F6FEC5B737E700E01C43DB
:10E4D000B70620002320D718F58F0F10000019C1B0
:10E4E00091C111E637E700E02320F7108280910503
:10E4F00003A7C5FF11057D16232EE5FEDDB737E71F
:10E5000000E01C43B70620002320D718F58F0F101A
:10E51000000001C53307C50011E637E700E02320FE
:10E52000F71082800505A30FB5FEE31DE5FEF5B7E4
:10E53000B7E700E09843B706200023A0D718758FEF
:10E540000F1000008147B306F5008386060099E6A8
:10E55000B7E600E023A0E6103E8582808507E5B798
:10E5600037E700E01C43B70620002320D718F58FBB
:10E570000F10000001C599C1014711EA37E700E01B
:10E580002320F710054582800507E309E6FE3308DE
:10E59000E500B386E5000348080083C60600E305EE
:10E5A000D8FE37E700E02320F7100145828037E7E7
:10E5B00000E01C43B70620002320D718F58F0F106A
:10E5C00000001307F6FFBA952A966317C50037E7D0
:10E5D00000E02320F7108280FD1503C71500050514
:10E5E000A30FE5FEDDB737E700E01C43B7062000C8
:10E5F0002320D718F58F0F10000001C53307C50081
:10E6000019E637E700E02320F71001458280050571
:10E610008346F5FFE397B6FEE31BE5FE37E700E030
:10E620002320F71005458280797126D2B724002077
:10E6300022D403A4C49806D64AD04ECE52CC56CA91
:10E640005AC85EC662C44DC8372A00203729002048
:10E65000B7290020814BB72A002037CBC901130A04
:10E660000A99130989939389C99D8357240099EFC7
:10E670005C44639A0B0023A6F498032CC400228503
:10E68000113B6284B9A823A6FB00C5BF83A74A98A3
:10E6900082971C443307F5406376F50003A74900D1
:10E6A0001D8F2A979306FB3763ECE60623280900A3
:10E6B0008355240003450400970005E0E78060B11E
:10E6C0005C405844B1C70C4403A64900AE97BE86CF
:10E6D00063E4B70063E4C700B386C74014C4A28BE9
:10E6E0003A8441F4B727002093878793984B894653
:10E6F00063FCE604791798CBB25022549254025925
:10E70000F249624AD24A424BB24B224C4561828066
:10E7100063950B0023A6E4988DB723A6EB00B1BF49
:10E7200003274A0219CB63EDA7003385A74083274F
:10E7300009016374F5002328A900A28B404455B752
:10E7400003A74900BA97D5B723A8070075B7B7271D
:10E75000002003A7479D411122C406C63E8411C371
:10E760000297B727002083C7279893F7F70F99E3FD
:10E77000232A049CB24022444101828001114EC6EA
:10E78000B729002083A7499606CE22CC26CA4AC8BC
:10E7900052C456C281C7829723A20996B72400208B
:10E7A000938744C883C7570037240020938444C804
:10E7B000858B1304449681CF83C774001947631671
:10E7C000F70EA3820400EF0030615C4482971C4482
:10E7D00091C3829737240020372900209307849320
:10E7E0000327899803C61700130A849383478493E9
:10E7F00093961700BA9683D60600F9C2834784938E
:10E8000063E8C70C83A74996230C0492639407120C
:10E81000B727002083A74798638E0710B7270020EB
:10E8200083A7079E2328FA00013583C7B4006393AA
:10E83000071083C7940081CF83C7740093F7F70F45
:10E8400099E7A3840400976006E0E780E007B72714
:10E85000002083A7479BF9CF83270A01E1CF83C715
:10E86000740015476368F70CB7270020938707CD1E
:10E8700083C7C700918BDDEFB727002083C7279898
:10E8800093F7F70FC5EB83461A000326899863CCEC
:10E89000D70A6244F240D2444249B249224A924ADB
:10E8A0000561170305E0670043F183C774001D4746
:10E8B000E31FF7F0A3820400EF0010521C4839B7A1
:10E8C000850793F7F70F230CF492E3E1C7F23DB706
:10E8D00086073E978355070023100700034584935E
:10E8E000B727002083A7079613172500B72A002013
:10E8F000BA979C4323900A98829783D70A98034734
:10E90000849393C7F7FF7D8D93171700032789988A
:10E910003E97835707005D8D2310A700834784939C
:10E9200081C78507230CF4920347849383471A0019
:10E93000E37AF7ECF2406244D2444249B249224AB7
:10E94000924A056182801397170032970357070098
:10E9500075F385072DBF37C700408326C720B7074B
:10E96000FCFFFD17F58F2326F72001000100B727D4
:10E97000002093878793C84F832787262326D72095
:10E980006A0593C7F7FF99835D8D8280B7270020C2
:10E9900003A3079F6303030002831305F00F828024
:10E9A0000327851163000712411122C406C683475D
:10E9B000C5008345E5042A8493F7C70F2306F500B5
:10E9C000834697000356C70013958601618563F15E
:10E9D000C508635A05060345870093F6F607A304A6
:10E9E000D700054693E627006314C50093E6170099
:10E9F0002306D4005C4389075CC3A30AB400032543
:10EA000004112E864C430905513483278411034693
:10EA10005401D44303D7C700B296118FD4C32396B1
:10EA2000E7008947A30DF400B727002003476403DC
:10EA300083C7279A6378F7048347C40093E70701E5
:10EA40002306F40081A093E717002306F40075B7AE
:10EA50009376F60F635D050203458700854513E64F
:10EA600027006314B50013E617002306C400A30AA9
:10EA7000D400A30407008547A30DF4008327841165
:10EA80009C43DDF3B240224401454101828093E77B
:10EA900017002306F400A30AD400A30407000325EB
:10EAA00004114C430905DD328327841103465401C8
:10EAB000D44303D7C700B296118FD4C32396E7007F
:10EAC0008D475DBF05458280B727002083A7C7C655
:10EAD000411122C406C6858B2A84DDEB41651305EE
:10EAE00025F5972006E0E78040E05DC18347A5005B
:10EAF0002315F50083270412B5E72320A41223224F
:10EB0000A41285472311F4042320050083476401E0
:10EB100054412316F5000347D4002304E5000547BC
:10EB2000A304E50037270020032787CA13851702AF
:10EB300015811C437D151375F50F9CC25C43DCC227
:10EB40001C479CC65C47DCC61C4B9CCA5C4BDCCAA1
:10EB50001C4F9CCE5C4FDCCE19CD9386060213076A
:10EB60000702C1BF8327441288C38357240423228A
:10EB7000A412850741BFB7270020938787B403D726
:10EB8000870005072394E700B240224441018280B8
:10EB90008347C40023090400054593C747002306A3
:10EBA000F400DDB78347850193F7E70FDDEB83477B
:10EBB0009501C5EB034625018346C50009CA3727E1
:10EBC0000020834565030347379A63E7E50013F7A1
:10EBD000060149CB014709C6C18A0357E51881C61A
:10EBE0008356251936973DCFB727002003D5479E7A
:10EBF0001307C71237460F00B335A702411113069A
:10EC00000624814622C426C206C67D543305A702C7
:10EC100097D006E0E780E07EB727002083C7779A89
:10EC2000B384A700B727002003A787BD8327070960
:10EC300063F387003E84184375FBB727002083A742
:10EC40004798829781476364A400B307A440B24009
:10EC50002244B3B7970093C7170092443E85410101
:10EC6000828081473E858280B727002003A7C7CADC
:10EC70003C5BFDFF010001008280011122CC4AC8EB
:10EC80004EC606CE26CA52C456C25AC00347B50065
:10EC900085472A842E8983290509631AF71E83571D
:10ECA0000508035BC503372A00209306CA9D83DA53
:10ECB0008600130ACA9D63F4671B834605016390AF
:10ECC000E61A03278511631C07180327450A6318F2
:10ECD00007188346F5001D476393E6180355A503FF
:10ECE000330BFB409307204E33056503832444090F
:10ECF00037460F008146130606243305F502B72771
:10ED0000002083C7679AB3549502B3B5AA02BE9494
:10ED1000C204C180231394083385AA0297D006E069
:10ED2000E780206EB307350133B5A7002E953E87E7
:10ED300083264A0019E163E4D7003387D740B384C0
:10ED40005403B7460F009387F623938606242320A7
:10ED5000E900A697B3D7D702DA97636CF70E1D8F39
:10ED60002320E900B729002083A7499883240900BC
:10ED7000829763E1A4123385A4406350050C83A7F6
:10ED80004998372B0020130BCB9D8297032709004E
:10ED90006368E510198D8357E40303578B008E07D2
:10EDA000B387E7021307003293870719B3D7E70247
:10EDB00063EDA70E374A0F00930AFA23130A0A24B9
:10EDC0008357040485072310F4048347041499E34C
:10EDD0002285512A2285971006E0E78000D87DE140
:10EDE000832604098327C40803274B00B6973E8572
:10EDF00063E4D70063E4E7003385E7408347F40129
:10EE0000835464082328A4088507A30FF4008357BC
:10EE10008B00B384F402D694B3D444036363950C9B
:10EE2000B304954083A7499823209900829763EE05
:10EE3000A40A3385A440E34505F8B727002083C71B
:10EE4000779A63E2A708B727002023A087BE014571
:10EE50009DA883264A00B387F6403E9711B7835496
:10EE6000640837470F009307F723B3845403BE9415
:10EE700093070724B3D7F40263E7F900B387F94097
:10EE80002320F900C5B503274A00BA99C5BF23A0BE
:10EE90003501C9BDB727002083A7079EBE94E1BDF9
:10EEA00083274B00998F3E95FDB5A145228597108C
:10EEB00006E0E780A0C3A305A402B727002083A72C
:10EEC000079C81EF7D55F2406244D2444249B249E9
:10EED000224A924A024B05618280894515458297F4
:10EEE000D5B7B3049740AA9435BF83274B00BE948F
:10EEF00089B72DC901116C0022CC06CE2A84B53BFE
:10EF000029CDFD576305F502372700201307079920
:10EF10005453B2479DC62547637FF700D9173EC6B5
:10EF2000B2450345940297F004E0E7808041F24047
:10EF3000624405618280372700200327079EBA9725
:10EF4000F1BF0347770163E4E700998FC9BFB72694
:10EF5000002083A6069EB697CDBF971006E0E780F7
:10EF6000404DF1B78280797126D206D622D44AD09C
:10EF70004ECE52CC56CA5AC85EC683475503034488
:10EF80007513AA843E941374F40F9307400263F63A
:10EF900087001304B4FD1374F40F03AA841383AA27
:10EFA000C413A38B841222865285D68597D006E09F
:10EFB000E7806042058915E503CBD41201498149F8
:10EFC000337B6403930B50024A865285D68597D0D3
:10EFD00006E0E7804040058915C563916903137415
:10EFE000F90F238B8412B250225492540259F249E1
:10EFF000624AD24A424BB24B456182808509E2099E
:10F0000093D989410509E31179FDE1BF832785097A
:10F0100003560504797193D60701BD8EC206C182DD
:10F02000358E1357764093575640898B058B5D8FED
:10F0300093573640918B5D8F93571640A18B5D8F10
:10F0400093171600C18B5D8F9317360093F7070255
:10F050005D8F931756009355860093F707041E069D
:10F060005D8F1376F60F518F93D7554013D63540E9
:10F07000118A898BD18F13D67540D18F13D6154045
:10F08000218AD18F13961500418AD18F13963500AE
:10F0900013760602D18F13965500137606049E054B
:10F0A000D18F93F5F50FCD8FA20745465D8F3307BE
:10F0B000C70222D42A8426D252CC56CA032A8413E9
:10F0C000832AC4135AC806D63697420741839357FA
:10F0D0007740135557400989858BC98F13553740A1
:10F0E0001189C98F135517402189C98F131517002E
:10F0F0004189C98F1315370013750502C98F131580
:10F10000570093558700137505041E07C98F1377A1
:10F11000F70FD98F13D5354013D755401189098B77
:10F12000498F13D57540498F13D515402189498FD3
:10F13000139515004189498F139535001375050204
:10F14000498F13955500137505049E05498F93F556
:10F15000F50F4D8F2207D98FB387C7024AD04ECE05
:10F160005EC662C4B697C207C18313D7774013D572
:10F1700057400989058B498F13D537401189498F2D
:10F1800013D517402189498F139517004189498F5D
:10F190001395370013750502498F1395570093D5C2
:10F1A0008700137505049E07498F93F7F70FD98FD2
:10F1B00013D5354013D755401189098B498F13D585
:10F1C0007540498F13D515402189498F1395150036
:10F1D0004189498F1395350013750502498F1395A1
:10F1E0005500137505049E05498F93F5F50F4D8F56
:10F1F0002207D98FB387C702130650025285D685DE
:10F20000B697BD8E93940601C18033F6C402137B7A
:10F21000F60F97D006E0E780001C05890DED8347C7
:10F22000D41201498149B3849702130C5002C18062
:10F230004A865285D68597D006E0E780C0190589B1
:10F24000937BF90F11C563863403850993F9F90F90
:10F250000509E31F89FD230B6413B2502254925415
:10F260000259F249624AD24A424BB24B224C4561A2
:10F2700082805E8BCDB70111B727002022CC03A47A
:10F2800087C026CA4AC84EC606CEAA8413092500DE
:10F29000854915C083C7140003473400858B630478
:10F2A000F700405CFDB71946930544004A85EFF02E
:10F2B0002FABE31835FF2285F2406244D244424925
:10F2C000B249056182804111B727002022C403A4FE
:10F2D00087C026C24AC006C693042500054901E836
:10F2E0002285B24022449244024941018280A6858F
:10F2F0001305A402974006E0E780C08DE30225FFD6
:10F30000405CF1BF0111B727002022CC03A407C045
:10F3100026CA06CE2AC42EC6854419E40145F24009
:10F320006244D24405618280834791000347140000
:10F33000858B6304F7000044CDB719469305A100FF
:10F3400013052400EFF0CFA1E31795FE0545C1BFDB
:10F35000EFF0EFBF73000000000000009712000004
:10F36000938262890383020023800200630F0300FB
:10F37000F32510342EC0970500009385A5FD7390EA
:10F380001534EF00A0477300203086DCEF00004703
:10F39000E65082800000B726002003A706C80111AE
:10F3A0004AC81C5F4EC606CE998322CC26CA858BDE
:10F3B0003689B7290020ADCF9307000637240020F7
:10F3C0001CDF930744C883C7670013070008930432
:10F3D00044C86319F70083A7C9C79C4393F7070480
:10F3E0002383F400834744C893F7070489CFB727E2
:10F3F000002083A747988297C8CC834744C893F7D7
:10F40000F70B2302F4C883C7440093F707048DE386
:10F410008547A382F400B727002083A7C7CA370710
:10F42000020098C7130700FC2382E4009848F8D331
:10F43000032709C81C5F9183858B95C31C5F93E7E5
:10F4400007011CDFB727002083A7C7CA054723A2EF
:10F450000706B7270020938747C82382E70083A7C2
:10F46000C9C7D8430583058B19C7D843759BD8C333
:10F47000D843799BD8C3F2406244D2444249B2494E
:10F4800005618280093F730020309317D50063DF48
:10F490000700B727002083A7C7CA7D57B8D7B7276B
:10F4A000002093878793D84F0507D8CF937785009F
:10F4B00099CFB7270020938747C803C72700136752
:10F4C00017002381E700130700F82382E7009377F2
:10F4D000150099CBB7270020938747C803C71700AB
:10F4E00013671700A380E700937765008DC7137734
:10F4F0004500B727002059CF03C747C81367170037
:10F500002382E7C8B727002003A707C85C57F19BF1
:10F5100093E717005CD79317F50063D20702B7276C
:10F520000020138787B483460707938787B4C18A6F
:10F53000BDCA8347070793E707022308F706931717
:10F54000E50063D60702B7270020938747C803C7A3
:10F550004700620761876355070005472382E7007C
:10F56000B727002083A7C7CA3707020098C7931799
:10F57000C50063D00702B7270020938787B403C76D
:10F580001707058B29C303C7170713672700A3882D
:10F59000E7068280938747C803C7370013671700C1
:10F5A000A381E70085B703C7070789463D8B63083A
:10F5B000D70003C707078D463D8BE312D7F81147E5
:10F5C0002388E706ADBF03C71707118B79D303C79D
:10F5D00017071367870065BFB7270020B7260020ED
:10F5E00003A6C7CA938746C803C746C8058B11C779
:10F5F00023820700A3820700828003C71700058BC0
:10F6000065FB785275F303C75700EDB73727002025
:10F61000032807C8832788039583858BC1E311C618
:10F6200083270803BD832300F60085CA832707C804
:10F63000985B4607935767016356070093E707C037
:10F64000C207C18303970600C207C18709C7BA97DB
:10F650000947B3C7E7022390F6009DCD8345150007
:10F6600085CDB7270020938747C883C767001387D6
:10F670009500894593F7070485C33A9583470500AC
:10F680000547994593F6F7066398E600E207E18798
:10F69000814563D30700B9452E8582808545EDBF3E
:10F6A000411126C206C622C44AC0B724002035ED47
:10F6B00083A6C4CAAE87F8527DFF372900201309FC
:10F6C00049C82301090037F400E03E85832704D1AF
:10F6D000B285ED9B2328F4D0832704D193E78702DA
:10F6E0002328F4D073005010975006E0E780E00A1A
:10F6F000B727002083A707C8B70680009843558F17
:10F7000098C3D857719BD8D783A7C4CAA30209004E
:10F71000A3000900094798C3832704D193E7870012
:10F720002328F4D07300501005A08D476314F5040E
:10F73000B727002083A707C8B70680009843558FD6
:10F7400098C3D857719BD8D783A6C4CAB7270020BF
:10F75000938747C803C72700058B19E703C73700FE
:10F76000058B51CB23820700B240224492440249C8
:10F77000410182808547E319F5FCB7F700E003A754
:10F7800007D16D9B23A8E7D003A707D11367870292
:10F7900023A8E7D07300501003A7C4CA8177FD17D0
:10F7A0005447F58F5CC70F10000003A7C4CAB70702
:10F7B0000200130600F81CC7B7270020938747C82C
:10F7C0002382C700B727002083A707C89C439D83D7
:10F7D000858B639FA700930760197CD354C737F7C5
:10F7E00000E0832707D193E787002328F7D01DBFC8
:10F7F0009307E01BDDB7F85231FFBDB7B7270020F4
:10F8000083A7C7CA8847D847798D09C988C7B7274A
:10F81000002003A3878963030300028382803727C4
:10F820000020B7260020138606CB130707CD834799
:10F83000D7008345B601484AAE97FD8BB355F50016
:10F84000A300F600A306F700858995E90347170191
:10F85000814613080002B3F7E7020147B355E500FC
:10F8600085899378F70F89C96395D700A30016019E
:10F870008280850693F6F60F0507E31107FF828065
:10F88000B727002083A74798011122CC26CA52C46B
:10F8900006CE4AC84EC68297B7240020938704CD6F
:10F8A0008047014A6301A406938404CD63668506FC
:10F8B000018D37270020930707CB83C7A701135477
:10F8C0005500137AF501130907CB636BF402B729CE
:10F8D00000209389C99DA1378346A90103A884000C
:10F8E00083A54900139756004297158C3A866364A6
:10F8F00007016364B7003306B74090C4E37DD4FCCE
:10F900001604336A4401F24062445285D2444249AB
:10F91000B249224A05618280B727002083A7079E4B
:10F9200033848740229571B7B727002003A7C7CA41
:10F930008967938707F47CD3B727002083A707D074
:10F9400083A60709139656006358060083A6070985
:10F9500013966600634406007453FDF28280000033
:10F96000B72700203727002083A707930327879214
:10F9700001456313F700828083D6670081E683D652
:10F98000470036959C43F5B7B727002083A5079914
:10F990003727002093870799138605222328C792CB
:10F9A00003D74700938785FFB72600204111BA97F8
:10F9B000056523A4F69206C61D05935637006374A9
:10F9C000E500930600203307D600372500202326C4
:10F9D000E59223A0E522E1162312D60023130600A8
:10F9E0001CC3998FE1172312F700231307008D3FE3
:10F9F000B240B7270020239FA79241018280B727FA
:10FA00000020B726002083A7079303A686922A87A3
:10FA1000B305B5406314F6003A8529A8938687009C
:10FA20009C43E369D7FEE377F7FE2E85E3E4D5FE3A
:10FA3000E3F2F5FE828023AC05FE1C4191E7010054
:10FA400001000CC18280BA8703A787FF6DFF23AC3A
:10FA5000B7FE8280184183A785FF6319B7001CC1D8
:10FA6000FD5723AC05FE238FF5FE8280232CF6FE86
:10FA7000C5BF411122C437E400E026C20440370765
:10FA8000200006C6F98C2320E4180F10000009E9B5
:10FA9000232094101545B2402244924441018280B3
:10FAA0000347E5FF9307F00F6306F7002320941048
:10FAB0001145D5B79700FB1FE7800067014523205C
:10FAC0009410D1BF411126C2B7E400E04AC003A997
:10FAD0000400B707200006C622C43379F90023A02A
:10FAE000F4180F10000009E923A02411B2402244A9
:10FAF00092440249410182809565938505D0C98D64
:10FB00002A842105C2054205C18141819700FB1F5E
:10FB1000E780405301CDFD572320050023128500C7
:10FB20002303F50023A024112105C9B723A0241124
:10FB300001456DBF0111B7E700E04AC803A90700FE
:10FB40004EC63707200006CE22CC26CAAA893379B2
:10FB5000E90023A0E7180F10000037250020032438
:10FB600045938144014619E499E8A1654E85EF006B
:10FB7000B00631A88347E4FF6397370395C8A6858D
:10FB800013054593C13D75D0A1654E85C92EF24040
:10FB90006244B7E700E023A0271126854249D244FA
:10FBA000B2490561828091E02286032484FF65BF0B
:10FBB000A284E5BF41114AC037E900E022C4032412
:10FBC00009003707200006C626C2798C2320E918D1
:10FBD0000F10000089E523208910154515A0B727CF
:10FBE000002083C79793AA842E8563F5F400894784
:10FBF00063EE9700BD3DB7E700E023A087100D45F9
:10FC0000B2402244924402494101828083A785FF89
:10FC100099E703C7E5FF9307F00F6308F700913DED
:10FC2000B7E700E023A087104DBF37250020238FC2
:10FC300095FE130545930135A16526850D260145E1
:10FC40002320891075BFB727002023AA079282803E
:10FC5000B727002083A7C79899E33E85828003D702
:10FC600027006316B70003C70700E308A7FEDC47B9
:10FC7000E5B7B9CD011106CE22CC26CA8147C146CF
:10FC800033D7F540058B21C312053E953147330527
:10FC9000E502372700208324079D05443314F40030
:10FCA0002EC642044180AA949C40C8408297B24527
:10FCB00023A0040023A20400A18DF2406244D24498
:10FCC0002E85056182808507E39CD7FA0144EDB754
:10FCD0002E858280BDCD797122D406D626D24AD017
:10FCE0004ECE01444147B3D78540858BB1CF120535
:10FCF000314722953305E502B727002003A9079D68
:10FD00008544B3948400C204C180BE892A99032724
:10FD1000090011C7032549002EC60297B245314795
:10FD20003304E40283A7099D3E941C4489E7232001
:10FD3000090023220900B2502254A58D0259925481
:10FD4000F2492E85456182800504E31EE4F8814472
:10FD5000DDB72E8582804111B7E700E026C28443DB
:10FD60003707200006C622C4F98C23A0E7180F101D
:10FD70000000B727002083A7079B37140020130437
:10FD8000847D91C782971C403E9508C031A0B7275B
:10FD9000002083A74798FDF70840B74703009387E3
:10FDA000D73F3305F502B7A72600938737ECB2405B
:10FDB0003E9508C02244B7E700E023A09710924484
:10FDC000410182800111B7E700E022CC80434AC89C
:10FDD0003707200006CE26CA2A892E86798C23A0D2
:10FDE000E7180F100000131506019305F004418178
:10FDF00032C69700FB1FE780E024AA8419C532466B
:10FE0000CA859700FB1FE780A041B7E700E023A069
:10FE10008710F240624426854249D24405618280BF
:10FE20007971B7E700E022D480433708200006D676
:10FE300026D24AD04ECE52CC56CA5AC85EC662C4EA
:10FE40003374040123A007190F10000005E123A05B
:10FE500087100945B250225492540259F249624A1D
:10FE6000D24A424BB24B224C45618280B7270020D8
:10FE700083A74798BA8A368AB28B2E8BAA89829733
:10FE8000B727002003A7079D3E898144B146C1479B
:10FE9000338CD40233068701104241E6C165938555
:10FEA00005F041459700FB1FE780C01919EDB72702
:10FEB000002083A7079C81C7814511458297B7E73A
:10FEC00000E023A087102D4571B7B727002003A7B6
:10FED000C79821E723A6A798230005008327099D3B
:10FEE00005473317970023260500232475012311A6
:10FEF000E50023225501E29723A0370123A26701E1
:10FF000023A4570163040A0023009A00B7E700E026
:10FF100023A0871001453DBF3E875C47F5FF48C7DA
:10FF200065BF8504E396F4F6B7E700E023A08710E9
:10FF300021450DB7B727002083A7879D411122C413
:10FF400006C6372400201304849389C782975C482F
:10FF50003E9548C84848B240224441018280B7E7F4
:10FF600000E09843B706200023A0D718758F0F1024
:10FF70000000B726002083C696936372D502372609
:10FF800000209316150003258698369583560500A4
:10FF9000D58D2310B50023A0E7100145828023A052
:10FFA000E7100D458280B7E700E09843B7062000D0
:10FFB00023A0D718758F0F100000B726002083C626
:10FFC00096936374D50237260020931615000325F7
:10FFD000869893C5F5FF369583560500F58D231059
:10FFE000B50023A0E7100145828023A0E7100D454E
:10FFF0008280011137E700E026CA0443B7062000DB
:020000040005F5
:1000000006CE22CC4AC84EC652C4F58C2320D7183F
:100010000F100000130705FF1377F70FFD4763E28A
:10002000E70AB146B306D502B727002003A7079D0C
:1000300036971C43D9C71359450005443D893315EC
:10004000A400131405014180AE894A85A2850931B7
:100050002A8A39C9A2854A85B937B727002083A7DC
:100060004798372900201309C99D82978357890033
:100070002A848146B385370313060064B3B7370378
:1000800013850532B335B500BE95EFE04110B307D7
:1000900085003E878326490063E4A70063E4D70018
:1000A0003387D7402324EA00B7E700E023A0971066
:1000B0000145F2406244D2444249B249224A0561B4
:1000C0008280B7E700E023A097100945DDB7011152
:1000D000B7E700E026CA84433707200006CE22CCCB
:1000E0004AC84EC6F98C23A0E7180F100000BD4780
:1000F00063E8A70431473307E502B727002083A749
:10010000079DBA979C438DCF05443314A400420445
:1001100041802E890145A285253EAA8911C5A28567
:100120000145513523A42901B7E700E023A097102A
:100130000145F2406244D2444249B249056182809D
:10014000B7E700E023A097100945E5B779714AD0D9
:1001500037E900E026D283240900B707200006D63D
:1001600022D44ECE52CC56CA5AC85EC6FD8C23202D
:10017000F9180F100000B727002083C79793637802
:10018000F500B727002083AB479863970B00B7E7CC
:1001900000E023A0971099A0B72900209389C99D5A
:1001A000AE8A03AB490083D58900B74736FE9387F3
:1001B00007C83E9BB387C5022A84328A8146B3B5FD
:1001C000C50213850732B337F50013060064BE95E8
:1001D000EFD0F17B6370AB02232099100145B25040
:1001E000225492540259F249624AD24A424BB24BCB
:1001F00045618280829B83D589002A891306006429
:10020000B38745038146B3B5450313850732B3373A
:10021000F500BE95EFD0B177B30725013E8903A75E
:10022000490063E4A70063E4E7003389E740D6852B
:100230002285393C09C923242501B7E700E023A022
:100240009710054569BF936504F0C205C18141451A
:100250009700FB1FE78000DF11E9B727002083A785
:10026000079C95D7A2851145829715B7372700209F
:100270008327C79895E32326A7988547232605005B
:10028000232425012311550123008500A300F50037
:10029000232205005DB7BA87D84775FFC8C7F1BFED
:1002A0007971B7E700E026D284433707200006D6ED
:1002B00022D44AD04ECE52CC56CA5AC85EC662C468
:1002C00066C26AC0F98C23A0E7180F1000002DC188
:1002D0004144B689B28A2E8A2A89B14C372B002034
:1002E000054D130C0003B30B940303270B9D5E977E
:1002F0001C43A5E39375F400B315BD0013554440AA
:10030000C2055686C1811375F50F893539C183271A
:100310000B9DDE9723A0270123A2470163840900D8
:1003200023808900B7E700E023A09710014521A0B2
:1003300023A097100945B250225492540259F24911
:10034000624AD24A424BB24B224C924C024D45611A
:1003500082800504E31984F9B7E700E023A0971031
:100360002145D1BF0111B7E700E026CA844322CC62
:100370004AC84EC63707200006CE2A84AE89328985
:10038000F98C23A0E7180F100000C9332285CE8511
:10039000C1302A8405C5B727002083D5479E1306A0
:1003A00000648146B3872503B3B52503138507325F
:1003B000B337F500BE95EFD0915D48C013351400FA
:1003C000F2406244B7E700E023A097104249D244CC
:1003D000B2490E05056182800111B7E700E04AC805
:1003E00003A9070022CC4EC63707200006CE26CA36
:1003F000AA892E843379E90023A0E7180F100000A2
:10040000EFF01F85AA8419C123110500A2854E852E
:10041000593EB727002083C7879363993701B727D1
:10042000002003D70798598C23908798B7E700E0FE
:1004300023A02711014591E01945F2406244D244BE
:100440004249B2490561828001114AC837E900E09A
:1004500022CC03240900B707200006CE26CA4EC6C8
:100460007D8C2320F9180F1000009307F00263E63B
:10047000A704B147B304F502B729002083A7099D5B
:10048000A6979C439DCB9377F5008545B395F500E2
:10049000C205C1811181893783A7099D0145A697AE
:1004A00023A0070023A2070023208910F240624402
:1004B000D2444249B24905618280B7E700E023A0F7
:1004C00087100945E5B74111B7E700E026C284432C
:1004D00006C622C437072000F98C23A0E7180F10A6
:1004E0000000EFF0EFF619E90145B2402244B7E70A
:1004F00000E023A09710924441018280B72700209A
:1005000083A7479800458297B72700209387C79D08
:100510006368A402D843B74636FE938606C83305FF
:10052000A4403697E372E5FC13070064B335E50297
:1005300003D6870081463305E502EFD0514575B7F4
:10054000D8433A94C1BF411122C426C237240020A7
:10055000B72400201307C49D938484939448584380
:10056000B727002006C683A747981304C49D63924B
:10057000E60882975440B74736FE938707C8B69778
:100580003387A7003A856364F7006364D7003305B7
:10059000D740B7240020938744C8DC53938444C8D1
:1005A00099CBB727002083A607D03707CDFF7D174B
:1005B0009C46F98F9CC611E14840B727002083A7CD
:1005C000479B829719E5DC5085C3EF60215CEF50B3
:1005D000B15ADC5091CBB727002003A707D0B7064C
:1005E00033001C47D58F1CC7B240224492444101BE
:1005F0008280829794485840B387A6003E8563E482
:10060000D700E3E8E7F83385E74061B74111B72742
:10061000002006C623ACA79C0295B240B727002055
:1006200023A8A794014541018280994763E9B70057
:10063000B72700208A0593874796BE9588C1828098
:10064000B727002023AAA79C11C5B727002005477C
:100650002381E7988280B727002023A60798B72731
:10066000002023AC079CB727002023A2079837253A
:100670000020B72700204111238107987146B72732
:10068000002081451305459606C623AA079C22C46F
:1006900026C2372400209700FB1FE78080BF130588
:1006A00084931306800281459700FB1FE78060BE9C
:1006B000EFF08FADB72700209387079903C5C703D5
:1006C00083C7D7031304849385453E958D4733052F
:1006D000F5029947B724002039051375F50F23015A
:1006E000A4003305F502130505249700FB1FE780DE
:1006F000609523A8A49C49C10346240099478145DD
:100700003306F602130606249700FB1FE78060B845
:1007100083A7049D03472400B72400209387072460
:100720000A0723A0F496BA97372700202324F798C6
:10073000EFF06FD1A5218347140083A604963706F6
:100740000500139727003697130646CD10C313876D
:1007500017001377F70F0A073706050036971306B9
:1007600026C710C313873700890793F7F70F8A0747
:10077000A300E400B69790C3B240224492444101E2
:10078000828037270020130787938347170083460B
:10079000270063F0D702B726002083A606961386AB
:1007A0001700A300C70013972700369708C33E859C
:1007B00082809307F00FE5BF1C41638C07104177DF
:1007C0007D8FB706002089476316D7100357450071
:1007D00063020710411126C21946AA849305F00F3F
:1007E000610506C622C49700FB1FE78000B90547D4
:1007F0008D47630AE50C9C4491C7D858994761C757
:10080000985C71C33724002013060004814513054A
:1008100004999700FB1FE780C0A713060004A68574
:10082000130504999700FB1FE780809F93070499A5
:1008300003D7C70009E7130700102396E70003C793
:10084000E70001E705472387E70003D7070101E732
:100850006D472398E70003C7F70001E71547A38713
:10086000E70003C7270101E705472389E70003C71E
:10087000370109E703C7F700A389E70003C757015A
:1008800001CB937637000983238ED702A38EE7022C
:1008900003C7470101E75547238AE70003C76401FF
:1008A00009E71307C003238BE7009C5791C7829782
:1008B000B72700202390A794B72700207D57A38255
:1008C000E7D6513B8147B240224492443E854101E4
:1008D000828089473E85828001114AC837290020DD
:1008E0008327C99D06CE22CC26CA52C456C24EC604
:1008F0008297130A0064B33545031309C99D835ACF
:1009000089008146568633054503EFD05108B72745
:10091000002013878793004FAA8401456306940241
:100920009389879333858440636E9400032549003F
:1009300056868146B335AA023305AA02EFD03105A7
:10094000018D269523AC9900F2406244D24442497D
:10095000B249224A924A05618280011122CC2E843A
:10096000B7E506000A8541469385C55D06CEEFD002
:10097000913B180806043A94B7270020035504FF5A
:1009800083D7679EF2406244AA9737450F0013054C
:1009900005243355F50205618280B727002083D7EF
:1009A000679E51471D45637CF70279471945637877
:1009B000F7021307200315456373F7021307B0040A
:1009C0001145637EF700130740060D456379F70074
:1009D0001307600909456374F70013B5B70F8280E8
:1009E000011122CC06CE2A842EC6EFF0CFB6B24536
:1009F000F240818D33A5A502229562441375F50F4F
:100A000005618280011122CC06CE2A842EC6EFF029
:100A10008FB4B245F240818D33A5A5022295624480
:100A20004205418105618280011122CC06CE2A84D3
:100A30002EC6EFF04FB2B245F240818D33B5A5021C
:100A40002295624405618280B727002013870799A9
:100A500018572DC3411122C426C24AC006C61389A5
:100A600007990297B72700201387879303578700BA
:100A70002A84938487930DCBBA876373A700AA87D0
:100A8000C207C183BA866373E400A286C206C1822C
:100A9000958F5147635AF7008327C90291C3829704
:100AA000EF50F17723948400B240224492440249EB
:100AB0004101828082800111B727002022CC372497
:100AC000002023A8079E93070499DC5706CE26CA68
:100AD000AA851304049981C72AC68297B245C9C161
:100AE0009C410545ADCBDC41BDC783D78500A5C77B
:100AF00083D7A500ADC3B72400201385C49D5146FC
:100B00009384C49D97F0FA1FE780807123860400C8
:100B1000B727002083A6C79D372700202322D79818
:100B2000034774011DE39387C79D03D5870093078F
:100B3000805737460F003305F50213060624814619
:100B40008145EFD0C164A30BA40037150500130540
:100B5000858D6D3C0145F2406244D244056182803E
:100B6000B7270020938787933707002023AE07001D
:100B70001307676EB727002023AEE79C3787320044
:100B80009387C79DFD56130727A1D4C398C7238613
:100B90000700B7C7004023A4D7269DBF011122CC70
:100BA0003724002093070499884706CE26CA4AC8EE
:100BB00001E90545F2406244D24442490561828020
:100BC000130404995C58F5D7185C65D77000854507
:100BD00082971844B247E30EF7FC0355C40093050F
:100BE000E004B724002097F0FA1FE780A0451387A0
:100BF000849308D3938484934DDD0356C4009305F6
:100C0000F00F014997F0FA1FE780A0688347E400DE
:100C10009050634DF900328597F0FA1FE780C0507D
:100C2000014523A0040223A2040269B78355C4002E
:100C30000844185CB3872503898105093E9508C2DD
:100C40000297E9B701114EC6B72900209387099989
:100C50009C4726CA4AC852C406CE22CC56C25AC0A5
:100C60002A8AAE843289638D071E9389099903A766
:100C70004903630407121307F01F6362A7123724A6
:100C8000002013078493832A070213048493639A32
:100C90000A0803D5C9009565938515E097F0FA1FFA
:100CA000E780403A08D02A866DC983D5C90083A75A
:100CB000490303A589008981829783A78900832A34
:100CC00004025CD089476316FA08C1476397F40CA5
:100CD00083D5C9009147938505FCB3C5F5028A0504
:100CE000D69503C725009307A0056314F70A83D799
:100CF00005006390470B4A852686910597F0FA1FF9
:100D0000E78000521C505685639357130145F2400B
:100D10006244D2444249B249224A924A024B056196
:100D200082805850E380E7FA03D5C9009565938522
:100D300025E097F0FA1FE780E030AA8A39CD83D505
:100D4000C9002A8683A7490303A589008981829760
:100D500095BF8D47631BFA00C1476390F40483D5A8
:100D6000C900938545FDF199A5BF91476318FA0025
:100D70006395440383D5C900A115F5B79307001007
:100D8000631DFA00A14763EA970083D5C900C11526
:100D9000D9BF1C5056856390570D29458DBF9D6A5C
:100DA000637C5509930A05E01947B3CAEA0203D7E1
:100DB000C900372B0020B38AEA02BE9A93078B93AF
:100DC000DC53130B8B936395570103240B021DE037
:100DD00003D5C9009305E00497F0FA1FE780802649
:100DE0002A8445DD83D5C90083A749032A868981E2
:100DF0005685829791451307A00589819397250011
:100E0000A29783C627006393E60483D60700639CFA
:100E1000460385058A052686A2954A8597F0FA1F1E
:100E2000E780004083270B02E38287EE228597F05C
:100E3000FA1FE780602FD9BD21677917E36FA7F408
:100E4000B30A5541ADB783C5370045BF83270B02B1
:100E5000E38587F4228597F0FA1FE780E02C35BF01
:100E6000B727002083A587958DD991479306A005C4
:100E70008983139727002E9703462700E31FD6F098
:100E800003560700631C460185078A072686BE9520
:100E90004A8597F0FA1FE780A0388DBD8347370059
:100EA000C1BFB727002093870799984729C3985F48
:100EB0001DCF8546631DD502411122C43724002071
:100EC00013048493105006C619CE83D5C70048502A
:100ED00089810297085097F0FA1FE780E0242320C9
:100EE000040223220402B240224441018280828013
:100EF000011122CC372400209307049956C283AAFB
:100F0000870026CA4AC84EC606CE52C42A89AE8475
:100F1000B28913040499638C0A1C1C5C99EB294563
:100F2000F2406244D2444249B249224A924A05619F
:100F300082805C58EDD79307F01F63E8A70C372A2F
:100F4000002093078A939C53130A8A93B9C70844D5
:100F500083274A02639FA70489476317F906C1479D
:100F6000E39FF4FA0355C4009147130505FC33458C
:100F7000F5029317250003250A022686CE853E95A5
:100F80009307A0052301F50023102501110597F013
:100F9000FA1FE780E028014561B70355C4009305B7
:100FA000E00497F0FA1FE780E0092320AA0245F148
:100FB000BDB78355C4005C5803260A028981829715
:100FC0001C442322FA0249BF8D47631CF900C14724
:100FD000E397F4F40355C400130545FD9377C5FF6B
:100FE00059BF91476318F900E39B24F30355C400EC
:100FF0002115EDB793070010E313F9F2A147E3E0E1
:1010000097F20355C4004115D1BF9D676378F5067B
:10101000930705E01947B3C7E7020357C400372A0F
:101020000020B387E702BE9A93078A939C53130A62
:101030008A93A1CF83274A026395570703250A02A3
:1010400091461308A0059305F00F93D72600139738
:1010500027002A97034627006316060783580700D0
:1010600003463700639C2805B306D64063C6960442
:1010700085078A072686CE853E9511BF2167791799
:10108000E36FA7E8B307F54049BF0355C4009305D4
:10109000E00497F0FA1FE780E0FA2320AA0259F94A
:1010A000BDBD8355C4005C5803260A02898156855C
:1010B000829723225A0359B72310B70093160601CB
:1010C000C18261B70356C400B3859600910513062B
:1010D00006FCE3F6C5E413863400719A1106B29655
:1010E0002301070123102701A301D70051B7372A95
:1010F000002093078A939C53130A8A93A9C303255C
:101100000A0291461308A0059305F00F93D7260015
:10111000139727002A970346270063140605835870
:1011200007000346370063982801B306D640E3D191
:1011300096F42310B70093160601C182C1BF034580
:10114000E4008357C4009305E0043305F50242052B
:10115000418197F0FA1FE780E0EE2320AA0245F1D3
:101160007DBB0356C4008345E400B385C5023386C6
:1011700096001106E3E5C5DAB9BF0145828083C751
:1011800005002300F50083D72500A300F50083D7D1
:101190002500A1832301F50083C74500A301F500C5
:1011A00011458280B727002023A60780B72700209B
:1011B00023A40780828029C1411126C206C622C409
:1011C000AA8401458DC52E84B7E5060022854146D7
:1011D0009385C55E97F0FA1FE780800483C70400FB
:1011E00005452306F40083C71400A306F400B240AB
:1011F000224492444101828001458280011122CC27
:1012000026CA06CE0947AA8432846381E504414692
:101210008147639BC500638FE6006397B6000DA806
:1012200041478147638EE600F2406244D2443E85E6
:10123000056182808A852285BD3F41468A8519A83D
:101240008A85953F41468A85228531A0E39AB6FC7E
:101250002E86A285268597F0FA1FE780A009AA8727
:10126000E1B7B727002023A4A7808280B7270020FA
:1012700023A6A7808280011122CC0354650006CEEC
:1012800026CA4AC84EC641C083298500AE842A8832
:1012900003C9090081471317890161876355070254
:1012A000B147054563FA87045114420403552800E9
:1012B000418033878900A2864E868545EFA0900C39
:1012C000B337A00085077D141355690042040589D2
:1012D0001379F90341802380F400A380A4002381C3
:1012E000240123928400014719C01387190098C470
:1012F00009476383E7000145F2406244D244424912
:10130000B249056182800545C5BFC167F917630A07
:10131000F502D94763F7B702011122CC2EC606CEDB
:101320002A84EF703055B2456368B5002285624467
:10133000F24005616F90E078F24062440545056136
:10134000828005458280C167F9176314F5006F70CC
:101350007052411106C6EF90806511E15D45B240C3
:101360004101828091476394F50283470500230081
:10137000F6008347250003471500A207D98F2311E4
:10138000F6008347350001452302F60082801145AF
:1013900082804111814522C426C206C6AA84052541
:1013A0002A8409E9B727002083A7878081C7F945E8
:1013B000268582972285B240224492444101828050
:1013C00039714ED656D25AD006DE22DC26DA4AD8F9
:1013D00052D4AA8A2E8BB28941EF36C6AD379145D9
:1013E000EF70105BAA844D492DC9B246054A23808F
:1013F00034010544630A0B00B68513851400029B73
:101400000505131405014180E20993D9894163D38D
:101410000902C1455685EF90C067654905E93386E5
:101420008400A2852685EFA000472A8905E13104C2
:101430004204418091472C085685231CF10026CE9A
:10144000231D8100EF8010702A8901C963070A00FB
:10145000268597F0FA1FE78020CDF25062544A8526
:10146000D2544259B259225A925A025B2161828067
:10147000BA84014AADBF011122CC26CA4AC84EC661
:1014800006CE2A893284B689253FAA840DE1B72782
:10149000002083A7C78081CF05476317E40003C4FA
:1014A000090005041374F40FA2854A858297F2405F
:1014B000624426854249D244B24905618280AE86A3
:1014C000B7150500014705469385E5176DB783D726
:1014D00005002300F50083D70500A183A300F500D4
:1014E0000945828083D705002300F50083D70500D6
:1014F000A183A300F50083D725002301F50083D73E
:101500002500A183A301F5001145828083D7050042
:101510002300F50083D70500A183A300F50083D73E
:1015200025002301F50083D72500A183A301F50041
:1015300083C755002302F50083C76500A302F500A9
:1015400003D58500190542054181828083D70500B6
:101550002300F50083D70500A183A300F50009450A
:10156000828083D705002300F50083D70500A1837F
:10157000A300F50083D725002301F50083D72500BC
:10158000A183A301F5001145828003D5450006051E
:1015900042054181828083D705002300F50083D76F
:1015A0000500A183A300F50003D525000905420528
:1015B0004181828083D705002300F50083D7050091
:1015C000A183A300F50083D725002301F50083D76D
:1015D0002500A183A301F50003D5450011054205AF
:1015E0004181828083C705002300F5000545828084
:1015F00083D70500411122C406C62300F50083D716
:1016000005002E841105A183A30EF5FE83D72500C6
:101610009505230FF5FE83D7D5FFA183A30FF5FE14
:1016200003C6F5FF97F0FA1FE78080BF034544002B
:10163000B24022441105410182808947639CF50034
:1016400083471500034705000145A207D98F2310E2
:10165000F60082801145828003D70500D94763FEDA
:10166000E702011122CC06CE2EC62A84EF7090200C
:10167000B24683D70600636DF50022856244F240CE
:10168000B7150500014709469385E54C05610DBB7B
:10169000F240624409450561828009458280914794
:1016A0009DC583460500FD15C2058547C18163922E
:1016B000F60213D725008D89914791E9914701CB17
:1016C00005052301D6002310E60048C281473E8568
:1016D000828009479147E39CE6FEC94733D7F5026C
:1016E000B3F5F502D1BFAE86B71505000147114627
:1016F0009385454EF1B193F7350091EB8981914780
:1017000089C52310B60048C281473E858280914733
:10171000EDBF03C745008947631AF702011122CCC8
:101720002A84C84506CEAE86014719C52EC69D45FA
:10173000EFE0EFACB2462A8722856244F240B7154B
:10174000050019469385C55005619DB909458280FC
:1017500099E1114582808347050005472311F60072
:10176000E379F7FEFD1593F5F50F33D7F502B3874F
:10177000E702E390F5FE050548C22310E6000145A7
:10178000828083C745000947AE866385E7004147ED
:101790006399E700B7150500014721469385055F6A
:1017A00005B1094582802310B60091E1014548C288
:1017B00001458280AE86B71505000147294693850D
:1017C000C554FDBE2310B60091E1014548C2014554
:1017D0008280AE86B71505000147314693852556B0
:1017E000C5B62310B60091E1014548C2014582808B
:1017F00003D74500854763FDE702011122CC2A8407
:10180000884106CE0DC12EC68545EFE04F9F2A8741
:1018100022856244B246F240B715050039469385E9
:10182000A558056171BEF240624409450561828098
:101830000945828091479DC5034705008D46914724
:1018400063F2E602FD15C205C181B3C6E5023308A5
:10185000D7026399050105052310D6002311E60080
:1018600048C281473E85828083C745000947AE86CE
:101870006385E70041476399E700B7150500014715
:1018800041469385055F2DBE09458280B335B00082
:10189000139525008280011122CC26CA06CE03C7EB
:1018A00085008547AA842E8449466310F702613C6F
:1018B0008357240049151306200963C8A700F24086
:1018C0006244D244094505618280034794008547FC
:1018D0006314F70013660604484011C58D4532C6EF
:1018E000EFE0EF913246A2866244F2402A872685D5
:1018F000D244B7150500938565590561D1B48D476C
:1019000063FFB7028347150003470500F115A207DF
:10191000D98F2310F6008347350003472500C20501
:10192000A207C181D98F2311F6002312B60089C501
:10193000110508C60145828023240600E5BF114534
:101940008280011122CC2A84884506CEAE8611C53C
:101950002EC69545EFE0AF8AB2462A8722856244BB
:10196000F240B715050059469385455B056189BC72
:10197000B335B000139525008280AE86B7150500FB
:10198000014761469385455E25BC8547114563F453
:10199000D7028347160083450600A207CD8F231088
:1019A000F7009387E6FF2311F70089476386F60067
:1019B000090650C30145828023220700E5BF014785
:1019C000814679468145EDBA83D705002300F500AD
:1019D00083D70500A183A300F5000945828083C752
:1019E000250005472300F50003D505006397E700B0
:1019F0000A050505420541818280C9473305F50284
:101A0000CDBF03D505000A0542054181828083D7F9
:101A100025002300F50003D5050083D725003305F5
:101A2000F502050542054181828003D505008280CB
:101A300003D50500828003D50500828083D7250069
:101A40002300F50003D5050083D725003305F502F3
:101A5000050542054181828083D705002300F500FA
:101A600083D70500A183A300F50083D725002301B8
:101A7000F50083D72500A183A301F50003D5450018
:101A8000110542054181828083D705002300F500BE
:101A900083D70500A183A300F50003D52500090520
:101AA00042054181828089471145639BF600834747
:101AB0001600834606000145A207D58F2310F700C4
:101AC000828003D70500D947AE8663F9E700B725C2
:101AD000050001470D469385859C71BA09458280B2
:101AE00011456393A602834716008346060001450D
:101AF000A207D58F2310F7008347360083462600C0
:101B0000A207D58F2311F700828083C725000547E0
:101B1000FD1793F7F70F6361F70483D705008DCFA7
:101B2000011122CC2A84C84106CE15C12EC6894592
:101B3000EFD0FFEC2A8722856244B246F240B725F7
:101B4000050015469385E59D05616FF0DF92F24033
:101B500062440945056182800945828095471145A7
:101B600063F9D706411122C426C24AC006C683477C
:101B70001600BA8403470600A2073284D98F239047
:101B8000F400834736000347260093054400A2076C
:101B9000D98F2391F40089472382F40009461385E5
:101BA0005400368997E0FA1FE78080679307A9FF02
:101BB0002394F4009947631BF90023A60400B24064
:101BC0002244924402490145410182801904C0C463
:101BD000FDB7828083D705008DCF011122CC2A84E6
:101BE000C84106CE15C12EC68545EFD05FE12A87D4
:101BF00022856244B246F240B72505001D46938512
:101C000025A005616FF03F87F240624409450561F8
:101C100082800945828099476395F604894741117E
:101C200006C62302F7008347160083460600B285E6
:101C3000A207D58F2310F70083473600834626007E
:101C400003464700A207D58F130557002311F7005D
:101C5000910597E0FA1FE780A05CB2400145410181
:101C60008280D14711456394F600C1474DBF828001
:101C700083D705008DCF011122CC2A84C84106CE1E
:101C800015C12EC68945EFD09FD72A872285624489
:101C9000B246F240B725050025469385E5A00561CB
:101CA0006FF06FFDF240624409450561828009458D
:101CB000828089471145639BF6008347160083465F
:101CC00006000145A207D58F2310F700828001117D
:101CD00022CC2A84C84106CEAE86014719C52EC63D
:101CE0008545EFD0DFD1B2462A8722856244F24093
:101CF000B72505002D469385A5A205616FF0AFF7C6
:101D000011456393A60283471600834606000145EA
:101D1000A207D58F2310F70083473600834626009D
:101D2000A207D58F2311F7008280011122CC2A84CB
:101D3000C84106CEAE8611C52EC68545EFD03FCC34
:101D4000B2462A8722856244F240B725050035460F
:101D5000938505A305616FF00FF293F71600114507
:101D600089EB89476387F60085822312D70010C369
:101D700001458280011122CC2A84C84106CE15C1BA
:101D80002EC68545EFD0BFC72A8722856244B2465A
:101D9000F240B72505003D46938565A305616FF0C8
:101DA0008FEDF240624409450561828083D70500CA
:101DB0008DCF011122CC2A84C84106CE15C12EC672
:101DC0008945EFD0DFC32A8722856244B246F240BC
:101DD000B725050045469385C5A305616FF0AFE9BA
:101DE000F240624409450561828009458280854749
:101DF00063FCD7022304A700A304B700834716009F
:101E000083450600A207CD8F2310F7009387E6FFD6
:101E10002311F70089476386F600090650C3014580
:101E2000828023220700E5BF114582800147814659
:101E30004D4681456FF02FE48D47114563FBD70276
:101E40008347160083450600A207CD8F2310F700B5
:101E50008347360083452600A207CD8F2311F70064
:101E60009387C6FF2312F7006386A600110610C7EA
:101E70000145828023240700E5BF011122CC2A847A
:101E8000884506CEAE8611C52EC69545EFD03FB724
:101E9000B2462A8722856244F240B72505005D4696
:101EA000938585A505616FF00FDD85471145639723
:101EB000F6008347060001452300F70082800147B2
:101EC0008146654681456FF00FDB011122CC2A84E3
:101ED000C84106CEAE86014719C52EC68D45EFD046
:101EE0001FB2B2462A8722856244F240B725050018
:101EF0006D46938585A805616FF08FCC011122CCCA
:101F00002A84C84106CEAE86014719C52EC68D4526
:101F1000EFD0FFAEB2462A8722856244F240B72551
:101F200005007546938585A805616FF06FC901119D
:101F300006CE2EC6EF80D02301C9B245F24003552C
:101F4000250005616FC0102EF24049450561828071
:101F5000B7270020A38C0782B7270020238C078295
:101F6000B727002023A00782B727002023A20782DB
:101F7000B727002023A40782B727002023A60782C3
:101F8000B727002023AE0780B727002023AC0780A7
:101F9000B7270020239A07A013064038938747A14C
:101FA0002391C70271761307400B130606B82391DD
:101FB000E7002392C70211671D46930600059305AB
:101FC000000A1305007D2392E7002393C7024147CF
:101FD0000546130810F82395E7002396E700239998
:101FE000E700239AE700239BE700239CE700239464
:101FF000E7022393B7002394B7002397D7002398D1
:10200000D700239DA700239E0700239F070023904E
:1020100007022395C7022396070323970702930815
:10202000F007239807022392E7042393E704239FF2
:10203000E7042390E7062391E7062392E706239916
:1020400017031307C01C239AC702239BC702239CB4
:102050000702239D0702239E0702239F0702239066
:1020600007042391C70423940704239507042396A8
:10207000C7042397D7042398D7042399A704239A46
:102080000704239B0704239C0704239DD704239E56
:10209000D7042393A70623940706239507062396C0
:1020A00007062397B7062398B70623990706239AAE
:1020B000E7067D57239B0706239007092391E7082E
:1020C0008280011126CAAA84214522CC06CE2E8404
:1020D00032C636C43AC2EFD0FF9E1DC9A24612478F
:1020E0003246930700FD2300F5009947A3009500B1
:1020F0002301F5002303D500A303E5002312C50047
:10210000AA8522856244F240D24405616FD09FAA1D
:10211000F2406244D24405618280B727002023A4A4
:10212000A7828280B727002023A6A7828280011180
:1021300022CC4AC806CE26CA2A890144B3048900A3
:102140006368B400F2406244D2444249056182802F
:102150002EC6EFD05FC093170501C183A183B2459E
:102160002380F4009307140093F7F70F850463F9B5
:10217000B700CA9709042380A7001374F40F7DBF2A
:102180003E847DBF411122C4372400201304449FA4
:1021900003556400C16706C6FD17630FF500B72736
:1021A000002003C687B3B725002093850583EF8001
:1021B000E05AFD572313F400B240224441018280CB
:1021C00009C925151375F50F1335850E134515002F
:1021D00082800145828023900500C9C6797122D48E
:1021E00026D24ECE52CC5AC806D64AD056CA5EC661
:1021F0003684328AAE892A8B814463F34407B3075D
:10220000940083C70700138914004209939A0701B9
:1022100093DA0A011359090163840A04CA976341D6
:10222000FA04B307240183CB07005E85513F0DC933
:102230009387FAFF2390F90063906B03130519004D
:102240002295B250225492540259F249624AD24A1B
:10225000424BB24B45618280D694C204C18071BFAB
:102260000145C5B701458280011122CC37240020E9
:1022700026CA4AC84EC69307449F06CE2E89D0CBA5
:102280008CCBC8C7AA8441469305F00F4A8597E0D6
:10229000FA1FE780800E85491304449F63193503B4
:1022A0000848C145693541469305F00F268597E0FA
:1022B000FA1FE780800C05496315250348446244F2
:1022C000F240D2444249B249C14505618DB541460B
:1022D00081454A8597E0FA1FE780200AE31535FD1E
:1022E000C1B741468145268597E0FA1FE780E0089F
:1022F000E30625FDF2406244D2444249B2490561F9
:102300008280411122C43724002026C24AC0AE84F4
:102310002A891306000281451305449F06C697E0EB
:10232000FA1FE78000F79307449FA3812701B7278F
:102330000020238E97B2EFC02071854719C18147D5
:102340004945230AF49EB240224492440249410185
:102350008280814781CD19C98547631BF50083C7FA
:10236000550093E707FCA382F50085473E858280F0
:1023700089476317F50083C7550093F7F703E5B75F
:102380000D478547E314E5FE03C755001377F703B0
:1023900013670704A382E500D1BF81478DC105C142
:1023A00003C755009306000C85471377070C630895
:1023B000D700930600048D476303D70089473E8505
:1023C0008280411122C4005D06C626C21DC8AA84AF
:1023D000085009C597E0FA1FE78000D5485009C5A5
:1023E00097E0FA1FE78040D4085409C597E0FA1F28
:1023F000E78080D3228597E0FA1FE780E0D223AC04
:102400000402B240224492444101828019E9B72774
:10241000002083C7679F91C73725002013050581DA
:102420008280372500201305C5A08280B7270020B1
:1024300003C5679F8280B727002003A507A082807D
:10244000B727002003A547A08280B727002083A7D5
:1024500087A088438280B72700209387479FD44B6B
:102460009842050798C203C537009307F00F63052C
:10247000F50091656FD0BFAE8280011122CC06CEEF
:102480002E8432C6EF80605F9147B2456310F5023B
:10249000B727002083A7C78295C303A30700630F54
:1024A000030022856244F24005610283B7270020C1
:1024B00083A7478281C703A34700D5B7F240624490
:1024C000054505618280011122CC2A84035545000F
:1024D00006CE26CA4AC84EC6EF8040383DC92A8972
:1024E000834405008349C500E93D4A85EF80101803
:1024F00003554400EF80A053372900201309898336
:1025000083470900B9CB639A9704B727002083C596
:1025100097832685293C19E12300090003554400CF
:10252000EF80A0559147631FF500B72700209387E0
:10253000479F8356440003D767006395E6007D57A5
:102540002393E700F2406244D2444249B249056114
:10255000828081499304F00F45B79307F00FE38F12
:10256000F4FA8346640003564400034524004E8772
:10257000A685813E65B779715EC6AA8B2E8552CC41
:1025800056CA5AC806D622D426D24AD04ECEAE8AD1
:10259000328B368AEF80802C7DC1045D2A89E5C0AC
:1025A0009C50614599C3130540039C5481C7510554
:1025B0004205418163050A00710542054181DC50F5
:1025C00081C75D0542054181EFD0CFCF2A8445C93F
:1025D0006146814597E0FA1FE780A0CBB72700202E
:1025E00083C947A46394090083490900930700FD48
:1025F0002300F400A947A30074012301F40023037E
:1026000064018C50231254011305840191C908C43C
:102610007146930A440397E0FA1FE78060C056852D
:102620008C5491C948C45146930A450197E0FA1F5A
:10263000E78000BF5685630C0A0008C87146D28542
:10264000930AC50197E0FA1FE78080BD5685CC50FC
:1026500099C548C85D4697E0FA1FE78060BCA2852F
:102660004E85EFD02FD52254B2509254F249624A8F
:10267000D24A424BB24B4A850259456199B3B25096
:10268000225492540259F249624AD24A424BB24B06
:102690004561828001114EC6AA892E854AC806CEA0
:1026A00022CC26CA2E89EF80601B21C9B7270020C3
:1026B00083C447A499E0834405001945EFD08FC037
:1026C0002A8405CD8145194697E0FA1FE78060BC52
:1026D000930700FD2300F400B947A3003401230150
:1026E000F40023122401A2856244F2404249B24917
:1026F0002685D24405616FD0EFCBF2406244D244CC
:102700004249B2490561828039715ECEAA8B2E851D
:1027100026DA4ED652D456D25AD006DE22DC4AD819
:10272000AE84328BB68A3A8ABE8942C6EF800013E5
:1027300021CD2A894145EFD0EFB82A8431C54146E1
:10274000814597E0FA1FE780C0B4B727002003C592
:1027500047A419E103450900930700FD2300F40095
:10276000BD472301F400B247A30074012312940073
:1027700023046401A304540123054401A305340187
:102780005CC4A285EFD00FC3F2506254D2544259B8
:10279000B259225A925A025BF24B216182807971BE
:1027A00026D2AA8439454AD04ECE06D622D42EC689
:1027B000B2893689EFD00FB121C1B2459307000D20
:1027C0002310F500B1472A842312B5002301F50038
:1027D000CE851905194697E0FA1FE78060A4230605
:1027E0002401A2852254B2500259F24913F5F40F84
:1027F000925445616FD00FBCB2502254925402598A
:10280000F24945618280411126C2B7240020938499
:10281000449F03C7340006C622C44AC09307F00F82
:10282000630CF7042A893945EFD0CFA92A8429C53A
:10283000930700FDB72500202300F500A300250124
:10284000230105009385C5A00D05194697E0FA1FE1
:10285000E780009D83D78400A28503C5340023153B
:10286000F40083C714002306F4002244B2409244CB
:10287000024941016FD00FB4B24022449244024950
:102880004101828001115AC02A8B314526CA4EC6A9
:1028900052C456C206CE22CC4AC8AE84B28A368A08
:1028A000BA89EFD02FA23DCD2A842685EF70107B08
:1028B00011C50347C500A1476314F704B7270020DB
:1028C00003C9779F930700FD2300F4009D47A300F1
:1028D00064012301F40023129400231354012314F0
:1028E000440123153401A2856244F240D244B24926
:1028F000224A924A024B4A85424905616FD08FAB0A
:10290000B727002003C9D7B3E31E0BFAB72700206F
:1029100083A7878D9C47DDD7CE865286D6852685B0
:1029200082974DB7F2406244D2444249B249224AAA
:10293000924A024B05618280011122CC2A842145F2
:1029400006CE2EC6EFD00F9821C1B245930700FDE9
:102950002300F500C5472301F50083C73500A30117
:10296000F50083D745002312F50083C765002303D4
:10297000F50083C77500AA85A303F500228562448C
:10298000F24005616FD00FA3F2406244056182807E
:10299000397162CC2A8C594526DA4AD84ED652D49F
:1029A00056D25AD05ECE06DE22DCAE8432C636C4A3
:1029B000BA8B3E8BC28A468A83590104034941047B
:1029C000EFD04F9025C93246930700FDA246230061
:1029D000F5009547A301C500A30085012301F5007B
:1029E0002A8419461105A9C2B68597E0FA1FE78027
:1029F000208323066401230A24012315740123176D
:102A000054012318440123193401A2856254F25061
:102A10004259B259225A925A025BF24B624C2685B5
:102A2000D25421616FD00F99814597E0FA1FE7805A
:102A30004086C1B7F2506254D2544259B259225A18
:102A4000925A025BF24B624C21618280411122C496
:102A5000372400201304449F8347240006C626C25F
:102A60008DCBB7240020AA8519461385048197D001
:102A7000FA1FE780E07A0345240093850481EFF094
:102A80005F8D2244B24013850481924441016FB0AE
:102A9000707CB24022449244014541018280411140
:102AA00026C2B72400209387449F06C622C44AC08A
:102AB00003C737009307F00F9384449F6304F70420
:102AC0002A892945EFD00F802A840DCD930700FD78
:102AD0002300F500A147A30025012301F50083C7CA
:102AE0002400B725002093850581A301F500194630
:102AF000110597D0FA1FE780A07203C53400A285A4
:102B0000EFD04F8B03C724008D476311F702B7271F
:102B1000002083A7878299CB03A387006308030063
:102B20002244B2409244024941010283B24022440D
:102B30009244024941018280797122D406D626D27C
:102B40004AD04ECE52CC56CA09445DCD2A8903558F
:102B50000500AE895144EF707050AA8455C53727DF
:102B60000020930787B383C747008546BA8AFD17BD
:102B700093F7F70F494463F9F6080347C500A147E7
:102B80006314F700639209089C5C4544B5EF9165B6
:102B9000938545711305C00297D0FA1FE780804ADC
:102BA00088DC2A8A4D442DC11306C002814597D086
:102BB000FA1FE780006E8357090093064A003685A6
:102BC0002311FA0071469305490036C697D0FA1FC3
:102BD000E780006589472300FA0003C5C400B246B8
:102BE0000356090083C58AB3611513351500EF80BC
:102BF000506D2A8463860900CE852685EF80A05615
:102C000001C42685EFF0EFFB2285B2502254925486
:102C10000259F249624AD24A45618280B7270020B0
:102C200083C7C7B30547FD1793F7F70F6378F70816
:102C3000894751C6011122CC26CA4AC84EC652C481
:102C400006CEAA89368AB2842E89EF7030412A8452
:102C5000D14729C9485509C597D0FA1FE780C04C0C
:102C6000F1452685EFD00F9648D4CD4705CD834654
:102C7000C40021478147639FE600630D0A000347B4
:102C8000A5010356050193062501AA854E85EF800F
:102C90002055AA8703474400630F090013676700A4
:102CA0002302E400F2406244D2444249B249224A3B
:102CB0003E850561828013674700DDB7C9473E85C1
:102CC00082809307000463EBA700B7270020938757
:102CD00047A106053E9503550500828041657D1597
:102CE0008280011122CC2A842E8526CA06CEAE848B
:102CF000EF70D0361DCDB7470F009387F7230945F6
:102D000063E4870281450A85414697D0FA1FE78030
:102D10004058A685231081000A8541802301810047
:102D2000A3010100EF809045F2406244D244056166
:102D300082804945D5BFB7270020238DA7B2828066
:102D40006F805052797152CC2A8A328522D426D291
:102D50004AD04ECE56CA5AC85EC606D662C4AE8B9C
:102D6000B28A368BBA843E89C2894684EF70102FAE
:102D700015C92A8C63140A0213774B008347450058
:102D800015CF93E727012302FC008DEC631C090299
:102D9000639A090205E8ED9B2302FC00832B8C0358
:102DA000639F0B06B250225492540259F249624A70
:102DB000D24A424BB24B224C45618280F59B93E74D
:102DC0000701D1B793E747002302FC0001CC1C4860
:102DD0004146A2852324FC0213058C0197D0FA1FDB
:102DE000E780004463910B02D5D80325CC0209C5C6
:102DF00097D0FA1FE7804033F1452685EFC09FFC4E
:102E00002326AC0261BFE30B09F80325CC0209C5F8
:102E100097D0FA1FE7804031F1454A85C5B79DC478
:102E200083A70B0299EB916593853571714597D016
:102E3000FA1FE780202123A0AB0203A50B0219C5CE
:102E40007146A68597D0FA1FE780803D6388090206
:102E500083A74B0299EB9165938525715D4597D0CA
:102E6000FA1FE780201E23A2AB0203A54B0219C55F
:102E70005D46CE8597D0FA1FE780803A1DC483A7B0
:102E80008B0299EB916593851571514597D0FA1F87
:102E9000E780401B23A4AB0203A58B0219C5514652
:102EA000A28597D0FA1FE780A0372254B2509254DF
:102EB000F249B24B224CCA865A860259424BD685F9
:102EC0005285D24A624A45616FF0EFEA011126CA83
:102ED00052C406CE22CC4AC84EC62A8AAE84EF70AF
:102EE000F01725C5AA893945EFC0DFBD2A8431CD49
:102EF000B727002003C947A46314090003C90900C8
:102F00009307000D2310F400AD472301F4009385CF
:102F1000690013053400194697D0FA1FE780403046
:102F200093F71400858085882306F400A306940097
:102F300023154401A2856244F240D244B249224A98
:102F40004A85424905616FC0FFC6F2406244D244DF
:102F50004249B249224A0561828001114EC652C4DB
:102F600056C206CE22CC26CA4AC8AA8A2E8AB2895E
:102F7000EF70D00E2DCD2A891305C002EFC09FB48B
:102F80002A8435C5B727002083C447A499E0834429
:102F900009009307000D2310F400E9472301F40012
:102FA0009305690013053400194697D0FA1FE7808E
:102FB0002027D285231554011305C400414697D01C
:102FC000FA1FE780E025CE851305C401414697D05E
:102FD000FA1FE780E024A2856244F2404249B249E8
:102FE000224A924A2685D24405616FC0BFBCF24096
:102FF0006244D2444249B249224A924A05618280DF
:10300000411122C43724002013048481084006C6DD
:1030100019C597D0FA1FE780201123200400B24081
:10302000224441018280011106CE22CC26CA4AC820
:103030002EC6EF70B00239CDB245B727002003C9C4
:1030400047A40CD5AA84631409000349050041452F
:10305000EFC05FA72A841DCD9307000D2310F50054
:10306000A5472301F50083C754009385640011052B
:10307000A30FF5FE194697D0FA1FE780601A9C54FB
:10308000A285F2405CC46244D2444A85424905614B
:103090006FC05FB2F2406244D2444249056182800F
:1030A0001D71A2CC86CE2A842EC6EF70207B05CD62
:1030B0008346C5001147AA8749456392E6029C5F93
:1030C000B24599C383C56701B7D605002308B1008F
:1030D0009386A6A7100889452285EF70907FF64059
:1030E0006644256182805145DDBFB727002083C734
:1030F000C7B30547FD1793F7F70F637AF7048947BE
:1031000021CA411122C426C24AC006C6B2842E89F1
:10311000EF70C0742A84D14705C56308090083474E
:10312000450093E727002302F5004146A6851305D5
:10313000840197D0FA1FE780A00E9C481CD48147D9
:10314000B2402244924402493E8541018280C947EF
:103150003E858280797122D406D62A842EC6EF70ED
:10316000E06F01CDB2452285230EB1006C08EF70EF
:10317000107CB2502254456182805145DDBF6F7092
:103180009004C1671387E7FF6395E502B727002026
:1031900083A7478291EB494582804945B24022444A
:1031A000924402494101828003A30700E30503FE24
:1031B0000283411122C426C24AC006C6FD172A89CD
:1031C0002E84B284639AF502B727002083A7478232
:1031D00091CF9C4381CF829711E9B7270020238CA0
:1031E0002783B7270020A38C97824DBFA6854A85E9
:1031F000EFE0FFD345F5D5B72E85EF70206651DDA2
:10320000834705000D45E39B27F922852244B24000
:103210000249A685924441016FB0D0009307000493
:1032200063E2A7064111C16722C406C626C2FD1784
:103230002A8409456382F502C547AE846313F4020C
:103240002E85EFB0B00537250020130545A10604F3
:103250002A94231094000145B24022449244410133
:1032600082809307A0036316F4002E85EFB0407CA4
:10327000D9BF9307B003E318F4FC13F5F50FEFB0D3
:10328000607BD1B709458280011106CE2AC6EFE0E6
:103290003FCCEF10C01CEFA0910EB7270020938702
:1032A000479F130700F02391E70023820700B72709
:1032B00000203245138787B3FD562301D700F24023
:1032C000238CA7B2954505616F50F06659719397AD
:1032D0000501A6D286D6A2D4CAD0CECED2CCD6CA2A
:1032E000DAC8DEC6E2C4E6C2EAC06EDEC187AE84DA
:1032F00063D3075237240020034584B337290020C5
:10330000372A0020EFC01F83AA8C22CCB72A0020C6
:10331000B72B00201304499F372C002063930C0225
:103320002165258DB650265496540659F649664AAD
:10333000D64A464BB64B264C964C064DF25D65611F
:10334000828083C70C001307200A639CE70083492F
:10335000340003D52C00C1656686FD15EFF0EF91B2
:103360009DA26247130787B38349270013071009FB
:103370006398E71683C71C001547639FE7006685BF
:10338000EFF06F946685EFC0CFEEE24703C587B3D9
:10339000EFC04FFAAA8C59B73947639BE71603D59C
:1033A0004C008567A5076316F50483A58C0003CB45
:1033B0000500631D0B00850591C9372500201946BE
:1033C0001305C5A097D0FA1FE78080E50347499F02
:1033D00085476317F71063080B00230A099E5A8577
:1033E000EFF06FC245B78947230AF99EEFB04066F8
:1033F00051BF896713872700631CE50403AB8C006A
:1034000063000B0E83470B0089EF83472B000347B4
:103410001B00A207D98F2314F40083473B00A300AD
:10342000F4000347499F8947631CF70A83470B0051
:1034300091C7230A099E03450B005DB7834514001D
:10344000035584008D47230AF99EEF50D051E5B70C
:1034500095076319F50083A78C0003C50700EFF0FB
:103460000FE40DB7F9771387A7FF2A974207418327
:10347000914663F1E6049387A7FCAA97C207C1832C
:1034800071476371F70289671387B7006310E5041A
:1034900083A70A82E38807EE9C43E685E38407EE70
:1034A000829715A0370700181307F770B357F70076
:1034B000858BA9CB83278A82E38607EC9C43E38331
:1034C00007EC66858297E31F05EA19A81387C700F2
:1034D0006311E50283A78C0083C70700E38407EA32
:1034E0009307F00FE380F9EAE6854E85EFC08FEC95
:1034F00069BDB9076318F50083274C82E38407E8A8
:10350000DC4361BF896793871704E303F5F8C9BFFC
:103510003D476399E70403D54C0089671387D700BB
:10352000E30CE5FC13879701E308E5FCCD07E319FD
:10353000F5FA03576400C167FD17631DF700832781
:103540004C82E38107E4DC43E38E07E20965E6850C
:103550004D05B9B7B727002083A7C782E38407E2E8
:103560009C43DDB71307E003E39CE7F683C72C0019
:1035700005476398E70E83C76C0037270020930D3B
:103580008781E1E783A70D00D5CF03CB0700A149D1
:1035900003C57C00138D8C00EA85EFE01FE083C734
:1035A0004C01A383AC0083D80C0103D8EC0003D7F3
:1035B0004C002A8603C53C003EC283D72C01EA8614
:1035C000DA853EC0CE87EFF0AFBC83C73C0095E7FD
:1035D000DD4783D80C0103D8EC0083C67C0083D57B
:1035E0004C003EC283D72C016A873EC0CE87054679
:1035F0005A85EF70805FA381AC0083A70D0081C75F
:103600001145EFF0FF9F138B8B8303450B00E30BFA
:1036100005D6B727002083C59783EFE05F91E303CA
:1036200005D683C63C0093071003638AF60003D6D1
:103630004C0083450B004E873685EFE09FA8238C16
:103640000B8289B3034B340099B783278A82034BDB
:103650003400914995DFDC4385DF81450145829740
:1036600005BF29476398E70A83C76C003727002006
:10367000930D8781A5EF83A70D00B5C703CB070086
:10368000A14903C57C0093868C0093772500BDCBB0
:1036900013761500138E4C0183C70C0283D8CC011E
:1036A00003D8AC0103D74C0003C53C003EC283D70E
:1036B000EC01DA8572CE3EC0CE87EFF06FAD83C7E6
:1036C0003C00724E9DFBDD4783D8CC0103D8AC0192
:1036D00083C67C0083D54C003EC283D7EC01728741
:1036E0003EC0CE8729B7034B340059BF83278A8257
:1036F000034B34009149D1D7DC43C1D78145014503
:10370000829741B7B68536CEEFE03FC9F2462A86AA
:10371000368E59B70947639CE70083A70A82E38383
:1037200007C6DC43E38007C666858297A1B92D47AB
:103730006398E70083A70A82E38607C49C47DDB746
:103740000D476397E70066868D4503D54C0039B178
:1037500019476395E7069305610213051031EFA041
:10376000A14A2C1013052031EFA0014A03D66C00AA
:103770008357810203D54C0063E8C70083D68C00D1
:103780000357610263F7E60093050002EFB00030D3
:10379000D5BE6374E6002393EC0063F4D700239452
:1037A000FC0003D7CC0083D6AC0003D68C0083D5B5
:1037B0006C0001488147EFB0202DE9B61D47E38139
:1037C000E7D231476395E7006686B145BDBF35470F
:1037D0006398E70083A70A82E38607BADC4799B7B4
:1037E0004947639DE70083278A82E38B07CEDC434A
:1037F000E38807CE814505458297DDB14D47E391CA
:10380000E7CE83278A82E38D07CCDC43E38A07CCAB
:10381000E6850945D5B793F7150089CFB72700206E
:1038200083A7078289C7DC4399C30145829713C5E3
:103830001400CDBC93F7250091CFB727002083A7B4
:10384000878291C7DC4381C781450545829713C5AF
:103850002400C9BC93F745000145E38507ACB727B1
:10386000002083A7C781372400201304449F91CFF1
:1038700085472302F400B727002083A7878291C7DA
:10388000DC4381C781450545829748442C10EF7081
:10389000507B2810EFF08F9BB727002083D767A3BA
:1038A00081CF130600643386C702B727002003C503
:1038B00087B39145EFC09F8913C54400A5B441115A
:1038C00022C4372400200325C48106C619C597D019
:1038D000FA1FE7806085232E0480B2402244410114
:1038E00082805971A2D4372400208327C48186D6D0
:1038F000A6D2CAD0CECED2CCD6CADAC80545638D00
:10390000070C9305F1041305F041EF807113930543
:10391000F1041305F041EF80B112B727002093871F
:10392000479F83C727000347F104B337F00011C353
:1039300089070327C4813EDE03453700930547000E
:10394000EFE03FA10327C4812ADC0D458345270012
:103950002EDAEFF00FB72AD81145EFF08FB6032417
:10396000C4812AD665450347A400034BB4003AD46A
:10397000EFF02FB5AA846945EFF0AFB42A897145FD
:10398000EFF02FB4AA896D45EFF0AFB32A8A7545E1
:10399000EFF02FB3AA8A7945EFF0AFB2E204625894
:1039A000F2572257B2564256D2551375F50F93FA75
:1039B000FA0F137AFA0F93F9F90F1379F90FE184DB
:1039C0002ACC56CA52C84EC64AC426C25AC0930808
:1039D00044000545EFB0400DB650265496540659A4
:1039E000F649664AD64A464B65618280011122CC6F
:1039F00006CE26CA8D472E846315F50603C735000B
:103A0000B7240020E94703D545009384449F6316FB
:103A1000F70083D764006382A706EF60306409C5AE
:103A2000835764002317F5000357A40083568400CE
:103A3000035664008355440003453400EFE09FE4DF
:103A40000357440083D764006309F7008547F240B9
:103A50006244D2443E8505618280FD572393F40081
:103A6000F5B78967CD07631DF50083C7250031478A
:103A70006385E7004547E39BE7FCEFE0AFF0F9B76C
:103A8000B1476319F500B727002003C5D7B3EFE0AE
:103A9000BFEA6DBF41677D178147E31AE5FA83C628
:103AA00055004947E395E6FA83C5450003552400D0
:103AB000300023140100EF60B04649BF411122C419
:103AC000372400208347A48326C206C64AC01307B2
:103AD000E00FAE846386E7041307F00F1304A4839A
:103AE0006387E7021145EFB0FFFD15C1930700FDA5
:103AF0002300F50089472301F5008547A3009500C1
:103B0000A301F500AA8503450400EFC0AF8AF95769
:103B10002300F400B24022449244024941018280D1
:103B20002A891145EFB01FFA75D5930700FD2300D0
:103B3000F50089472301F500A3009500A3012501A5
:103B40002244B7270020B24092440249AA8503C507
:103B5000B78341016FC00F8679714AD037290020A1
:103B60008327C98122D406D626D24ECE52CC56CA3D
:103B70004544D5EFB7240020938784B383C747001B
:103B80004944958BCDC7B72700202E8A9165A38D18
:103B9000A782AA8993857571314597C0FA1FE7807E
:103BA000604A232EA9804D4459C123003501A3004A
:103BB00005002946D285090597C0FA1FE7804066AF
:103BC0008327C981914603C7270063EDE60835EBDB
:103BD0004D472381E70003C72700136707012381AF
:103BE000E700930571001305F041EF80616583479D
:103BF0007100F1EBB727002003C7679F8D4763145F
:103C0000F70CEFE05F832C00EF70B0432800EFE08B
:103C1000FFE34545EFF0EF8A014411C91306006444
:103C20003306C50203C584B39145EFC02FD2228568
:103C3000B250225492540259F249624AD24A456122
:103C4000828085466314D700754761B7894663143F
:103C5000D7004947BDBF8D466314D700414795BF84
:103C6000554785BF9546CA8A630ED70099466316A5
:103C7000D70009472381E70031A01D466314C7021E
:103C8000238107006545EFF0CF839307F007E30A30
:103C9000F5F403A7CA818347270093E707042301AC
:103CA000F70081B721466314C7000547E1B72546F1
:103CB0006315C7002381D700F1B7A9460544E3186F
:103CC000D7F6114745BF31392A8435D1CD3E85B766
:103CD000011126CAB724002083A7C48122CC06CEB6
:103CE0004AC84944B1C783C707000D446392A7047B
:103CF00037290020034589B38945EFC0EFED03451F
:103D000089B3B72700209145239E0782EFC0CFECEF
:103D100083A7C48101478146A38087001306F10071
:103D2000854785450145A307F100EFA0505B2A8434
:103D30002285F2406244D2444249056182800111E9
:103D400006CE22CC26CA4AC88547631EF50637240C
:103D500000201304C48383570400A9CB3727002015
:103D60000347879F21E71307B003636CF702B7246B
:103D7000002003C584B38945EFC00FE60356040055
:103D80009307006403C584B33306F6028945EFC088
:103D9000EFBB23100400F2406244D2444249056163
:103DA0008280938747FC2310F400F5B7B7270020E3
:103DB00083A7C781EDD36244F240D244424903C590
:103DC0000700056131B7B724002083A7C481E1D77C
:103DD00037270020130987B383474900918BC5DF3C
:103DE00089476313F5062D452EC6EFB0BFCD2A8453
:103DF0005DD1B245930700FD2300F500E547A30020
:103E000005002301F50083C7350015051946230F6A
:103E1000F5FE83C745009505A30FF5FE97C0FA1F71
:103E2000E7800040034559009307F00F6316F50043
:103E300083A7C48103C50700A2856244F240D2442F
:103E4000424905616FB01FD7034587B38945EFC06D
:103E5000AFD86244F240D2444249B7270020239EA3
:103E6000078205616FF0BFA549458280B727002012
:103E700083C7C7B3958B638F07129307C01C63FC7E
:103E8000C70009458280F2406244D2444249B249A7
:103E9000094505618280B727002083A7C781638B0E
:103EA0000710B72700209387A78303C807001307CD
:103EB000E00F6311E810011122CC4AC806CE26CAD1
:103EC0004EC62380A700130586004205368932843A
:103ED0004181ADC991659385657197C0FA1FE780EF
:103EE0006016AA894DD1B724002003A54484938489
:103EF000448409C597C0FA1FE78000231385890011
:103F000023A0A9002286814523A0340197C0FA1F6F
:103F1000E78020389C402286CA85884397C0FA1FD4
:103F2000E78000309C40A286F240239287006244E2
:103F3000D2444249B249984305468D45054505613D
:103F40006FA0703991659385557197C0FA1FE7800E
:103F5000600FAA890DD9B724002003A5C4849384D7
:103F6000C48409C597C0FA1FE780001C1385890027
:103F700023A0A9002286814523A0340197C0FA1FFF
:103F8000E78020319C402286CA85884397C0FA1F6B
:103F9000E78000299C40A286F24023928700624479
:103FA000D2444249B249984305468D4505450561CD
:103FB0006FA0B032494582809307C01C63FCA70004
:103FC000094582800945F2406244D2444249B249DF
:103FD0000561828045CD011122CC2A8421054EC67F
:103FE0004205AE8991659385657141814AC806CEC7
:103FF00026CA97C0FA1FE780E0042A8961D5B72452
:10400000002003A544849384448409C597C0FA1F03
:10401000E7808011130589002320A90022868145AD
:1040200023A0240197C0FA1FE780A0269C40228687
:10403000CE85884397C0FA1FE780801E9C4023925C
:104040008700B727002083A7C7818DCFB72700201F
:1040500083C7C7B3958B8DCBB727002083A7478431
:1040600099CF984383D647006244F240D2444249F4
:10407000B24905468D45054505616FA0D02501472C
:104080008146DDB7014581B7494535BFB7270020D7
:1040900083A7C78195C7B727002083C7C7B3958B70
:1040A00095C3B727002083A7478481CB984383D645
:1040B000470005468D450545C9B701478146D5BF2F
:1040C00001458280494582809307C01C63FCA7009C
:1040D000094582800945F2406244D2444249B249CE
:1040E0000561828045CD011122CC2A8421054EC66E
:1040F0004205AE8991659385557141814AC806CEC6
:1041000026CA97C0FA1FE780E0F32A8961D5B72451
:10411000002003A5C4849384C48409C597C0FA1FF2
:10412000E7808000130589002320A90022868145AD
:1041300023A0240197C0FA1FE780A0159C40228687
:10414000CE85884397C0FA1FE780800D9C4023925C
:104150008700B727002083A7C7818DCFB72700200E
:1041600083C7C7B3958B8DCBB727002083A7C784A0
:1041700099CF984383D647006244F240D2444249E3
:10418000B24905468D45054505616FA010150147EB
:104190008146DDB7014581B7494535BFB7270020C6
:1041A00083A7C78195C7B727002083C7C7B3958B5F
:1041B00095C3B727002083A7C78481CB984383D6B4
:1041C000470005468D450545C9B701478146D5BF1E
:1041D00001458280494582809307C01C63F4A70093
:1041E00009458280797122D44ECE06D626D24AD095
:1041F000AE892A842DC1210591654205938575718B
:10420000418197C0FA1FE780E0E32A8909456306E8
:104210000908B724002003A584849384848409C5F5
:1042200097C0FA1FE78040F0130589002320A900FA
:104230002286814523A0240197C0FA1FE7806005EC
:104240009C402286CE85884397C0FA1FE78040FDB8
:104250009C4023928700B727002083A7C781014590
:104260008DCFB727002083C7C7B34945958B95C726
:104270006C001305D030EF903119B247014593F728
:10428000070F81CFB727002083A787848D45054579
:10429000944303D64700EFA0D004B2502254925466
:1042A0000259F24945618280B727002083A74784DD
:1042B00091CF03D647008C43411106C697C0FA1F21
:1042C000E78000F6B24001454101828009458280C5
:1042D000B727002083A747848DC7B727002003A7EF
:1042E000C784894705C3035647000C43411106C6DE
:1042F00097C0FA1FE780C0F2B24081473E85410176
:10430000828089473E858280797106D622D426D262
:104310004AD04ECE52CC8D4763FCA7008944B250A0
:104320002254268502599254F249624A456182809C
:10433000372900200347499FC144E312F7FE930742
:10434000F5FF9309499F93F7F70F8546AE842A84BA
:1043500003CA29001309499F63EAF6068DE19945CE
:104360002800EFD0DFDCB729002003C589B39145D1
:1043700023018900EFC04F8635E481444DB71946CB
:104380008145280097C0FA1FE780A0F019462C004D
:10439000268597C0FA1FE780E0F549F11946930595
:1043A000F00F280097C0FA1FE780A0EE19462C00F6
:1043B000268597C0FA1FE780E0F32DF11946A68500
:1043C000280097C0FA1FE780A0E571BFE31DE5F85C
:1043D00003A5C9002C00EF70C046AA8449D52381EB
:1043E000490135BF2800EFE06FE6AA840DED930583
:1043F00071001305F041EF70B16483447100B5FCA6
:104400008D47E31CF4F64545EFE0BF8B3DD5B7770C
:104410001800938707A03306F50203C589B39145B9
:10442000EFB05FF4EDBD23014901D5BDB7270020F2
:1044300083C7C7B3918B8DC3372500204111130566
:10444000058406C6EFD01FCEB240B72700207D57A7
:10445000239DE79E4101828001456FD0BFCCB727E5
:1044600000207D57A38DE782B72700207957238D41
:10447000E782B7270020238C07A8B7270020239EB8
:104480000782B727002023A20784B727002023A68E
:104490000784B727002023A4078437470500B727E0
:1044A00000209387078E1307876798C33747050057
:1044B0001307E7D3D8C3374705001307278E98C7DC
:1044C000B7470500372700209387C79E2320F7842E
:1044D0008280411126C2B724002083A7C48106C66A
:1044E00022C48DCF2A840D45EFB0CFDDAA8505C14A
:1044F000930700FD2300F5008D47A30085002301ED
:10450000F50083A7C48103C50700EFB0AFEA19C463
:104510002244B240924441016FF06FBAB24022444B
:10452000924441018280797152CC372A002083273E
:10453000CA814AD006D622D426D24ECE56CA0149C6
:10454000B1C703C91700B72400208547AA899384FF
:10455000449F6307F90483C74400054985EB0D4573
:10456000EFB04FD6AA8505C1930700FD2300F500E3
:104570009147A30035012301F5008327CA8103C5B4
:104580000700EFB02FE3EFF08FB30549B25022548C
:104590004A8592540259F249624AD24A4561828060
:1045A000B727002083A74784D28A85E30145EFE03F
:1045B0004FF12A8601CAB727002003C587B3894572
:1045C000EFB0DFB883A7CA8181A8944303D6470020
:1045D0009305E1000545EFD01FC069D98347050069
:1045E000858BE9D70545EFE0CFED9307B0032A842B
:1045F00063F0A704B727002003C587B35D661306E1
:1046000006708945EFB01FD6B7270020130444FC7D
:10461000239E87828327CA810947A380E70083C737
:10462000440081C72382040095B74E855D35B9BF2C
:10463000130600643306C502B5BF411122C42A84A3
:104640000D4506C6EFB00FC805C5930700FD230052
:10465000F500CD472301F500A30085002244B727CC
:104660000020B240AA8503C5B78341016FB08FD443
:10467000B24022444101828083564500011189677E
:1046800006CE22CC26CA138667002A876399C60005
:104690001C47014583C50700EFF04FC23DA81386B4
:1046A00087006397C6001C47054583C50700EDB723
:1046B000138697006395C602B727002083A7C7819A
:1046C000014595C71847034507006311050E0547C7
:1046D000A380E7000545EFA02038054509A813860B
:1046E000A700639BC6001C4703C507002D3DF24091
:1046F0006244D2440561828013866703E38AC6F868
:1047000013867703E381C6FA138687036392C60A8A
:104710001C45372400201307E00F83C4070083479C
:10472000A4831304A483638EE7021307F00F638648
:10473000E7021145EFB00FB9AA8505C1930700FD47
:104740002300F5008947A30095002301F500A3018C
:10475000050003450400EFB0EFC5F9572300F4004E
:10476000ADBFB727002003A7C7813E84014541D3D1
:104770008DEC85447D4523059100EFE08FD4231611
:10478000A10013050002EFE0CFD38327C481A30566
:10479000A1001307B100A380970074001306A100C5
:1047A00085450545EFA0A0330DBF26851D3335B7E0
:1047B00013869703E389C6F21386E7036397C6005F
:1047C0001C45094583C50700C1BD9387F703014513
:1047D000E39FF6F01C4703C5070005E96C001305CD
:1047E000D030EF906142B247414793F7070FE3861D
:1047F000E7EE9305B10013056031EF90E14003450A
:10480000B1008545EFA0202EC9BD053DF9B5B727FC
:10481000002083C7C7B3411106C6958B99CB3725B6
:1048200000201305058EEFD05F8F4D45B24041014A
:1048300082800145EFD07F8E0145CDBF03C70500C3
:10484000937625009377D70F99C2936727001318A3
:1048500085011358884113F7F7076354080013E7DD
:104860000708937685009377770F99C2936787003F
:104870001377050293F6F70D19C393E60702238019
:10488000D500634508009377A50281CB83470600D6
:1048900093E7C7002300F60082807DFD8347060072
:1048A000CD9BCDBF2D456319071403C805000947EB
:1048B0006310E814C84103471500034505002207AB
:1048C000498F42070D654187930825A0630B170B9D
:1048D000011122CC26CA4AC84EC606CEBE89B6846D
:1048E00032842E8963CEE800930705A0630DF7029A
:1048F000130515A06300A706239004000545B5A085
:10490000930745A06309F7086348F706130565AAEE
:10491000E314A7FE85472390F600DC4583C7070014
:104920002300F60091A0C84597C0FA1FE780809940
:10493000420541814E86637335012A862390C40067
:10494000420641828325C900228597C0FA1FE7806D
:10495000208D19A8DC4583D707002390060123008A
:10496000F600A183A300F6000145F2406244D24460
:104970004249B2490561828099472390F600194661
:10498000D1B785472390F600DC45014583C7070072
:104990002300F6008280DC45A9CB21472390E60066
:1049A00003D707002300E60003D707002183A300F5
:1049B000E60003D727002301E60003D72700218361
:1049C000A301E60003D747002302E60003D7470010
:1049D0002183A302E60003D767002303E60083D701
:1049E0006700A183A303F60041B723900600ADBF83
:1049F0002390060005458280828083C80500894790
:104A00006394F816DC41797122D406D626D24AD0B6
:104A10004ECE52CC56CA03C8170083C707002E8457
:104A200022083368F80042088D6713580841138341
:104A300027A0630C68102A8A3A89B684B285634C31
:104A40000301138707A0630BE802938717A0630194
:104A5000F80A854711A8138737A06303E80C13876A
:104A600067AA8D47E317E8FEB250225492540259C8
:104A7000F249624AD24A3E8545618280484432C644
:104A800097C0FA1FE7800084420541819D47E36D8E
:104A900025FDB72A0020938A2A8583C70A00B30917
:104AA0009900B24563D43701B5477DBF4844268697
:104AB000C2094A9597B0FA1FE780807603C60A00BC
:104AC000484493D9090105063306364181454E9580
:104AD00097B0FA1FE780E07BB727002083A74785C0
:104AE00099E3814751B79C438145E5DF52853DA05D
:104AF000AD47E31B09F6E39916FB8347160083468F
:104B000006005844A207D58F2310F700B7270020CE
:104B100083A74785F9D79C438545E1D78297D1B7CD
:104B2000AD47E31309F49947E390F6F84844194672
:104B300097B0FA1FE780C06EB727002083A747858C
:104B4000CDD39C43D9DF8D4555B7AD4711FF854780
:104B5000E39CF6F40347060093070008E3E6E6F05B
:104B6000DC452380E700B5BF85473E858280B727B7
:104B7000002023AA0784B7270020A3890784B7272A
:104B8000002023890784B7150020B707A00093856C
:104B9000457E938707059CC1B707E803DCC137F65C
:104BA0000600B71700209387076F1306C6C1D0C34E
:104BB000B71E002037F606000947938EFE7D1306C8
:104BC00006BF371E00202380EE00130ECE7DD0C717
:104BD00023AED70137230020B71800203718002054
:104BE0003715002037F60600B7FE06008546130687
:104BF00006C02300EE009388087E23AEC70313038C
:104C000003851308E87D1305D57D938E8EC037FE8E
:104C100006002380E8002380E7002388E700238044
:104C2000E7022388E7022380E7042300E8002384C7
:104C3000D70023950700D0CB238CD700239D0700F6
:104C400023A2D7032384D7022395070223A60702B2
:104C5000D0DB238CD702239D0702231003002300FF
:104C6000D500130E8EBF23A2C7052388E70423AE09
:104C700017052380E7062388E7062380E708B7F8AF
:104C8000060037F706001307C7BF938888C123A221
:104C9000E7082384D7042395070423A66704F0CBF1
:104CA000238CD704239D070423A217072384D70648
:104CB00023950706ECD7F0DB238CD706239D070648
:104CC00023AE07072384D7082395070823A6A70840
:104CD00037570500B7170020938707781307478ACF
:104CE00098C3375705001307A79FD8C323A407000D
:104CF0008280A54763ECA710B7E706009387C75FDC
:104D00000A053E951C41011122CC26CA06CE4AC88E
:104D1000B2842E8482879307800F63F9B7006145C0
:104D2000F2406244D2444249056182803719002032
:104D30009307096FC8571309096F09C997B0FA1F7C
:104D4000E780803EB72700202389078413061400DC
:104D5000916593850571328532C697B0FA1FE78059
:104D6000602E2326A90245DD3246814597B0FA1F01
:104D7000E78020520325C9022286A68597B0FA1F34
:104D8000E780004AB727002023898784014549BF6F
:104D90008947E396F5F803570600B72700202398C4
:104DA000E784EDB7A147E39CF5F6371500202146CF
:104DB000A6851305457E97B0FA1FE7806046F9B7D0
:104DC0008547E39EF5F4B71500209385056FD04D18
:104DD0009385850203C50400EFF05FA645BF8547B4
:104DE000E39FF5F2B71500209385056FD05D93859D
:104DF0008504CDB78547E394F5F203470600B7175E
:104E00000020A38EE77C59B7094519BF0945828068
:104E100005476302E5044111AA8706C62E8581CFA6
:104E200011476383E70425476388E7048947B24055
:104E30003E8541018280B717002083A5C77189474D
:104E4000FDD5B727002003C6278597B0FA1FE78056
:104E5000203D8147E9BFB727002083D707852390EE
:104E6000F50081473E858280B71500202146938555
:104E7000457EEF90416BF1BFB717002083C7D77D08
:104E80002380F500F9B7B72700209387378503C73C
:104E9000070015E305472380E700058909CDB7160C
:104EA000002037150020938606784146A545130556
:104EB000056F6F30406D01458280011106CE22CC16
:104EC0000546638CC50211460944639EC5023EC671
:104ED0003AC436C2EFD0EFC22A8492462247B24784
:104EE0001DE13E86BA853685EFD00FB8EFF03F92D0
:104EF000EFF0CFD3EF60F06F39A0EFD08FC02A84EE
:104F000019E1EFF0DF902285F24062440561828072
:104F100079714ECEAE896C0022D426D24AD006D604
:104F20002A89B284EF00707A2A840DE1CE854A8501
:104F3000EFC05F882A8419E93245B7160500268735
:104F40009386667A2D468145EF10C0122285B250B5
:104F5000225492540259F2494561828079714ECEB1
:104F6000AE896C0022D426D24AD006D62A89B284D1
:104F7000EF00B0752A840DE1CE854A85EFC0BF9160
:104F80002A8419E93245B726050026879386C68804
:104F90004D468145EF10000E2285B25022549254A6
:104FA0000259F24945618280397126DAAE844C009B
:104FB00022DC4AD84ED652D406DEAA893289368AF5
:104FC000EF00B0702A8431EDA6856303090283D710
:104FD00004002C002314F10083D724002315F100D2
:104FE000930720302316F100930780022307F10076
:104FF0004E85EFC00FF92A840DE55946A6851305A5
:10500000A1002304210197B0FA1FE7806021124517
:10501000B716050052879386067525462C00EF10BB
:1050200060052285F2506254D2544259B259225A34
:1050300021618280797126D2AE846C0022D44AD05C
:105040004ECE06D6AA893289EF0030682A840DE157
:10505000A6854E85EFC0EFF72A8419E93245B716C9
:1050600005004A879386467C3546A685EF1080006A
:105070002285B250225492540259F24945618280ED
:10508000BD47638CF50663E9B702A5476387F5065C
:1050900063EDB7009947638CF5049D47638FF50472
:1050A0009547638CF50401458280B5476387F50415
:1050B00063E1B704AD47F5B7DD47638EF50263EAF8
:1050C000B700C947638BF502D9476386F502C54728
:1050D000C9BFF5476383F50263E4B700ED47D1B775
:1050E00093072005638BF5009307200D5DBF4845AE
:1050F00082800841828008458280484182809307EF
:10510000F00F630EF506011126CAAA8413050002EA
:1051100022CC4AC84EC652C456C206CE3A89B68977
:10512000B28A2E8AEFA01F9A2A844D4515C893078C
:1051300000FB2300F400A3005401231144012302C7
:10514000340113058400614663050902CA8597B0DE
:10515000FA1FE780E00CA2852685EFA0BFA50145D8
:10516000F2406244D2444249B249224A924A05611D
:105170008280814597B0FA1FE780A011E9BF0945F9
:105180008280011122CC06CE2A842306B100A30618
:10519000C100EF50A06C15C18346C500B7270020A1
:1051A0002147938787B3639EE60003C567007800B5
:1051B0009306E0070146A2859937F24062440561F3
:1051C000828078009306E0070146A28503C5570058
:1051D000E5B7930700643306F6026FB06F8C05C91C
:1051E0000347050085469307270093F7F70F63F001
:1051F000F602411122C42A843A8506C6EFB0CFA434
:10520000FD572300F400B240224441018280828095
:10521000035705009307000B6313F702834745000C
:105220004947639CE7000347150185476399E700F9
:105230000355250085456F3090646D47C5BF82805A
:1052400001112314B1006C0022CC26CA4AC806CE34
:105250002A89B6842315C100EF0030472A840DE166
:105260002C004A85EFC02FC82A8419E93245B716A9
:10527000050026879386E66915462C00EF00905FAF
:105280002285F2406244D2444249056182807971AC
:10529000930720302314B1002315C1002316F10019
:1052A0002C0093078002014606D62307F100EFF099
:1052B000BFCFB25045618280C177797185073EC406
:1052C000894726D22316F100AE84930780024C0052
:1052D00022D44AD006D62A892307F100EF00F03EF7
:1052E0002A840DE12C004A85EFC00FD82A8419E9E1
:1052F0001245B726050026879386468345462C002F
:10530000EF0050572285B250225492540259456101
:105310008280B28605466FF03FC9797126D2AE848D
:105320006C0022D44AD04ECE06D6AA893289EF002C
:10533000D0392A840DE1A6854E85EFC0EFB12A84CD
:1053400019E93245B71605004A879386A6630D46CC
:10535000A685EF0030522285B25022549254025951
:10536000F249456182807971930720202314B100AE
:105370002315C1002316F1002C009307800201467B
:1053800006D62307F100EFF03FC2B250456182809C
:10539000011122CC06CE2A842EC632C436C2EF506A
:1053A000E04B0DCD0345C500B7270020A1469387EC
:1053B00087B312472246B245631CD50003C5670078
:1053C000B2862E86A2856244F24005616FF03FD31B
:1053D000B28603C557002E86A285F5B7F240624417
:1053E0000545056182806FF0BFB26FF07FB26FF04C
:1053F0007FC46FF03FC479714ECEAE896C0022D469
:1054000026D24AD006D62A89B284EF00102C2A84EC
:105410000DE1CE854A85EFC0AFBD2A8419E932453A
:10542000B716050026879386267E3D468145EF0008
:1054300070442285B250225492540259F249456177
:105440008280B28601466FF03FB6011122CC2E84D5
:105450006C0026CA06CEAA84EF003027DD47630A17
:10546000F500930710102314F400A2852685EFC0E1
:105470008FC2F2406244D2440561828023940500C9
:1054800083D7850099E36FF07FAD09458280FDB732
:10549000B727002003C7E788854763F9E7020111B2
:1054A00022CC2E846C0026CA06CEAA84EF00F021FE
:1054B00009E9930700102314F400A2852685EFC0A4
:1054C0008FBDF2406244D24405618280594582809A
:1054D000B727002023ACA7848280B727002023AE03
:1054E000A7848280011122CC26CA06CE2A84AE84EB
:1054F000EF50C036A6852285EFB03FE10DE9228549
:1055000023169100EF5080351DC18346C500B72793
:1055100000202147938787B36390E60203C56700A5
:1055200078009306F0070146A285EFF05FBDF240D8
:105530006244D2440561828003C55700D5B701118A
:1055400026CA06CEB68422CCDD4663E2B608D9462A
:1055500063FED50AA5466381D50A63EEB604954677
:10556000638CD50899466387D50A054441687D1840
:10557000631606093AC6EFB01FDD33068540324791
:1055800042064182420441803305C4004205BA8587
:10559000418132C6EF30D03FAA8749C181C432462B
:1055A0002390C400B30580406244F240D2443E855B
:1055B00005616FA0CFC4C5466380D504C9460D44BC
:1055C000E395D5FAC167FD17E31EF6FA65B7F54610
:1055D0006380D50463E4B600ED46D5B79306200595
:1055E0006388D5029306200DE391D5F8C167FD17B6
:1055F0000D446319F600BDBF09448DBF9306200D0D
:10560000E392D5F8310642064182ADBF15445DBF35
:105610000D444DBFC167FD171D447DB7F240624484
:10562000D24405618280011122CC26CA06CE03C66F
:1056300045002E841307000281469945AA8401374C
:105640002AC629CD8357040003464400930554001D
:105650002310F100835724002311F10089472312FE
:10566000F100930780022303F10097B0FA1FE7804F
:1056700020BB834744008A8526852314F100EFC0B0
:105680004F892A8411C5324597B0FA1FE780C0A917
:105690002285F2406244D244056182804D44CDBFF0
:1056A0005D7186C6A2C4A6C2CAC04EDE8947630623
:1056B000F600C14709446319F6040144B1C52E89B7
:1056C0004C0832C6B689AA84EF0030002A843246DC
:1056D00005EDC1778507CA851305D1013ECC230EA0
:1056E000C10097B0FA1FE780A0B32C082685253F9C
:1056F0002A8419E95245B71605004E879386666FCE
:105700001D462C08EF0010172285B640264496440B
:105710000649F25961618280797122D436844AD077
:105720004ECE52CCB2892E8A3A8981461307100296
:105730002286D94526D206D6AA8411352AC629C181
:105740002286CA85231481002312410123133101CB
:1057500097B0FA1FE780C0AC4C002685EFC06F9E63
:105760002A8411C5324597B0FA1FE780E09B228555
:10577000B250225492540259F249624A45618280E1
:105780004D44F5B7011122CC26CA06CE4AC8DD47E2
:105790002A84AE84638DF5028147035504006C00B2
:1057A0002306F100EFC06F9D0545638DA4080345F6
:1057B0008400B165938505B8EFA0BF83E547230159
:1057C000F400B7270500938707975CC09DA803479F
:1057D00055013149B2863306270318499C42329756
:1057E0001043E31BF6FA83D7460003564700E31540
:1057F000F6FA8C46084797B0FA1FE780A0AF49DD5C
:105800008347540103474401850793F7F70FA30A21
:10581000F40063FFE702B387270318480355040029
:10582000BA97984783D6470003D6270083D5070049
:10583000E5353DF103458400B165938505B8EFA0DA
:105840004FFB5945F2406244D2444249056182808F
:105850008347640199B7011122CC26CA06CEDD47E1
:105860002A84AE84639BF50603550500EFB0BFADF7
:105870000356C40183562401035744016D162A962A
:1058800042064182B307D640C207231EC400C1832B
:1058900063F0E7089305C5FF3308F740635BB80280
:1058A000BA96918EC206184C835504010355040024
:1058B000C1823E97953515E103458400B165938516
:1058C00005B8EFA00FF35945F2406244D244056198
:1058D00082806D1593160501F9B7814703550400C1
:1058E0006C002306F100EFC04F890545E38EA4FC50
:1058F00003458400B165938505B8EFA08FEFE547B8
:105900002301F400B7270500938707975CC065BFA4
:105910008547E9B7397126DAAE842C0022DC4AD8F3
:105920004ED606DE2A89B2894D232A8421ED4A8586
:10593000EFB07FA183D644006D1563C5A600931612
:105940000501C182984403D6240083D504004A850A
:10595000EFF09FDC2A841DE53146A6850808230662
:10596000010097B0FA1FE780A08B83D7240022455F
:10597000B72605004E879386E68F5D466C00231E92
:10598000F100CD2D2285F2506254D2544259B259C1
:105990002161828041B7BDBF797126D206D622D45B
:1059A0004AD04ECE52CC56CA5AC88944C5C159CEE7
:1059B0002E842A89BA8A368B328AEFB0DF98930513
:1059C00044008147711503D705006352A70A850774
:1059D00093F7F70FB105E318FAFE8A854A85F5219A
:1059E000AA842DE531453305AA029165938515708A
:1059F000CD4497A0FA1FE780E064AA8921C9314607
:105A00003306CA02A28597B0FA1FE7806081184466
:105A10008356440003562400835504004A85EFF062
:105A2000BFCFAA841DED0245B726050085475687DE
:105A30009386E68F5D464C002302F1004EC4230698
:105A40004101A3060100230761012D25B250225414
:105A5000268502599254F249624AD24A424B456124
:105A600082804E8597A0FA1FE780006CC5B7ED4491
:105A7000F1BF79714ECE37F60600AE89C16526D2E8
:105A80000147AA848946130646C2FD15054522D45E
:105A900006D64AD0EF10301A054431CD2A891307B3
:105AA000300281461146F5452685EFF05FA92AC6EA
:105AB000554431C18357A900CE8601462314F10015
:105AC00091472315F10085472300F500B2472C00CC
:105AD0002685A38007003247FD572301F700324790
:105AE000A301F700EF10F00A2A8411C5324597A0F0
:105AF000FA1FE78060632285B25022549254025903
:105B0000F24945618280411106C6EFF06FD719C591
:105B1000B240410117A3FA1F67000361B24041017F
:105B20008280011106CE2AC6EFB0CFE73245B727F3
:105B3000002023AC0784B727002023AE07849145BB
:105B4000B7270020A38CA7B2EF30E05EF2400561DA
:105B50006F20F0387971939705014AD006D622D488
:105B600026D2C187014963DE070AB727002003C593
:105B700097B32E89EF901FFC2A844DC1034705007F
:105B80009307000A6319F70885474C08A305F1003D
:105B9000EFB06FEEAA840DED834761017147637921
:105BA000F708138717FE1377F70F9306000263F8C1
:105BB000E608858BD5CBB727002083A78785994436
:105BC00081CB035524001306B1004C088297AA84A8
:105BD0008347B10099C7084409C597A0FA1FE78019
:105BE000A05495E05247B7070001938707F07D8FD7
:105BF000B707120093870710630FF700034761018F
:105C0000ED47631AF700035524008545EF30204720
:105C1000CD476388F4002285EF90BFE5A167334943
:105C2000F900B25022544A8592540259456182804B
:105C30003707301405073357F700058B3DDB37274F
:105C400000200327C78549D70347510151F3230695
:105C5000F10099472308F100035524006C00231735
:105C60000100EFB0DF85ADB7B727002083A7C78558
:105C70009DC3035524001306B1004C08829729D90F
:105C8000AA8483475101A9F7834761012308910042
:105C90002306F100D1B79944EDB7397122DC26DA39
:105CA00006DE4AD84ED652D456D25AD0A5472A84B8
:105CB000B2846399F5108347450203570600835A5F
:105CC000260085072302F5029307F7FFB387FA0240
:105CD0005442C207C183B69703C9170083C70700A0
:105CE0008346C50022093369F90085476390F602AF
:105CF00033075703231006008149014A130B35016E
:105D0000931A070193DA0A0163E15907C167FD1786
:105D10006302F90C83570401637EF90A05094209FD
:105D20008346C4001359090123172401054703556D
:105D300004009305E400639FE6002315F100930738
:105D400020302316F100930780022314210123073A
:105D5000F1002C00EFB0FFA203458400B1659385EC
:105D600005B8EFA00FA95945BDA083D62400DC409B
:105D700083452401ED1613865900C206C1823E9662
:105D80005A85EFB0AFC705C9630C3A01C84003D6C6
:105D90002400B3053501529597A0FA1FE7804048CB
:105DA00083D724003E9A83D70400420A135A0A017B
:105DB00085072390F40083D72400BE99C20993D9A4
:105DC000090199B703474600A9476310F7028347C3
:105DD000450281CF0145F2506254D2544259B25922
:105DE000225A925A025B2161828083462401130960
:105DF000340137F506004A8689451305C5C1EFB061
:105E0000EFBF19C10545C1BF8346240137F5060020
:105E10004A868945130505C2EFB04FBE65F5834636
:105E2000240137F506004A868945130545C1EFB0C0
:105E3000EFBC69F98346240137F506004A86894597
:105E4000130505C0EFB08FBB55FD03C74400BD4728
:105E5000E3EAE7FAA56793874712B3D7E700858B94
:105E6000D5D38347440285072302F40203D92400D3
:105E700071BDB727002003C607B4B727002003A7CA
:105E8000078681476315F600814636858280BA868B
:105E900013078702835587FDE389A5FE850793F7DE
:105EA000F70FCDB7011106CE2EC6E13701CD8347DE
:105EB000A500B245138717006396E50093F707F82E
:105EC0002305F500F24005618280011106CE2EC641
:105ED0004D3705C5B24591C188C183478500130779
:105EE000E00F5D456388E7001307F00F014563830A
:105EF000E7005945F240056182800945E5BF41113F
:105F000022C42A84210506C626C24AC0EFF02FAD5E
:105F100083472400A51793F7D70F91EB0347C400DD
:105F200085476310F7061C4881443149A9E3FD57B2
:105F300023010400A304F400230204021305C40097
:105F40002244B2409244024961468145410117A36F
:105F5000FA1F67000334B38724033E95084509C53B
:105F600097A0FA1FE780401C850493F4F40F834741
:105F700044010848E3E1F4FE97A0FA1FE780C01A45
:105F80007DB7084C75F965B7411122C4416406C656
:105F900026C29307E4FF630CF500AA8491EDD13D7E
:105FA00019E51305F4FFF13519C123109500B2402E
:105FB000224492444101828085476394F504EFF0C6
:105FC0005FEB2A846DD5FD572310F50083478400CD
:105FD0001307F00F6384E7021307E00F638BE700FA
:105FE000834624000345940001475146A685EFF0FF
:105FF0000F9122852937FD572304F400230504005F
:106000007DB78947E395F5FA8545EF40902845F13E
:106010002685EFF01FE62A8455F951BF39C9034799
:1060200085009307F00F6306F704011122CC06CE1A
:106030002A848346250083550500034595000147C2
:106040005D46EFF0CF8B03472400E1476319F7006B
:10605000035504006C0023060100EFB01F92F957AE
:106060002304F4002285EFF09FE9F24062440561C9
:10607000828082809307F00F6306F706011122CC1D
:1060800026CA2A844EC6AE84B689AA8593068500A0
:10609000376505004AC852C43A89328A1305C501DA
:1060A000794606CEEFF0EF92A304240123014401C8
:1060B0002322340185C01305C4006244F2404249E2
:1060C000B249224AA685D2446146056117A3FA1F48
:1060D00067000315F2406244D2444249B249224A61
:1060E000056182808280B72700202382A786828074
:1060F0009547639CF506834745028546850723023D
:10610000F50283570600584203462600FD17C207D2
:10611000C1836318D6048A07BA9703C7170083C7D9
:1061200007002207D98F0357E50063F9E7044111FF
:1061300006C622C485072316F5002A849305C500E8
:1061400003550500EFB02FDA03458400B165938550
:1061500005B8EF901FEAB2402244D9473E8541017D
:106160008280C946B387D70245BF83464600294788
:1061700085476396E6000347450211C381473E8584
:1061800082809D476392F506834745028356E5006A
:1061900085072302F502835706005842FD178A0738
:1061A0003E978347170003470700A207D98F01478F
:1061B00063F6D704411106C622C485072A84231634
:1061C000F5009305C50003550500EFF0CFC5034565
:1061D0008400B165938505B8EF90BFE1B2402244D9
:1061E00059473A854101828083464600A9470547C1
:1061F0006396F60003474502133717003A858280FD
:10620000411122C406C626C2B5472A84639BF50401
:1062100083474502B28485072302F5020355050032
:10622000EFB06F9283D704001307F5FF014563C5F4
:10623000E7020357E400035504009305C400BA972E
:106240002317F400EFB0EFD803458400B1659385C0
:1062500005B8EF901FDA5945B240224492444101FB
:106260008280034746009D470545E317F7FE034537
:10627000440213351500CDB7C547639EF506835715
:10628000060003572600FD17B387E70203474502C0
:1062900005072302E5025842C207C1833E978347A0
:1062A000370003472700A207D98F41677D17639501
:1062B000E70081473E858280138717002316E5009B
:1062C0000357E500E3F7E7FE411122C49305C5003B
:1062D0002A840355050006C6EFB00FD90345840094
:1062E000B165938505B8EF90DFD0B2402244D9471D
:1062F0003E85410182808346460029478547E39BCE
:10630000E6FA0347450255F775B7011122CC26CAB4
:106310004AC852C406CE4EC683C7250015472A8AEE
:10632000AE8432843689639DE7043686A28526854D
:10633000EFF01FDCAA8955E985476318F40A034783
:106340004900A9476301F70203C594004A878546BF
:106350000146D285EFE0BFDA19E585454A85EFE0D1
:106360003FD21334150083C6240003C594000147AF
:106370006946D285EFE0BFD82685EFF05FB851A01F
:106380001D476398E7003686A2852685EFF07FDFFC
:1063900055B725476398E7003686A2852685EFF036
:1063A000DF8F49BF35476398E7003686A28526858B
:1063B000EFF01FE541B745476398E7003686A285B1
:1063C0002685EFF07FEBBDB75D47639FE70003C70E
:1063D000C50085473686A2852685631DF702EFF046
:1063E0006FBA8547631BF5048549A5476317F40217
:1063F000835709009DE30544E38709F6D947E39DE8
:10640000F9F62285F2406244D2444249B249224A16
:1064100005618280EFF02FC4E9B703C594004A8775
:10642000A2860146D285EFE09FCD71F5A2854A850F
:10643000EFE01FC513341500C1B70544D9B7397152
:1064400022DC06DE26DA4AD84ED652D456D283D77C
:1064500005001944B1E783C925002A89328A938748
:1064600059FE93F7D70FAE84DDE7B727002083C628
:1064700047861307F00F938A478619446382E60222
